:020000040800F2
:1000000000200010290003085D5D0108E12B0008B5
:10001000595D0108555D0108515D010800000000AF
:100020000000000000000000000000004D5D01081D
:10003000495D010800000000455D010885220008B7
:100040009100030891000308910003089100030840
:100050009100030891000308E12C00080D2E000810
:10006000D12D0008952D0008592D0008C98C0008D5
:10007000B98C0008A98C0008998C0008898C0008AC
:10008000758C0008618C000891000308910003083A
:10009000BD87010891000308910003081D2D000889
:1000A00091000308910003089100030891000308E0
:1000B00091000308910003089100030891000308D0
:1000C00091000308910003089100030891000308C0
:1000D000910003089100030891000308B922000869
:1000E000A52C000891000308355D01089100030864
:1000F0009100030891000308910003089100030890
:100100000000000000000000000000009100030853
:10011000910003089100030889DC01086DDC0108E7
:100120004D8C0008398C0008258C0008118C0008C3
:10013000FD8B000891000308000000000000000093
:1001400091000308910003089100030800000000DB
:10015000000000000000000000000000000000009F
:100160000000000000000000910003089100030857
:1001700091000308000000000000000000000000E3
:080180000000000091000308DB
:1001880090ED057A90ED004AD0ED066AD0ED014A6F
:10019800D0ED047A90ED035AD0ED025AA4EE007A1D
:1001A800B0EE406AB0EE470AB0EE667AA4EE867A00
:1001B80067EEC07AA5EE407AE5EE867A80ED057A9C
:1001C800C0ED067A704700BF38B50B4C23688BB179
:1001D8005A68821A002A054604DA0BE05A68AA1AF5
:1001E800002A07DB9A68226018461A689047236835
:1001F800002BF3D138BD00BF583100200D4B04212E
:100208000022890710B4027203F13C0402D519795F
:10021800815401329C4203F1140308D0082A06D005
:1002280099798907F3D49C4203F11403F6D15DF858
:10023800044B70470028030810B4104C04232146CF
:1002480013F001034FF0000201F1140108D101324B
:10025800042A0ED08B7913F0010301F11401F6D0B2
:1002680002EB820204EB82025DF8044B13790370FF
:10027800704703705DF8044B704700BF00280308FF
:10028800436A8269D154436A0169826B01338B42A4
:1002980028BF002343623AB370B4EFF311835022AE
:1002A80082F31288866B3268D20704D5DBB283F3F7
:1002B800118870BC7047716869B9D0E909429442E5
:1002C80018D085691544F56018D9A21A726084623D
:1002D800002280F85420326842F00102DBB232601A
:1002E80083F3118870BC7047026D136843F0800374
:1002F80013607047012280F85420D7E70469A21AD6
:1003080072608162E4E700BF034610B4446BD968A9
:10031800406954B15A6C8C1A013A005D5DF8044B7F
:1003280008BF0A46C0B25A6470471A6A805C013234
:100338008A4228BF2246C0B21A625DF8044B704751
:10034800836B13B190F854007047D0E90903181A69
:10035800B0FA80F040097047D0E909120369914268
:1003680038BFC9188A1A816B013B19B149680A4418
:100378009A4201D2981A704700207047436B43B1E4
:10038800426C5B689A4291BF981AC0689B1AC01861
:100398007047D0E907239A422FBFD01AC068801847
:1003A800C01A70472B2303732A2383700023837595
:1003B800704700BF03682DE9F041DD691DB12B4688
:1003C800BDE8F0411847002A174611DD04460E46DD
:1003D8000F4400E023689B68204698470028F9D01E
:1003E800236816F8011B1B6820469847BE42F1D1C6
:1003F800BDE8F08100232322027043708370C3702C
:100408007047152303701623C370172383712D2398
:1004180043702E2303712F23C37170470028F0B453
:1004280003DA2D230B7040420131092804464FF0AE
:10043800010307DD03EB83035B00B0FBF3F2092A3A
:10044800F8D883B10F48A0FB0326B4FBF3F2092ABE
:1004580002F1570C02F1300709DD03FB1244F308DF
:1004680001F801CBEFD100230B70F0BC704703FB00
:100478001244F30801F8017BE5D100230B70F0BCAE
:10048800704700BFCDCCCCCC884270B44FF001048B
:1004980042D301FB04F4B0FBF4F58D42F9D2ECB180
:1004A80042BB092D04FB150005F1570605F1300282
:1004B8000EDDB4FBF1F403F8016B7CB1B0FBF4F58D
:1004C800092D04FB150005F1570605F13002F0DC93
:1004D800B4FBF1F403F8012B002CEFD100221A70C1
:1004E80070BC704703F8016BB4FBF1F4002CF5D035
:1004F800B0FBF4F5092D04FB150005F1370605F1ED
:100508003002EFDCB4FBF1F403F8012B002CEFD13F
:1005180000221A7070BC70470546002AEAD1C0E76D
:100528002DE9F04714461D46064600234FF47A721B
:10053800204629462FF0A8FBDFF840814B4A4C4F54
:1005480088FB00310144C31782FB002CC3EB611107
:1005580088FB012887FB00278444464AC3EBEC2C20
:10056800C1EB011E82FB0C29A0EB8E0E0744424A08
:1005780086F806E0C3EB27474FEAEC7E08EB010A52
:10058800CEEBA90E82FB07824FEAE1780EEB4E0E06
:10059800C8EB6A18ACEBCE0CC8EB0818DFF8E0E043
:1005A80086F804C0A1EB880171718EFB0010F91761
:1005B800C1EBE21240F2B55101FB1272C3EBE050FD
:1005C800B2F5896F4FEA80073CDA40F2DA239A42A3
:1005D80042DCB2F5B77FB4BF4FF0000E4FF0010E0A
:1005E8004FEA4E09DFF89C8009EB0E0308EBC303C2
:1005F8001FFA8EFCD88A09EB0E0108EBC1011631EF
:100608000B2301E031F8020D904218DD013BF9D1CE
:10061800CE44012338F83E00B37007F2B2770132B6
:10062800121ABC44F270A6F800C0204629464FF4BE
:100638007A7200232FF028FB3281BDE8F08701335E
:10064800DBB2E9E74FF0030CE64640F29650DFF8DC
:1006580034804FF00609CEE74FF0020CDFF8248013
:10066800E64640F229404FF00409C4E7C5B3A29119
:1006780007452EC2ABAAAA2A73B06D168988888846
:10068800792D0311BC0D030803685A1C0260197008
:10069800704700BF2DE9F047089C2578002B80465D
:1006A80089460CBF4FF0200A4FF0300A661C25B36C
:1006B800002A26DD334601E0024698B113F8011BF3
:1006C800501E0029F8D1971E60B13D46013D5146A4
:1006D8004046C8476B1C002BF8DC257827EAE770F2
:1006E800013045B1041B29464046C847301916F861
:1006F800015B002DF7D1BDE8F087002A03DC28460E
:10070800F9E70020EEE7571EDFE700BFD0E9012335
:1007180000EB830101339342D0ED037A81ED040AA3
:10072800836004BF0023836000EB830393ED047AA6
:10073800036870EE277A9A42C0ED037A77EEC77A9B
:10074800C0ED037A0CDA013307EE103AF8EEC76A07
:10075800B7EE007A87EEA60A036030EE070A704704
:1007680007EE102AB8EEC77A87EE870A704700BFEF
:10077800D0ED057A90ED013AD0ED003AD0ED064A79
:1007880090ED024A90ED077A90ED035A90ED086AD1
:10079800D0ED045AC0ED067AF0EE406A27EE830ADF
:1007A800C0ED056AA3EEA60A80ED087AA4EE240A35
:1007B800A5EE470AA5EEC60A80ED070A704700BFF6
:1007C800D0ED007A90ED017A30EE670AE7EE007A14
:1007D800B0EE670AC0ED007A704700BF704700BFEF
:1007E8000A44914215D030B40139551E41F2210214
:1007F80011F8014F082380EA042004044CBF82EA60
:1008080040004000013B80B2F7D18D42F0D130BCAE
:1008180070477047E8B1E1B1F0B40E4B1B78002483
:100828000B2B0CBF4FF00E0C4FF0080C2346022781
:10083800012617FB036511F813204D5D0133DBB268
:1008480042EA0522634520F814201C46F1D3F0BC87
:1008580070477047000000204FF480538382704730
:10086800012380F84530704770B4D0E90041057B1A
:1008780042690223AB4063600B684FF6FE70034089
:100888000B60EFF31183502181F31288966B316866
:10089800C9071CD4706870B9D2E909418C4213D0D9
:1008A80095690D44F56017D81469611A71609062F2
:1008B800002182F85410326842F00102DBB2326043
:1008C80083F3118870BC7047012182F85410DBB2A1
:1008D80083F3118870BC7047611A71609462E7E70E
:1008E80070B40468037B2268022101FA03F31A42F8
:1008F80013D042690A495C2000FB02124FF6FE76CB
:1009080050685289C5680068296831402960C16803
:10091800D24392B20A40C260636070BC704700BFA5
:100928009441002030B40A4B1D7875B1094B002062
:1009380003EBC5051A6899885062D4682143D160D1
:10094800083323F8040CAB42F4D130BC704700BF25
:10095800744400207844002010B40268047B1168B5
:100968000223A340194209D00649406800240C70AC
:1009780001684FF6FE742140016053605DF8044B36
:10098800704700BF6C5D002070B5448806460D4670
:10099800C4F30B042246002128462FF0BFFD33691B
:1009A800094A934209D3094A934206D22246284665
:1009B8001946BDE870402FF097BC23B12146284660
:1009C800BDE87040184770BDE0770308DE7803087B
:1009D8002DE9F0478C4A8D4B12781C78D2070646D1
:1009E80048D58B4D012C00F091801ED3022C40F08D
:1009F8009B808849884A09881288884F914201D982
:100A080001241C70EB7AFBB12B89EBB1844B1B786A
:100A1800D3B11DF081F9002800F0E2802B7B8342DE
:100A28002CBF012300233B700FE0DFF8E8C17B4FA8
:100A38007C4CBCF800002288697B521A8242DFDABB
:100A4800EB7A0024002BDFD13B782A79632A07D878
:100A58007549022C087800F0B880002840F0A08082
:100A68007249AA7A9C4238BF1C460C70002A44D1AD
:100A7800BDE8F087DFF89CC1654DBCF80000BCF804
:100A8800021095F803E06A4F411A0029A4F1030205
:100A9800B8BF4942704597F80080D2B211D32F7879
:100AA80087420ED3012A45D9B8F1020F9AD15C4882
:100AB800604A007890800229CCBF00210121D180B2
:100AC80090E7B0EB4E0FEDDC012A40F28C80022952
:100AD800EADC0324514F524852494F4A1C70B8F17E
:100AE800020F4FF000033C7003700B80138089D114
:100AF800504A01219380D18084E7012C6BD0022CCD
:100B0800B6D10720BDE8F04726F080BC424A4149EB
:100B18001288687B0988121A914207DD414A1288B7
:100B28008A423CBF00241C703C4F6BE702241C70B7
:100B38003A4F67E70229B7DC95F800E090FBFEFE24
:100B48000EF1010EBEF1080FDFF8D4A0AA7869787B
:100B5800DFF8C490334C314FA8BF4FF0080E8AF825
:100B680000E01FFA8EFA11FB0AF112FB0AF2DFF815
:100B7800B8A0A9F8001092B200214FF06409B8F1AA
:100B8800020F228039701970CAF804108AF801908F
:100B98007FF452AF274A0121A2F804E0D18048E748
:100BA8004868301A244EB042C8BF4A703FF758AF61
:100BB800C2F16402214E00FB02F086FB0062C017FE
:100BC800A0EBA250643048704AE70028E8D101271A
:100BD8004E600F70ECE70820BDE8F04726F016BC21
:100BE80002233B7031E7032C7FF471AFB8F1020F99
:100BF8009AD10B4A0F4B12789A800229CCBF002158
:100C08000121D980054FFDE6454600207C4D002096
:100C1800F848002094370020804D00208C4D00209B
:100C2800364700207E4D0020844D00209459002036
:100C3800104B0020084B00207F9698006BCA5F6B12
:100C48000123102111224170427103720370037154
:100C5800704700BF2DE9F04F013083B0C3B2019354
:100C6800884C894E894DDFF838820A239B4612F05A
:100C780055FDDFF820C24FF4FA7A4FF0100E4FF40A
:100C88007A77DCF80430C3F30803002B40F0DD80EA
:100C9800EFF31183002B40F0D8802168AA6800BFC9
:100CA80023689942F9D1306807FB00F39A1AB2FB1E
:100CB800F0F207FB0121DCF80430C3F30803002B32
:100CC80040F08880EFF31183002B40F08380236885
:100CD800A86800BF22689342F9D1D6F8009007FBB4
:100CE80009F2101AB0FBF9F007FB03035B1AB3F51E
:100CF8007A7FE0D3BAF1010AC3D1019812F074FBEC
:100D08004FF47A7ADFF88CC157464FF0100EDCF8B2
:100D18000430C3F30803002B7BD1EFF31183002BBE
:100D280077D12168AA6800BF23689942F9D1306851
:100D380007FB00F39A1AB2FBF0F207FB0121DCF87B
:100D48000430C3F3080333BBEFF311831BBB2368E1
:100D5800A86800BF22689342F9D1D6F8009007FB33
:100D680009F2101AB0FBF9F007FB03035B1AB3F59D
:100D78007A7FE4D3BAF1010AC9D15B46013B9B46AD
:100D88007FF475AF4249434B4348444A0860DA60F0
:100D980003B0BDE8F08FEFF311808EF31288D5F819
:100DA80008902B68DB0304D50123C8F80030D5F878
:100DB80008902368D8F80020C0B280F31188306802
:100DC800134407FB00F2A2EB0902B2FBF0F207FBA7
:100DD8000323CBE7EFF311808EF31288D5F8089040
:100DE8002B68DB0304D50123C8F80030D5F8089038
:100DF8002368D8F80020C0B280F311883068134403
:100E080007FB00F2A2EB0902B2FBF0F207FB032397
:100E18006CE7EFF311828EF31288A8682B68D90368
:100E280003D50123C8F80030A8682368D8F8001053
:100E3800D2B282F311883268194407FB02F31B1AF5
:100E4800B3FBF2F307FB013179E7EFF311828EF37D
:100E58001288A8682B68D90303D50123C8F8003085
:100E6800A8682368D8F80010D2B282F311883268D3
:100E7800194407FB02F31B1AB3FBF2F307FB01311A
:100E880019E700BFF03500201438002010E000E01A
:100E9800FC9F002000ED00E0EFBEADDE0400FA0587
:100EA8001038002030B50446006D61710368A268EF
:100EB80023F00103036087B0A379009213F0040FB5
:100EC8004FEA03324FEA032314BF4FF4805500253D
:100ED80003F4806302F400520195CDE90223002552
:100EE80011F0010305952ED1049308238D07694657
:100EF80048BF049316F09EF96079236DA17900F03C
:100F08000202002A15BF4FF440324FF480324FF4EA
:100F18000034002410F0010F586808BF2246CC079F
:100F28004CBF024320EA02025A609A6809074CBF84
:100F380042F0080222F008029A601A6842F00102A0
:100F48001A6007B030BD042304930C23CEE700BF1A
:100F580030B50446006DA160036823F00103036007
:100F6800A379657987B013F0040F4FEA03324FEA8B
:100F7800032303F4806302F40052CDE902230091B5
:100F880014BF4FF480510021EB0748BF042301919F
:100F98004FF00001CDE9041154BF082304936946BA
:100FA80048BF0C23AD0748BF049316F043F9607996
:100FB800236DA17900F00202002A15BF4FF44032D8
:100FC8004FF480324FF40034002410F0010F5868B9
:100FD80008BF2246CC074CBF024320EA02025A60EF
:100FE8009A6809074CBF42F0080222F008029A608A
:100FF8001A6842F001021A6007B030BD2DE9F341CA
:10100800056906460F467DBBD0F80080C8F30A0381
:1010180023B30023D6F80080019312F055FD04286D
:1010280019D1224C236943F001032361BBB2A8F80C
:10103800003012F049FD04282ED108F10203019373
:10104800019B3F0C1F8012F03FFD2369042823F009
:101058000103236125D06FF0010505E012F034FD8E
:10106800042805D04FF0FF35284602B0BDE8F081CE
:101078000E4C236943F002032361C4F814802369EA
:1010880043F04003236112F01FFD2369042823F075
:1010980002032361BDD0E5E7236923F0010323613F
:1010A800D9E7336804333360DEE700BF002002402D
:1010B800F8B504460D468E180027B54201D12069BF
:1010C800F8BDE368591CE160234415F8012B1A7236
:1010D8000429F2D1A1682046FFF790FFC4E9037004
:1010E800EBE700BFF8B55D2012F0A4FC1449154BDE
:1010F8000D884A88DFF854C04C196E1C2779207176
:10110800D21B104400B283FB0034C3179CF8005074
:101118004880C3EBE403323306F00F029BB2032D81
:101128000A808B8200D0F8BDA3EB8303DB0003F6B3
:10113800E8031BB2044A83F30A031380F8BD00BF17
:10114800A8220020ABAAAA2A205B00203029002070
:10115800022828BF022010B4084C094B207000EB6D
:101168008002C0EBC20207495DF8044B013003EB73
:101178004203C0B20B6026F027BA00BF144B002010
:1011880036610020604900204B0901F01F0150F82A
:101198002320012303FA01F1114214BF184600204D
:1011A800704700BF38B5434B5A899989914224BF8B
:1011B80000225A81198ADA89914224BF0022DA81F1
:1011C800DA788AB3072A2FD03B493C4D91F853006F
:1011D800012400210A282C709C70D9713DD00C285C
:1011E80065D0DFED377A8ABB364C9FED370AA27897
:1011F800002918BFF0EE407A062A04D8334901EBDB
:10120800820191ED180A217959B3013A032A0AD8C3
:10121800F7EE007A87EE800A2FF05AFB238898426F
:1012280028BF1846208038BDD97921B1987804287C
:10123800B8BF04209870204890F853000A280CD0B2
:101248000C28CED1DFED227A002ACDD0072ACBD0C8
:101258000A282CD1DFED1F7AC6E70A20DFED1E7AB7
:10126800C1E79B78154907EE103A0A78B8EEC77AB5
:1012780067EE277A07EE102AB8EEC77A27EE277AA4
:10128800B4EEC70AF1EE10FACDDD80EE277AFDEE56
:10129800C77A17EE903A102BA8BF1023012BB8BFBE
:1012A8000123DBB29A4238BF1A460A7038BDDFED17
:1012B8000B7A99E77C3A0020903A00208A2900208E
:1012C8006F120339704100206F120338BC0D0308F8
:1012D8000AD7A3390F506E3A5304E9386F12833A8C
:1012E80038B50C4C0C4DAC4206D26168204614341B
:1012F800FFF74AFBAC42F8D3084A094B094C146083
:10130800002209491A705A7008480860BDE8384038
:101318002CF0EAB980730308E077030860490020DD
:10132800144B0020366100206449002042620020EE
:10133800F0B40C292BD8DFE801F0752A2A2A502AA4
:101348002A2A2C2A2A2A0700046AB2F80CC097888D
:1013580016686B4D24F480540462036A4468C169BA
:1013680023F4005343EA0C3321F4E641A84243EA4C
:10137800073341EA062100F0BC8005F50065A84264
:1013880000F0B78092684460C16102640362F0BCF7
:101398007047046AB2F80CC097881668584D24F450
:1013A80080740462036A4468C16923F4007343EAE1
:1013B8000C2321F07301A84243EA072341EA0601FE
:1013C80000F0848005F50065A8427FD092684460EB
:1013D800C161F0BCC26303627047046AB2F80CC012
:1013E80097881668464D24F010040462036A44681E
:1013F800816923F0200321F0807143EA0C1321F462
:10140800E641A84243EA071341EA06214BD005F515
:101418000065A84247D0926844608161F0BC82634D
:1014280003627047046A9389B2F804C01768344E9F
:1014380024F001040462046A4568816921F480315A
:1014480024F0020443EA0C0321F07301B04243EA9A
:10145800040341EA07010ED02A4CA0420BD004F540
:101468004064A04207D004F58064A04203D004F58C
:101478008064A04210D1D489168A578AB2F806C06F
:1014880023F00803234325F4407523F0040346EAB8
:1014980007044CEA03032543926845608161F0BC68
:1014A800426303627047D589178AD68823F0800380
:1014B80043EA051324F44064558A23F0400344EAC0
:1014C800870443EA061344EA8504A4E7D589178A02
:1014D800D68823F4006343EA052324F44054558A4C
:1014E80023F4806344EA071443EA062344EA051414
:1014F8006CE7158A24F4804444EA851442E700BF67
:10150800002C0140003401402DE9F04F282283B01F
:1015180000215648564D574F574E2EF0FFFF574B58
:101528009A6942F400529A619A6942F400529A61A7
:10153800DA6942F00102DA619A6942F480329A610A
:1015480005F1500A01934FF003094FF00208AB79F7
:10155800002B78D02B791C09013C052C03F00F03D4
:1015680071D837F8140040FA03F2D2076BD54FF060
:10157800010B0BFA03F3013B18402EF0D5FB404B4F
:101588001B5D184416EBC0045DD056F830303D485A
:10159800297A03F13842920A825C02F01F0052094C
:1015A800022A0BFA00FB5AD0032A52D0012A04D18E
:1015B800019842694BEA02024261B4F804C0BCFADD
:1015C8008CF2C2F11F0292B2D00803EB800002F045
:1015D8000702046A92004FF00F0E0EFA02FE24EA88
:1015E8000E040462046A01FA02F2224302624FF016
:1015F800010E00220EFA02F434EA0C0120D1500048
:10160800D3F808B009FA00F1C9430BEA010BC3F893
:1016180008B0D3F808B0C3F808B0B3F804B02BEAA0
:1016280004049C809C88A4B29C801C680C401C60AC
:101638001C6808FA00F020431860D8680140D96097
:101648000132102AD6D11435554580D103B0BDE8F2
:10165800F08F0198C2694BEA0202C261ADE70198B6
:1016680082694BEA02028261A7E700BF244D00208D
:10167800002803087C2803081838002000100240BE
:1016880088280308F827030800B9704703682DE97C
:10169800F04F03F138449C4EA40A0125345D04F050
:1016A8001F066409022C05FA06F500F07481032C64
:1016B80000F06C81012C00F022818088B0FA80F45F
:1016C800C4F11F04A4B2E50803EB850504F0070480
:1016D8002E6AA4000F27A74026EA07062E622E6A64
:1016E80001F00307A2407C1E3243012CC1F3810E96
:1016F800C1F300182A62C1F3411140F20981C607FB
:101708000BD51A6822F003021A601A683A431A6065
:10171800DA6822F003020A43DA6085070DD51A68F1
:1017280022F00C021A601A6842EA87021A60DA6824
:1017380022F00C0242EA8102DA6044070DD51A68E9
:1017480022F030021A601A6842EA07121A60DA6850
:1017580022F0300242EA0112DA6002070DD51A6857
:1017680022F0C0021A601A6842EA87121A60DA6820
:1017780022F0C00242EA8112DA60C6060DD51A6864
:1017880022F440721A601A6842EA07221A60DA687C
:1017980022F4407242EA0122DA6085060DD51A6801
:1017A80022F440621A601A6842EA87221A60DA68EC
:1017B80022F4406242EA8122DA6044060DD51A68B2
:1017C80022F440521A601A6842EA07321A60DA684C
:1017D80022F4405242EA0132DA6002060DD51A6854
:1017E80022F440421A601A6842EA87321A60DA68BC
:1017F80022F4404242EA8132DA60C6050DD51A6801
:1018080022F440321A601A6842EA07421A60DA681B
:1018180022F4403242EA0142DA6085050DD51A68A1
:1018280022F440221A601A6842EA87421A60DA688B
:1018380022F4402242EA8142DA6044050DD51A6852
:1018480022F440121A601A6842EA07521A60DA68EB
:1018580022F4401242EA0152DA6002050DD51A68F4
:1018680022F440021A601A6842EA87521A60DA685B
:1018780022F4400242EA8152DA60C6040DD51A68A1
:1018880022F040721A601A6842EA07621A60DA683F
:1018980022F0407242EA0162DA6085040DD51A68C6
:1018A80022F040621A601A6842EA87621A60DA68AF
:1018B80022F0406242EA8162DA6044040DD51A6877
:1018C80022F040521A601A6842EA07721A60DA680F
:1018D80022F0405242EA0172DA6002040DD51A6819
:1018E80022F040421A601A6842EA87771F60DA6875
:1018F80022F0404242EA8171D960BDE8F08F034C82
:10190800666935436561D8E6F82703080010024088
:1019180000224FF0010C4FF003090CFA02F636EAE8
:1019280000042ED15400D3F808A009FA04F5ED43B9
:1019380005EA0A0AC3F808A0D3F808B00EFA04FAB0
:101948004AEA0B0AC3F808A0B3F804A02AEA060674
:101958009E80B3F804A008FA02F646EA0A06B6B270
:101968009E801E682E401E60D3F800A007FA04F679
:1019780046EA0A061E60DE6801FA04F435402C4384
:10198800DC600132102AC8D1BDE8F08F044CE6694A
:101998003543E56191E6024CA6693543A5618CE6BD
:1019A8000010024003682DE9F04F03F13845AA4EB4
:1019B800AD0A0124755D05F01F066D09022D04FAB4
:1019C80006F400F0B581032D00F0AD81012D00F083
:1019D80067818088B0FA80F4C4F11F04A4B2E508D6
:1019E80003EB850504F007042E6AA4000F27A7401F
:1019F80026EA07062E622E6A01F0030702FA04F4AB
:101A08007A1E3443012AC1F3810EC1F300182C62F7
:101A1800C1F3411140F24981C60700F131818507C0
:101A280000F11C81440700F10581020700F1F080F4
:101A3800C60600F1DB80850600F1C680440600F189
:101A4800B180020600F19C80C60500F187808505FB
:101A580072D444055FD402054CD4C60439D4850435
:101A680026D4440413D4020401D4BDE8F08F1A68C4
:101A780022F040421A601A6842EA87771F60DA68E3
:101A880022F0404242EA8171D960BDE8F08F1A68BD
:101A980022F040521A601A6842EA07721A60DA683D
:101AA80022F0405242EA0172DA600204DDD5DEE734
:101AB8001A6822F040621A601A6842EA87621A605D
:101AC800DA6822F0406242EA81624404DA60CAD5E8
:101AD800DDE71A6822F040721A601A6842EA076263
:101AE8001A60DA6822F0407242EA01628504DA601C
:101AF800B7D5DDE71A6822F440021A601A6842EA8C
:101B080087521A60DA6822F4400242EA8152C60417
:101B1800DA60A4D5DDE71A6822F440121A601A6860
:101B280042EA07521A60DA6822F4401242EA015285
:101B3800DA60020591D5DDE71A6822F440221A60BE
:101B48001A6842EA87421A60DA6822F4402242EAB6
:101B580081424405DA607FF57EAFDCE71A6822F43B
:101B680040321A601A6842EA07421A60DA6822F4B8
:101B7800403242EA01428505DA607FF56AAFDBE769
:101B88001A6822F440421A601A6842EA87321A60D8
:101B9800DA6822F4404242EA8132C605DA607FF50B
:101BA80056AFDBE71A6822F440521A601A6842EA14
:101BB80007321A60DA6822F4405242EA0132DA60E7
:101BC80002067FF541AFDBE71A6822F440621A602B
:101BD8001A6842EA87221A60DA6822F4406242EA06
:101BE80081224406DA607FF52CAFDBE71A6822F41D
:101BF80040721A601A6842EA07221A60DA6822F408
:101C0800407242EA01228506DA607FF517AFDBE70A
:101C18001A6822F0C0021A601A6842EA87121A602B
:101C2800DA6822F0C00242EA8112C606DA607FF55D
:101C380002AFDBE71A6822F030021A601A6842EA3B
:101C480007121A60DA6822F0300242EA0112DA60FA
:101C580002077FF5EDAEDBE7F82703081A6822F0E4
:101C68000C021A601A6842EA87021A60DA6822F0DF
:101C78000C0242EA81024407DA607FF5D6AED9E762
:101C88001A6822F003021A601A683A431A60DA687E
:101C980022F003020A438507DA607FF5C3AEDDE769
:101CA800264D6E6934436C6193E600224FF0010CB7
:101CB8004FF003090CFA02F636EA00042ED154005C
:101CC800D3F808A009FA04F5ED4305EA0A0AC3F8AF
:101CD80008A0D3F808B00EFA04FA4AEA0B0AC3F8C7
:101CE80008A0B3F804A02AEA06069E80B3F804A068
:101CF80008FA02F646EA0A06B6B29E801E682E4028
:101D08001E60D3F800A007FA04F646EA0A061E6029
:101D1800DE6801FA04F435402C43DC600132102AF5
:101D2800C8D1BDE8F08F054DEE693443EC6150E64B
:101D3800024DAE693443AC614BE600BF001002406F
:101D480010B50409013C052C17D80E4B33F81420A4
:101D580000F00F0042FA00F313F001030FD0012343
:101D680003FA00F0013810402DF0DEFF064A074B59
:101D7800125D104403EBC00010BD002010BD1846D2
:101D880010BD00BF7C2803088828030818380020E5
:101D98001F4B98422CD0B0F1804F2BD0A3F5943331
:101DA800984229D003F58063984227D003F5006351
:101DB800984225D003F58063984223D003F59033E9
:101DC800984221D003F5406398421FD003F5806301
:101DD800984207D003F58063984208BF092202D0D1
:101DE8000020704708220B4B03EBC2031879704799
:101DF8000022F8E70122F6E70222F4E70322F2E7DD
:101E08000422F0E70522EEE70622ECE70722EAE7DC
:101E1800002C0140C42903082DE9F04F83B08E4DF2
:101E2800DFF8408201908B460BF1FF339B4601336C
:101E380000F00E8111F072FC884C894FDFF828C23F
:101E48004FF4FA7A4FF0100E4FF47A76DCF804303B
:101E5800C3F30803002B40F0DF80EFF31183002B5E
:101E680040F0DA802168AA6800BF23689942F9D156
:101E7800386806FB00F39A1AB2FBF0F206FB012160
:101E8800DCF80430C3F30803002B40F0A680EFF31E
:101E98001183002B40F0A1802368A86800BF226846
:101EA8009342F9D1D7F8009006FB09F2101AB0FB5B
:101EB800F9F006FB03035B1AB3F57A7FE0D3BAF1B6
:101EC800010AC3D1019B581CC0B211F08DFADFF88A
:101ED80098C1DCF804304FF47A7AC3F30803564605
:101EE8004FF0100E002B38D1EFF31183002B34D1B3
:101EF8002168AA6800BF23689942F9D1386806FBAF
:101F080000F39A1AB2FBF0F206FB0121DCF8043068
:101F1800C3F30803002B41D1EFF31183002B3DD10C
:101F28002368A86800BF22689342F9D1D7F80090C7
:101F380006FB09F2101AB0FBF9F006FB03035B1A63
:101F4800B3F57A7FE2D3BAF1010A3FF46DAFDCF85A
:101F58000430C3F30803002BC6D0EFF311828EF3CD
:101F68001288A8682B68D90303D50123C8F8003064
:101F7800A8682368D8F80010D2B282F311883A68AA
:101F8800194406FB02F31B1AB3FBF2F306FB0131FB
:101F9800DCF80430C3F30803002BBDD0EFF3118045
:101FA8008EF31288D5F808902B68DB0304D501233B
:101FB800C8F80030D5F808902368D8F80020C0B2D7
:101FC80080F311883868134406FB00F2A2EB09027B
:101FD800B2FBF0F206FB0323B1E7EFF311808EF3B7
:101FE8001288D5F808902B68DB0304D50123C8F8BC
:101FF8000030D5F808902368D8F80020C0B280F3E4
:1020080011883868134406FB00F2A2EB0902B2FB00
:10201800F0F206FB03234EE7EFF311828EF31288EA
:10202800A8682B68D90303D50123C8F80030A8682D
:102038002368D8F80010D2B282F311883A6819449C
:1020480006FB02F31B1AB3FBF2F306FB013117E799
:1020580003B0BDE8F08F00BF10E000E0F0350020CD
:10206800143800201038002000ED00E0204B5B6899
:10207800C3F3080330B4BBB9EFF31183A3B91D4A06
:102088001D481368846800BF11688B42F9D11B4A48
:1020980011684FF47A7202FB01F0001B30BCB0FBF0
:1020A800F1F002FB03007047EFF31182102383F372
:1020B80012881149124D8C680B68DB0344BF012359
:1020C8002B600C4B48BF8C681B682868D2B282F31F
:1020D80011880A4A11684FF47A72184402FB01F316
:1020E8001B1B30BCB3FBF1F302FB0030704700BF91
:1020F80000ED00E0F035002010E000E0143800208A
:10210800103800202DE9F84F0746264E264DFFF7D8
:10211800ADFF264A2649DFF89CC04FF0100E4FF459
:102128007A744FF001086B68C3F30803CBB9EFF377
:102138001183B3B91368D1F808A000BFD2F8009092
:102148004B45F7D1D6F8009004FB09FBABEB0A0A24
:10215800BAFBF9FA04FB03A31B1ABB42E3D3BDE89D
:10216800F88FEFF3118A8EF31288D1F808B00B6854
:10217800DB0344BFCCF80080D1F808B01368DCF862
:1021880000905FFA8AFA8AF31188D6F800A04B44C7
:1021980004FB0AF9A9EB0B09B9FBFAF904FB039351
:1021A800DAE700BF1438002000ED00E0F035002029
:1021B80010E000E0103800202DE9F84F2A4C2B4E93
:1021C8002B4D2C4F804618F1FF384AD3FFF74EFFAE
:1021D80029494B68C3F308034FF0100C4FF47A7287
:1021E8004FF0010EEBB9EFF31183D3B92368D5F89B
:1021F80008A000BFD4F800904B45F7D1D6F800905E
:1022080002FB09FBABEB0A0ABAFBF9FA02FB03A3D0
:102218001B1AB3F57A7FD6D24B68C3F30803002B99
:10222800E1D0EFF3118A8CF31288D5F808B02B6847
:10223800DB0344BFC7F800E0D5F808B02368D7F837
:1022480000905FFA8AFA8AF31188D6F800A04B4406
:1022580002FB0AF9A9EB0B09B9FBFAF902FB039394
:10226800D6E7BDE8F88F00BFF0350020143800200D
:1022780010E000E01038002000ED00E030B4EFF38B
:102288001183102282F312880649074C0A6807480E
:10229800013200250A602560DBB2026883F31188E9
:1022A80030BC7047F03500201038002010E000E006
:1022B8001D4B70B59C68236D626BDD69CAB1A36B59
:1022C80033B12B0700D470BD236D08221A6270BD8C
:1022D8002A06F6D5D4E909028242216D11D0501C94
:1022E800A669A062B25C26690A85B042E9D3A362F6
:1022F800E7E7A906E3D5E26A42B1988C216B9047DB
:10230800DDE70B6823F080030B60DAE7E1699B8C5B
:102318006069DBB24E1CE6614354E169E3689942A7
:1023280028BFE261CBE700BF0855002003685B6A5D
:1023380003B11847704700BF03681B6A03B1184709
:10234800704700BF03682DE9F041DD691DB12B46D8
:10235800BDE8F0411847002A174611DD04460E462D
:102368000F4400E023689B68204698470028F9D06E
:10237800236816F8011B1B6820469847BE42F1D116
:10238800BDE8F08103689B69184700BF03685B6973
:10239800184700BF0368DB68184700BF03689B68DD
:1023A800184700BF03685B68184700BF03681B68CD
:1023B800184700BF014B9869F8E700BFA822002022
:1023C800054B53F8203033B11A689B88918A0B4229
:1023D80018BF1B0493617047E0370020036803F1BE
:1023E80038422DE9F04F920AA74DAA5C02F01F056A
:1023F80052090124022A04FA05F400F09F81032AF5
:1024080000F09781012A00F0518101F003077A1E3C
:10241800012AC1F3810EC1F300188488C1F3411168
:1024280040F24981E60700F13181A50700F11A81E0
:10243800600700F10581220700F1F080E60600F14F
:10244800DB80A50600F1C680600600F1B180220697
:1024580000F19C80E60500F18780A50572D460052F
:102468005FD422054CD4E60439D4A50426D46004EC
:1024780013D4220401D4BDE8F08F1A6822F0404238
:102488001A601A6842EA87771F60DA6822F04042C9
:1024980042EA8171D960BDE8F08F1A6822F0405293
:1024A8001A601A6842EA07721A60DA6822F0405223
:1024B80042EA0172DA602204DDD5DEE71A6822F00A
:1024C80040621A601A6842EA87621A60DA6822F083
:1024D800406242EA81626004DA60CAD5DDE71A68C0
:1024E80022F040721A601A6842EA07621A60DA68D3
:1024F80022F0407242EA0162A504DA60B7D5DDE74E
:102508001A6822F440021A601A6842EA87521A606E
:10251800DA6822F4400242EA8152E604DA60A4D57D
:10252800DDE71A6822F440121A601A6842EA075274
:102538001A60DA6822F4401242EA0152DA6022058F
:1025480091D5DDE71A6822F440221A601A6842EA37
:1025580087421A60DA6822F4402242EA8142600522
:10256800DA607FF57EAFDCE71A6822F440321A6041
:102578001A6842EA07421A60DA6822F4403242EAEC
:102588000142A505DA607FF56AAFDBE71A6822F435
:1025980040421A601A6842EA87321A60DA6822F4FE
:1025A800404242EA8132E605DA607FF556AFDBE762
:1025B8001A6822F440521A601A6842EA07321A600E
:1025C800DA6822F4405242EA0132DA6022067FF5E4
:1025D80041AFDBE71A6822F440621A601A6842EADF
:1025E80087221A60DA6822F4406242EA8122600691
:1025F800DA607FF52CAFDBE71A6822F440721A60C4
:102608001A6842EA07221A60DA6822F4407242EA3B
:102618000122A506DA607FF517AFDBE71A6822F01A
:10262800C0021A601A6842EA87121A60DA6822F051
:10263800C00242EA8112E606DA607FF502AFDBE704
:102648001A6822F030021A601A6842EA07121A6001
:10265800DA6822F0300242EA0112DA6022077FF5D6
:10266800EDAEDBE71A6822F00C021A601A6842EA3B
:1026780087021A60DA6822F00C0242EA81026007D7
:10268800DA607FF5D8AEDBE7F82703081A6822F08E
:1026980003021A601A683A431A60DA6822F00302E1
:1026A8000A43A507DA607FF5C3AEDBE7264A55691A
:1026B8002C435461A9E600224FF0010C4FF00309A6
:1026C8000CFA02F636EA04002ED15000D3F808A01E
:1026D80009FA00F5ED430AEA050AC3F808A0D3F899
:1026E80008B00EFA00FA4AEA0B0AC3F808A0B3F8D1
:1026F80004A02AEA06069E80B3F804A008FA02F6A7
:1027080046EA0A06B6B29E801E682E401E60D3F8BE
:1027180000A007FA00F646EA0A061E60DE6801FA1B
:1027280000F035402843D8600132102AC8D1BDE8EE
:10273800F08F054AD5692C43D46166E6024A95694B
:102748002C43946161E600BF001002402DE9F04F70
:102758004A484B4B4B4C4FF090414FF0010A4FF019
:1027680002094FF004084FF0080E4FF0100C202714
:102778004026802530F8022B12F0010F03D0196093
:10278800A3F804A0083312F0020F03D01960A3F8CD
:102798000490083312F0040F03D01960A3F80480E2
:1027A800083312F0080F03D01960A3F804E00833C7
:1027B80012F0100F03D01960A3F804C0083312F008
:1027C800200F02D019609F80083312F0400F02D00A
:1027D80019609E80083312F0800F02D019609D8026
:1027E800083312F4807F05D04FF4807B1960A3F87A
:1027F80004B0083312F4007F05D04FF4007B196051
:10280800A3F804B0083312F4806F05D04FF4806B3E
:102818001960A3F804B0083312F4006F05D04FF420
:10282800006B1960A3F804B0083312F4805F05D078
:102838004FF4805B1960A3F804B0083312F4005F0A
:1028480005D04FF4005B1960A3F804B0083312F404
:10285800804F05D04FF4804B1960A3F804B00833BB
:10286800D20B04D04FF4004219609A80083301F566
:102878008061A1427FF47EAFBDE8F08F7C28030819
:10288800183800200018004800B97047036803F1A1
:1028980038422DE9F04F920AB24DAA5C02F01F05AA
:1028A80052090124022A04FA05F400F05F81032A80
:1028B80000F05381012A00F00D8101F003077A1E10
:1028C800012AC1F3810EC1F300188488C1F34111B4
:1028D80040F20581E6070BD51A6822F003021A6058
:1028E8001A683A431A60DA6822F003020A43DA6087
:1028F800A5070DD51A6822F00C021A601A6842EA78
:1029080087021A60DA6822F00C0242EA8102DA6071
:1029180060070DD51A6822F030021A601A6842EA78
:1029280007121A60DA6822F0300242EA0112DA600D
:1029380022070DD51A6822F0C0021A601A6842EA06
:1029480087121A60DA6822F0C00242EA8112DA605D
:10295800E6060DD51A6822F440721A601A6842EA2F
:1029680007221A60DA6822F4407242EA0122DA6029
:10297800A5060DD51A6822F440621A601A6842EA60
:1029880087221A60DA6822F4406242EA8122DA6019
:1029980060060DD51A6822F440521A601A6842EA95
:1029A80007321A60DA6822F4405242EA0132DA60E9
:1029B80022060DD51A6822F440421A601A6842EAC3
:1029C80087321A60DA6822F4404242EA8132DA60D9
:1029D800E6050DD51A6822F440321A601A6842EAF0
:1029E80007421A60DA6822F4403242EA0142DA60A9
:1029F800A5050DD51A6822F440221A601A6842EA21
:102A080087421A60DA6822F4402242EA8142DA6098
:102A180060050DD51A6822F440121A601A6842EA55
:102A280007521A60DA6822F4401242EA0152DA6068
:102A380022050DD51A6822F440021A601A6842EA83
:102A480087521A60DA6822F4400242EA8152DA6058
:102A5800E6040DD51A6822F040721A601A6842EA34
:102A680007621A60DA6822F0407242EA0162DA60AC
:102A7800A5040DD51A6822F040621A601A6842EA65
:102A880087621A60DA6822F0406242EA8162DA609C
:102A980060040DD51A6822F040521A601A6842EA9A
:102AA80007721A60DA6822F0405242EA0172DA606C
:102AB80022040DD51A6822F040421A601A6842EAC8
:102AC80087771F60DA6822F0404242EA8171D96054
:102AD800BDE8F08F244A55692C435461EDE6002285
:102AE8004FF0010C4FF003090CFA02F636EA040025
:102AF8002ED15000D3F808A009FA00F5ED430AEAF0
:102B0800050AC3F808A0D3F808B00EFA00FA4AEA92
:102B18000B0AC3F808A0B3F804A02AEA06069E80A8
:102B2800B3F804A008FA02F646EA0A06B6B29E808E
:102B38001E682E401E60D3F800A007FA00F646EA89
:102B48000A061E60DE6801FA00F035402843D860A6
:102B58000132102AC8D1BDE8F08F034AD5692C4349
:102B6800D461AAE6F827030800100240024A9569D2
:102B78002C439461A1E600BF0010024010B1036825
:102B880082881A85704700BF10B1036882889A61ED
:102B9800704700BF18B1838811B10268936170470C
:102BA8001B04FAE710B40A4B0A4A1C780123834035
:102BB800234052F8200029B9B3FA83F149095DF896
:102BC800044BE7E7191C18BF01215DF8044BE1E746
:102BD800DC370020E037002008B501210220FFF78C
:102BE800E1FF094B1B7803F00503052B08D00021F2
:102BF8000120FFF7D7FF00210846FFF7D3FFFEE7C4
:102C080019F058FAF3E700BFA45200200E4B1B88B6
:102C180001463BB90D4B0E4A1B7810680BB981F081
:102C28000101B7E70B4B5A691AB11A6810B910605D
:102C38005874704708480949008891FBF0F1012051
:102C480011605874704700BFEC370020EE37002041
:102C5800F0370020F43700200C38002020A10700AE
:102C680030B102688388128A1A4214BF01200020FA
:102C7800704700BF08B5074B1868FFF7F1FF00B9A8
:102C880008BDFFF7F3F9044B0122D86183F820202F
:102C980008BD00BF04450020A82200202DE9F0410E
:102CA8000B4E346873691C400FD0DFF82880012769
:102CB800B4FA84F3C3F11F0307FA03F558F82300A5
:102CC80003689847AC437561F2D1BDE8F08100BF55
:102CD80000040140BC4400202DE9F0410B4E34684B
:102CE80073691C400FD0DFF828800127B4FA84F3F9
:102CF800C3F11F0307FA03F558F823000368984740
:102D0800AC437561F2D1BDE8F08100BF0004014019
:102D1800BC4400202DE9F0410B4E346873691C4017
:102D28000FD0DFF828800127B4FA84F3C3F11F031A
:102D380007FA03F558F8230003689847AC43756110
:102D4800F2D1BDE8F08100BF00040140BC4400207E
:102D58002DE9F0410B4E346873691C400FD0DFF841
:102D680028800127B4FA84F3C3F11F0307FA03F597
:102D780058F8230003689847AC437561F2D1BDE861
:102D8800F08100BF00040140BC4400202DE9F0415F
:102D98000B4E346873691C400FD0DFF82880012778
:102DA800B4FA84F3C3F11F0307FA03F558F82300B4
:102DB80003689847AC437561F2D1BDE8F08100BF64
:102DC80000040140BC4400202DE9F0410B4E34685A
:102DD80073691C400FD0DFF828800127B4FA84F308
:102DE800C3F11F0307FA03F558F82300036898474F
:102DF800AC437561F2D1BDE8F08100BF0004014029
:102E0800BC4400202DE9F0410B4E346873691C4026
:102E18000FD0DFF828800127B4FA84F3C3F11F0329
:102E280007FA03F558F8230003689847AC4375611F
:102E3800F2D1BDE8F08100BF00040140BC4400208D
:102E4800A8B18388B3FA83F3C3F11F035A1C08D0CF
:102E5800012202FA03F329B906490A6822EA0303A0
:102E68000B607047034A11680B43136070470123D6
:102E7800F1E700BF00040140084A094808B5936912
:102E880043F001039361002140222DF047FB054BDD
:102E98004FF0FF321A60C3F8032008BD001002404B
:102EA800BC440020FC44002003681B6A184700BF8C
:102EB80070B44E1C0568C2728672AC69A44670BCB8
:102EC800604700BF2DE9F041044618460D461646F6
:102ED8001F462CF00BFA2844A0722068E672294697
:102EE80045693B4632462046AC46BDE8F04160475E
:102EF800036810B504461B689847236820469B68FA
:102F08009847A37B0133A37310BD00BF03681B69F7
:102F1800184700BF10B5036804469B689847FF230D
:102F280001226373227310BD08B5FEF709FF38B19B
:102F38002D2282710022C271BDE8084010F0B0B89D
:102F480008BD00BF0B4B984211D0A3F578439842B7
:102F580002D04FF0FF3070470122074B03EB0213FA
:102F68005A89013292B25A81588980B27047002238
:102F7800F3E700BF003001402C5500202DE9F04F49
:102F880090F8553085B00746002B40F0D784A84B01
:102F9800786993F82130BA69002B00F01281038810
:102FA80023F040031B041B0C038003889BB223F00F
:102FB800380343F038030380038843F04003038059
:102FC80097F84E1012B1136892881A8540F2E933C7
:102FD80002E0002B00F001850289013B12F0020F8C
:102FE8009BB2F6D01A23037300F10C0440F2E933C4
:102FF80002E0002B00F0F1840289013B12F0010F7E
:103008009BB2F6D02378786940F2E93302E0002BCE
:1030180000F0DF840289013B12F0020F9BB2F6D068
:10302800017340F2E93302E0002B00F0D2840289F8
:10303800013B12F0010F9BB2F6D0037BBB6913B1C1
:103048001A689B889361FFF711F80446FFF70EF89A
:103058008442FBD07869038823F040031B041B0CCF
:103068000380038823F038031B041B0C03800388A8
:1030780043F0400303803B7C022B36D0B7F93A304B
:103088005BB2013302D005B0BDE8F08F97F9383054
:103098000133F8D10A2610F041FB4FF4FA75FEF718
:1030A800E5FF0446FEF7E2FF001BB0F57A7FF9D38F
:1030B800013DF4D1072010F097F94FF47A75FEF727
:1030C800D5FF0446FEF7D2FF001BB0F57A7FF9D38F
:1030D800013DF4D1013EDED15649574B5748584A75
:1030E8000860DA6005B0BDE8F08FBB6913B11A68F3
:1030F8009B88138540F2E93302E0002B00F0C2847C
:103108000289013B12F0020F9BB2F6D0C32303736E
:1031180040F2E93302E0002B00F0B4840289013B5D
:1031280012F0010F9BB2F6D0037B7869838903897B
:1031380099074FF0050C02AD4FF47A724FF0FF0675
:103148004FF6FF7406D4531E9BB2E2B11A460389A8
:103158009907F8D506734FF47A7302E08BB2A3424D
:1031680011D00289D20703F1FF31F7D5027BD2B221
:103178000DB12A7001350CF1FF32BCF1000F04D0FB
:1031880094461A46E3E7FFF7DDFEBB6913B11A68F8
:103198009B8893619DF80A509DF80B309DF8084074
:1031A8009DF809109DF80C009DF80D2043EA0523B1
:1031B8001BB241EA042142EA00227B873987BA8799
:1031C8005EE7038823F040031B041B0C038003887D
:1031D8009BB223F0380343F038030380038843F09D
:1031E8004003038012B1136892881A8540F2E933CC
:1031F80002E0002B00F042840289013B12F0020F2A
:103208009BB2F6D06B23037300F10C0140F2E93353
:1032180002E0002B00F032840289013B12F0010F1A
:103228009BB2F6D00B78786940F2E9330DE000BF25
:10323800A8220020FC9F002000ED00E0EFBEADDEDC
:103248000400FA05002B00F015840289013B12F0F6
:10325800020F9BB2F6D08023037340F2E93302E0F9
:10326800002B00F007840289013B12F0010F9BB28A
:10327800F6D0037BBB6913B11A689B8893619623C8
:10328800A84CA94EDFF8A882A84DDFF8A8920197AC
:103298004FF0100A1F46FEF7E9FE4FF47A7C4FF014
:1032A800010ED8F80430C3F30803002B40F028833C
:1032B800EFF31183002B40F023832368A96800BF34
:1032C80022689342F9D132680CFB02FBABEB010197
:1032D800B1FBF2F10CFB03131B1AB3F57A7FE0D3B1
:1032E800013FD8D1019FBB6913B11A689B88138528
:1032F800786940F2E93302E0002B00F0B8830289D4
:10330800013B12F0020F9BB2F6D06823037340F220
:10331800E93302E0002B00F0AA830289013B12F096
:10332800010F9BB2F6D0037B786940F2E93302E0E3
:10333800002B00F099830289013B12F0020F9BB227
:10334800F6D00323037340F2E93302E0002B00F0C8
:103358008B830289013B12F0010F9BB2F6D0037BED
:10336800BB6913B11A689B8893619623DFF8C08103
:103378006E4DDFF8C09101974FF0100A1F46FEF717
:1033880075FE4FF47A7C4FF0010ED8F80430C3F381
:103398000803002B40F09682EFF31183002B40F0D6
:1033A80091822368A96800BF22689342F9D13268E4
:1033B8000CFB02FBABEB0101B1FBF2F10CFB0313BD
:1033C8001B1AB3F57A7FE0D3013FD8D1019FBB69BF
:1033D80013B11A689B881385786940F2E93302E0D3
:1033E800002B00F03E830289013B12F0020F9BB2D2
:1033F800F6D06B23037340F2E93302E0002B00F0B0
:1034080030830289013B12F0010F9BB2F6D0037B97
:10341800786940F2E93302E0002B00F01F8302894B
:10342800013B12F0020F9BB2F6D00323037340F264
:10343800E93302E0002B00F011830289013B12F00E
:10344800010F9BB2F6D0037BBB6913B11A689B8846
:103458009361FEF70BFE0446FEF708FE001B0E28DC
:10346800FAD9BB6913B11A689B881385786940F249
:10347800E93302E0002B00F0EE820289013B12F0F2
:10348800020F9BB2F6D06A23037340F2E93302E0DD
:10349800002B00F0E0820289013B12F0010F9BB281
:1034A800F6D0037B786940F2E93302E0002B00F0A4
:1034B800CF820289013B12F0020F9BB2F6D0102393
:1034C800037340F2E93302E0002B00F0C182028965
:1034D800013B12F0010F9BB2F6D0037BBB6913B11D
:1034E8001A689B889361FEF7C1FD0446FEF7BEFD8E
:1034F800001B0E28FAD9BB6913B11A689B8813857B
:10350800786940F2E93302E0002B00F09E820289DC
:10351800013B12F0020F9BB2F6D06C23037340F20A
:10352800E9330CE0F03500201438002010E000E00A
:1035380000ED00E010380020002B00F086820289A0
:10354800013B12F0010F9BB2F6D0037B786940F281
:10355800E93302E0002B00F075820289013B12F08A
:10356800020F9BB2F6D00023037340F2E93302E066
:10357800002B00F067820289013B12F0010F9BB219
:10358800F6D0037BBB6913B11A689B889361FEF779
:103598006DFD0446FEF76AFD001B0E28FAD9BB69CB
:1035A80097F8501013B11A689B881385786940F210
:1035B800E93302E0002B00F042820289013B12F05D
:1035C800020F9BB2F6D01923037340F2E93302E0ED
:1035D800002B00F034820289013B12F0010F9BB2EC
:1035E800F6D0037B786940F2E93302E0002B00F063
:1035F80023820289013B12F0020F9BB2F6D00173BD
:1036080040F2E93302E0002B00F016820289013B08
:1036180012F0010F9BB2F6D0037BBB6913B11A6895
:103628009B889361FEF722FD0446FEF71FFD001BF1
:103638000E28FAD9BB6913B11A689B881385786973
:1036480040F2E93302E0002B00F0F3810289013BEC
:1036580012F0020F9BB2F6D01B23037340F2E9333A
:1036680002E0002B00F0E5810289013B12F0010F16
:103678009BB2F6D0037B786940F2E93302E0002B75
:1036880000F0D4810289013B12F0020F9BB2F6D000
:103698001823037340F2E93302E0002B00F0C681DF
:1036A8000289013B12F0010F9BB2F6D0037BBB6984
:1036B80013B11A689B889361FEF7D8FC0446FEF79D
:1036C800D5FC001B0E28FAD9BB6913B11A689B8870
:1036D8001385786940F2E93302E0002B00F0A381FA
:1036E8000289013B12F0020F9BB2F6D01C23037330
:1036F80040F2E93302E0002B00F095810289013B9A
:1037080012F0010F9BB2F6D0037B786940F2E933DF
:1037180002E0002B00F084810289013B12F0020FC5
:103728009BB2F6D01023037340F2E93302E0002B7A
:1037380000F076810289013B12F0010F9BB2F6D0AE
:10374800037BBB6913B11A689B889361FEF78EFCF3
:103758000446FEF78BFC001B0E28FAD9BB6913B18F
:103768001A689B881385786940F2E93302E0002BD8
:1037780000F053810289013B12F0020F9BB2F6D090
:103788003723037340F2E93302E0002B00F0458150
:103798000289013B12F0010F9BB2F6D0037B7869D6
:1037A80040F2E93302E0002B00F034810289013B4A
:1037B80012F0020F9BB2F6D01023037340F2E933E4
:1037C80002E0002B00F026810289013B12F0010F74
:1037D8009BB2F6D0037BBB6913B11A689B889361CF
:1037E800FEF744FC0446FEF741FC001B0E28FAD9FC
:1037F800BB6913B11A689B881385786940F2E9336D
:1038080002E0002B00F003810289013B12F0020F55
:103818009BB2F6D03823037340F2E93302E0002B61
:1038280000F0F5800289013B12F0010F9BB2F6D03F
:10383800037B786940F2E93302E0002B00F0E48072
:103848000289013B12F0020F9BB2F6D001230373E9
:1038580040F2E93302E0002B00F0D6800289013BF8
:1038680012F0010F9BB2F6D0037BBB6913B11A6843
:103878009B889361FEF7FAFB0446FEF7F7FB001BF3
:103888000E28FAD97A69138823F040031B041B0C0D
:103898001380138823F038031B041B0C1380138830
:1038A80043F040031380FEF7E1FB0446FEF7DEFB1E
:1038B8008442FBD07A490123D7E9050281F82130F7
:1038C800FFF76DBBEFF311818AF31288D5F808B0C2
:1038D8002B68DB0344BFC9F800E0D5F808B02368BB
:1038E800D9F80020C9B281F31188316813440CFB60
:1038F80001F2A2EB0B02B2FBF1F20CFB03235FE532
:10390800EFF311818AF31288D5F808B02B68DA032F
:1039180044BFC9F800E0D5F808B02368D9F80020FA
:10392800C9B281F31188316813440CFB01F2A2EB90
:103938000B02B2FBF1F20CFB0323CDE41D09013DA0
:10394800052D03F00F034CD8564A32F8150040FAFB
:1039580003F2D40745D5012404FA03F3013B1840C8
:103968002CF0E2F9504B514A5B5D184412EBC0054C
:1039780037D000232021EB71A97152F830004C4A4E
:1039880000F138439B0AD25C02F01F035209022A55
:1039980004FA03F37AD0032A31D0A2427BD0AB8851
:1039A800029302A9002303930FF034FB3946414BDD
:1039B80041F80C3F284613F01DF8AB88B3FA83F39F
:1039C800C3F11F03591C3FF4E2AA012202FA03F3D0
:1039D8000FE0FFF7B7FAFFF731BBFFF7B3FAFFF7CE
:1039E80012BB3946334B41F80C3F002013F002F864
:1039F800012331490A6813430B60FFF7C8BA2F4AFD
:103A0800D1690B43D361CAE7FFF79CFA2DE7FFF7AB
:103A180099FA0EE7FFF796FADDE6FFF793FABEE6A6
:103A2800FFF790FA8DE6FFF78DFA6EE6FFF78AFA50
:103A38003DE6FFF787FA1EE6FFF784FAEDE5FFF7A4
:103A480081FACFE5FFF77EFA9CE5FFF77BFA7DE583
:103A5800FFF778FA42E5FFF775FA23E5FFF772FA00
:103A6800F2E4FFF76FFAD3E4FFF76CFA78E4FFF7B4
:103A780069FA59E4FFF766FAFFF7FCBBFFF762FA49
:103A8800FFF7D1BBFFF75EFAFFF74FBB0B4A91690F
:103A98000B43936183E7094A51690B4353617EE7FE
:103AA800A82200207C28030888280308183800204A
:103AB800F8270308690800080004014000100240C4
:103AC800F0B5836983B0064613B11A689B881385DD
:103AD8007069DFF898C08389C3244FF47A73062786
:103AE8006D464FF6FF710CF1010C03E0013B9BB2F0
:103AF8008B421CD002899207F8D504734FF47A736D
:103B080002E0A3B28B4212D00289D20703F1FF343C
:103B1800F7D5027BD2B20DB12A7001354FB1013F02
:103B2800FF24BCF1000FE5D09CF80040DBE7FFF76D
:103B380009FAB36913B11A689B8893619DF8050067
:103B48009DF801509DF802109DF803409DF804204F
:103B58009DF8063041EA052143EA002342EA04229F
:103B6800012031877287B38703B0F0BD380E030890
:103B7800037A022B01D000207047F0B5036983B0A7
:103B880013B11A689B881385014640F2E933C0686F
:103B980001E0002B5ED00289013B12F0020F9BB2BC
:103BA800F7D0BB23037340F2E93301E0002B51D077
:103BB8000289013B12F0010F9BB2F7D0037BC86862
:103BC800838903899C074FF005076E464FF47A7284
:103BD8004FF0FF0C4FF6FF7506D4531E9BB2D2B1BF
:103BE8001A4603899C07F8D580F80CC04FF47A73FD
:103BF80002E0A3B2AB420ED00289D20703F1FF3430
:103C0800F7D5027BD2B20EB1327001367A1E27B1D7
:103C180017461A46E5E7FFF795F90B6913B11A68D5
:103C28009B8893619DF800609DF801009DF8025003
:103C38009DF803209DF804409DF8053040EA0620D1
:103C480042EA052243EA0423C88201200A834B83FF
:103C580003B0F0BDFFF776F9B1E700BF427A4AB189
:103C680010B5044604F10A01D0E900309847002352
:103C7800637210BD704700BF437A5A1C0344D2B226
:103C880042729972037A93420AD84AB110B504462F
:103C980004F10A01D0E9003098470023637210BD8F
:103CA800704700BFA8B10D4B012210B402FA01F110
:103CB80003F1750402E00333A3420BD013F8012C7F
:103CC8008242F8D11A780A42F5D001205DF8044BF7
:103CD8007047704700205DF8044B7047410E030899
:103CE80030B40A4D002305F1840401E0272B0AD0E3
:103CF80003EB43020133A15C8142F7D12A4430BC73
:103D080092F886007047002030BC7047BC0D03084D
:103D1800064B07498B4202D30023184670471A887E
:103D2800C2F30B029042F8D01433F3E78073030810
:103D3800E0770308024A136823EA0000106070471E
:103D4800BC6700202DE9F84F0BF0C6F9DFF858835F
:103D5800B64B434525D2DFF85493B54F03F114060B
:103D68009A464C462588621985B1BA420ED2052D6D
:103D78000CD936F8143C6188C3F30B03994200F060
:103D8800E780144625886219002DEED156F8101CDC
:103D980050460AF1140AFCF7F7FDC24506F114066D
:103DA800DFD3A4490B78A3F11702022A0FD9A24A3C
:103DB80012F83300002840F00381D80002445278FA
:103DC8002AB19E4A12F83330002B00F027819C4B11
:103DD8005A78022A40F2E58000225A701A789948E7
:103DE80099490160022A00F2E78002EB8201974BB1
:103DF800C2EBC10203EB4203998C5A8C944C91425A
:103E0800236001D300225A84924B9A78042A00F046
:103E1800E08032B91A88B2F5F07F84BF4FF4F072AF
:103E28001A808D4DFDF7BEF92B688C4A1A40002A7E
:103E380000F0F780DE0700F1EC80580400F1E48020
:103E4800190700F1DC809A0100F1D3809B0400F18E
:103E5800C98010F02FFA10B9814820F039FF4020AE
:103E6800FFF768FF8020FFF765FF4FF40070FFF74A
:103E780061FF4FF40030FFF75DFF4FF40010FFF7CC
:103E880059FF4FF08060FFF755FF4FF00060FFF7D4
:103E980051FF18F069FF0021302272482CF03EFBD8
:103EA800206817F04BFD704B256803F1640102E0B0
:103EB8000533994273D01A78002AF9D19C78D878BA
:103EC8008442F5D269496A4B0E796A4CC82064214C
:103ED80011FB060159600021674883F82010C3E9E7
:103EE8000211C3E90411C3E9061183F82110634BD9
:103EF8002270C0E915530AF0DBFE614B9FED615A51
:103F08001B88614A9FED616A5079614906EE903AD3
:103F1800F8EEE66A1388C5EE265A07EE103A53887B
:103F28001279C1ED005A07EE903AB8EEC77AF8EE6A
:103F3800E77A584B27EE067A67EE867A18725A7235
:103F480083ED017AC3ED007ABDE8F84F0BF06AB84B
:103F580063799B077FF415AF56F8101C94F804B0EA
:103F68005046FCF711FD36F8143CBBEB133F07D065
:103F78000AF1140AC24506F11406FFF4F2AE10E77E
:103F880036F8123C56F8100CAA1FC3F30B039A42DA
:103F980004F10601A8BF1A462CF0A6F9E8E70122A9
:103FA80090E72949274802EB420201EB82011A787F
:103FB8000160022A7FF619AF00221A70234B1BE713
:103FC800D80014186468002C7FF4F8AE17240C701D
:103FD800F4E69A8AB2F57A7FBFF423AF4FF47A7287
:103FE8009A821EE72C48FFF7A5FE4020FFF7A2FEA5
:103FF8002FE746F20900FFF79DFE2B6826E72748C2
:10400800FFF798FE2B681EE72548FFF793FE2B68FD
:1040180016E72448FFF78EFE2B680EE718230B706F
:10402800D5E643F400532B6004E700BF8073030810
:1040380000000408A02D0020902803085C2E030827
:10404800144B0020644900204262002036610020A1
:104058006049002070410020BC6700200960000210
:1040680074390020CC220020BC310020B04F002041
:10407800285B0020D8020020A8220020662D0020FE
:1040880034520020C0C9FB480459002017B7D13862
:1040980038520020104D0020094000020160000243
:1040A8000920000208600002E077030802F0030814
:1040B800F8B5174D2B78A52B28D16B78BE2B25D1B9
:1040C800022229464FF6FF70FCF78AFB114FAC1C01
:1040D80022884AB1A618BE4218D2052A16D9214606
:1040E800FCF77EFB3446F3E721460222FCF778FB17
:1040F8000222A118FCF774FB0634074B641B1C80D2
:1041080041F60F53C31A58425841F8BD0020FCE746
:1041180000F0030800000408982900202DE9F04F5A
:10412800DFF844914B4F8BB00326A7EB0907102209
:10413800002106A82CF0F2F9CDE90497464B1A693C
:10414800120604D5454A5A6002F188325A600122A3
:104158008DF824203422DA60414B424C1B88ADF89C
:1041680000300222694604A8FCF7A2FF0222694631
:104178004FF6FF70FCF734FBDFF8F0A080464FF0F5
:10418800000B544536D30AAC002524F8245D0222DE
:10419800214604A8FCF78CFF022221464046FCF782
:1041A8001FFB40BAC043ADF80800022202A904A8C8
:1041B800FCF77EFF079860B106ABC0F10402294600
:1041C80018442CF0ABF9069904A8FCF717FFCDE9C1
:1041D80007509DF82430089A23B11F490B6943F012
:1041E80080030B61013E2DD0002AA0D1FFF760FFAC
:1041F80050B32CE065888DF80DB0C5F30B05AB1DE9
:10420800ADF808302388C3F30B02ADF80A201B0B66
:10421800062202A904A88DF80C30FCF749FF0622F3
:1042280002A94046FCF7DCFA616880462A4604A8E1
:10423800FCF73EFF616840462A46FCF7D1FA143481
:1042480080469EE7002AD1D00520FCF703FD0BB07D
:10425800BDE8F08F000004080020024023016745F4
:10426800B50E03088073030800F00308E07703081D
:1042780008B50AF031FFFFF751FF0AF0D3FEFFF748
:1042880061FD0120BDE8084023F09EB92DE9F04703
:10429800C94C636820469847002800F0C180C74B86
:1042A8001B780122042B84F83C2000F0BB80B4F971
:1042B8001610B4F91820B4F91A30A363C4E90C1223
:1042C800BF4B1B88002B69D0BE4DD4ED0C7AD5EDC1
:1042D800004A95ED050A95ED015A95ED067AD5ED5A
:1042E800035A95ED026AF8EEE76AD5ED047AA4EE72
:1042F800A60AA5EE267A67EEC07AA5EEC07AE6EEA3
:10430800267A85ED057AC5ED067A2CF0E1FAD4ED2A
:104318000D6AD5ED094A95ED0E0A95ED0A5A95ED07
:104328000F7AD5ED0D7AD5ED0C5A95ED0B6A206311
:10433800F8EEE66AA4EEA60AA5EE267A67EEC07A3B
:10434800A5EEC07AE6EE267A85ED0E7AC5ED0F7AEF
:104358002CF0BEFAD4ED0E6AD5ED124A95ED170A87
:1043680095ED135A95ED187AD5ED167AD5ED155ABF
:1043780095ED146A6063F8EEE66AA6EEA40AA6EE66
:10438800857A67EEC07AA0EE657AE6EE867A85EDE4
:10439800177AC5ED187A2CF09BFAA0638A4DA17F95
:1043A8008A48DFF844820AF005FC2B88D8F85810B0
:1043B800002B7FD1864B1B685A0741D4B1F9007096
:1043C800226BB1F90260B1F904508249D4E90D3089
:1043D800D21B07EE902A9B1B401BB8EEE77A06EE2D
:1043E800100A07EE903A7C4D91ED005AD1ED015A32
:1043F800D1ED026A6363F8EEE77AB8EEC66A2B6815
:10440800226337EE057A77EEA57A76EE866A01336F
:10441800A06381ED007AC1ED017AC1ED026A2B60DB
:10442800BDE8F0876D4BB4F91600B4F91810B4F96B
:104438001A2018802063598061639A80A2633FE73D
:10444800B8F868C0BCF1320F00F09080BCF1000FE2
:1044580040F0CC8098F88630002BAFD008F1780077
:104468000DC85F4DA68A85FB03C7DB17C3EB27136F
:104478009B1B85FB007685FB0275D217C2EB2512C4
:10448800C017584D8B80C0EB2610002308804A8047
:10449800AB81EB8188F886300AF01EFEFFF73EFEFE
:1044A8000AF0C0FDFFF74EFC012023F08DF8D8F884
:1044B800581083E7B3F5C87F4FF00003226B2363DE
:1044C8000B80288814BFD8F85C600026B0F5C87F38
:1044D80018BFD8F86030606B32442E88C8F85C206A
:1044E80000270344B6F5C87F6763C8F860304F807B
:1044F8005BD0D4F838C0D8F86400A7636044012EB4
:104508008F80C8F864002ED1DFF8D4C0B4F814E066
:10451800C8308CFB00A9C832C833C017C0EBE910FB
:104528008CFB02A98CFB03ACDB17C3EBEC13D21793
:10453800DFF8B0C04B80A0EB0E00C2EBE912888018
:104548000A80ACF80C70ACF80E700AF0C5FDFFF7E5
:10455800E5FD0AF067FDFFF7F5FB304623F034F878
:104568002E88D8F85810701E288023E71D4A0B683B
:10457800D2688888C8F87420226BC8F87820C8F8F0
:104588006C30A26BA8F870000023606B23630B806B
:104598006363C8F87C004B80A363C8F880208B80D5
:1045A8000CF1FF3CA8F868C054E7A36BC8F8643066
:1045B800A7638F80D7E700BF14490020104B002065
:1045C800E0300020E43000208E50002044490020D4
:1045D800183D0020E84D0020E44D0020084B002045
:1045E8001F85EB51602D0020A8220020D8F88050AC
:1045F800206BD8F87870626BD8F87C60A36B38446D
:104608002B4432440025BCF1010FC8F8780025631B
:104618000D806563C8F87C204D80A563C8F880309C
:104628008D80BDD11E4B88F884501B6888F885C0E2
:104638009B032AD41B48002203461D780B2D03F147
:104648000C030DD00132182AF7D1D8F86C20164B7C
:104658000A60B8F87000D8F874208880DA609FE79C
:10466800124D2F68530037B19E1800EB86067F78ED
:104678007678BE42E9D213440D4E0E4A00EB830011
:104688000023286033801360DFE70B4B1B78032B74
:10469800D0D122F09FFED8F85810B8F868C0D4E7F7
:1046A800AC32002060230308602D0020FC4F00205E
:1046B80000500020045000209459002008B5FCF751
:1046C8000FFE0AF009FDFFF729FDBDE808400AF0D2
:1046D800A9BC00BF08B50AF0FFFCFFF71FFDBDE845
:1046E80008400AF09FBC00BF0378202B024600F167
:1046F8000100F9D0092BF7D02D2B00F0A4802B2B2B
:1047080003BF5378B7EE000A0246B7EE000AA3F1DA
:104718003001C8B209289FED577A10D8F2EE046A22
:1047280007EE901AF8EEE77A12F8013FE7EE267ADC
:10473800A3F13001C8B20928B0EE677AF0D92E2B60
:1047480063D003F0DF03452B02D020EE070A704741
:1047580010B451782D294FD02B2979D0A1F13003ED
:10476800092B02F101027AD80024002303EB83030A
:1047780001EB430312F8011FA1F130000928A3F14E
:104788003003F3D9B3F59A7F1A4628BF4FF49A72CB
:10479800072B6CD9DFED386A1346F7EE007A083B31
:1047A800072B67EEA67AFAD802F00702DAB1F2EE22
:1047B800046A012A67EEA67A15D0022A67EEA67A5D
:1047C80011D0032A67EEA67A0DD0042A67EEA67ADE
:1047D80009D0052A67EEA67A05D067EEA67A062ADA
:1047E80018BF67EEA67A002C3BD087EE277A5DF8D3
:1047F800044B20EE070A70479178A1F13003092B8A
:1048080002F1020230D80124AFE75378A3F1300156
:10481800C8B2092802F1010293D8F2EE046AF0EE58
:10482800665A07EE901AF8EEE77A12F8013F87EE1B
:10483800A66AA3F13001C8B2092866EEA56A37EE68
:10484800067AEED97DE75378BFEE000A02465EE7A6
:104858009178A1F13003092B02F1020284D9F7EE15
:10486800007A27EE277AC2E7F7EE007ABDE7F7EE7F
:10487800007A9BE70000000020BCBE4CF8B5064655
:1048880015460846B6FBF2F434B905FB14640C4B24
:104898001B5D00F8013BF8BDB4FBF2F75FB905FBFF
:1048A8001747074B05FB1464DA5D00F8012B1B5D05
:1048B80000F8013BF8BD3846FFF7E0FFEFE700BF1F
:1048C8003C380308B5EEC00ADFED677A674AF1EEB7
:1048D80010FACCBF30EE270A30EE670ADFED647AB3
:1048E80020EE270A2DE9F047FDEEC07A88B017EED2
:1048F800904A84EAE4760023A6EBE476CDE9023315
:104908000493A2FB06325FEAD208054641D105AFFF
:1049180058483946554BA3FB0623DB0803EB8303B2
:10492800A6EB4303002CC35C0B704FF00002ACBF36
:1049380020232D234A7038468DF808302AF0D6FCFB
:104948000128394639D0022842D0032805BF302330
:1049580002A802A88DF809302BF0E8FD02A82AF079
:10496800C5FC0338C4B2224602A928462BF014FE1F
:1049780000232B5528462AF0B9FC2E22431C02A9F5
:104988002A542144E8182BF0EDFD284608B0BDE86C
:10499800F087394BA3FB06235B0922D105AF3548C5
:1049A8003946324AA2FB0832D20802EB8202A8EB4F
:1049B8004202835C01F8013BACE7302302A88DF882
:1049C80009308DF80A308DF80B302BF0AFFDC5E7B4
:1049D800302302A88DF809308DF80A302BF0A6FD97
:1049E800BCE7264AA2FB06125FEA92190ED105AF70
:1049F800204839461D4AA2FB03C2D20802EB8202B4
:104A0800A3EB4203C35C01F8013BCAE71C4AA2FBC3
:104A180006125FEA523A0ED105AF16483946134AD4
:104A2800A2FB09C2D20802EB8202A9EB4202825C15
:104A380001F8012BDEE71348B6FBF0F058B905AFD3
:104A480039460A20BAFBF0F200FB12A20948825C40
:104A580001F8012BE3E705AF39460A220193FFF776
:104A68000DFF019B0146ECE76F12033ACDCCCCCC8D
:104A780000007A443C3803081F85EB51D34D62107F
:104A88005917B7D1A08601000F4B2DE93048D3E95B
:104A9800004554EA05020AD1034640F201120020FB
:104AA8001880988098715A801881BDE83088074B23
:104AB8001A6814EB020B45F1000C5A466346FBF7E3
:104AC8002FFD0120BDE8308810590020F035002066
:104AD80030B403888278C478144DA3F2B27303F01B
:104AE800030101EB4101013A02EB81029B0835F811
:104AF80012500279611E40F2B55404FB03132B4493
:104B080003EB430302EBC303427981790089C3EBCA
:104B1800031302EB8303C3EB031301EB83034FF48B
:104B28007A720021C2FB030130BC7047BC0D030838
:104B380002B370B48E1803E0121B14D1B14215D021
:104B480010F8012BA2F14103192B11F8013BA3F135
:104B5800410598BF2032192D03F12004ECD9D21A4F
:104B680001D1002BEAD1104670BC704700221046D4
:104B780070BC7047104670474FF0FF32FFF7D8BF40
:104B8800A0F16103192B98BF20387047A0F14103A9
:104B9800192B98BF20307047202805D009380428E1
:104BA8008CBF002001207047012070476138192808
:104BB8008CBF002001207047413819288CBF002085
:104BC80001207047303809288CBF00200120704729
:104BD800A0F13003092B07D920F02000413819280B
:104BE8008CBF0020012070470120704730B4026854
:104BF8001146531C036011F8024B0160D31C517815
:104C080003609378151D05601B0443EA0123D078DF
:104C1800234343EA006030BC704700BF0368591C57
:104C28001A46016012F8021B0260587841EA002017
:104C3800704700BF03685A1C02601878704700BFAD
:104C48002DE9F04FB64B1D788DB0002D40F0C18096
:104C5800B44BB54C1E78DFF808B3DFF808A3A4F10D
:104C68000A0706F0010607F26E2854F80A3C3BB31F
:104C78004FF0CC0909FB05791846FDF793FBF8B10D
:104C880054F80A0CFDF786FB14F8023C03BB2428F1
:104C98003BD054F80A3C1A46002EEDD1232864D0A4
:104CA800A249897C8142E7D1A14BA249CBF80010E7
:104CB800C3F80CA013461846FDF774FB0028DFD193
:104CC800CC34444505F10105CFD10DB0BDE8F08FD6
:104CD800012B20D0022B28D0032B37D0042B00F037
:104CE8006C81052B6FD114F8063C14F8051C14F8D8
:104CF800042C994200F2B081904200F0C581002353
:104D080004F8023C54F80A3CB6E7012304F8023CD4
:104D180054F80A3CB0E74D2854F80A2C0CBF02237B
:104D2800002304F8023C1346C5E700233C2804F896
:104D3800023C00F04F813E2848D10323012204F8A9
:104D4800023C04F8012C54F80A3C95E7C028D6D850
:104D58000423002204F8023C04F8050C04F8040CAF
:104D680004F8062C54F80A3C86E773497348C97856
:104D7800734ADFF8E0C19361003118BF0121017067
:104D88007049C2F888104021C2F88C3082F890101F
:104D980082F891606C496D480B608832CCF800202D
:104DA8005F4A0123137016F037F9694815F050FE71
:104DB8004FF4006023F0E8FC5C4B9B7C232B00F055
:104DC8005A8114F8023C062B00F0618154F80A2C31
:104DD80070E7604B186800283FF477AFFEF73EFF96
:104DE800DFF864A1DFF88081DAF80000FDF7DAFA6D
:104DF80000283FF46AAFDAF80000DFF87091FDF799
:104E0800C9FA0928D9F800601AD03F2818D0002E0E
:104E18006CD1042800F0D1810C2800F0C7807F28CD
:104E2800E2D0A0F12003DBB25E2BDDD82028DBD056
:104E3800731C08F80600C9F8003015F001FED3E726
:104E4800002E65D1444B354603F58C77002D46D0AE
:104E58000833BB42FAD1DFF818B12868DBF8002024
:104E6800845D935D9C42304402EB060140F0A981C9
:104E7800741E4444324613B9FD2A40F2E38004F814
:104E8800013F0132C9F8002010F8013F11F8017FF5
:104E98009F42F0D00AB15D4513D0304815F0D8FDD7
:104EA8005D4508D855F8080B15F0D2FD092015F016
:104EB800C7FD5D45F6D9264815F0CAFDD9F800208A
:104EC8000026964290D2741E444414F8010F15F03F
:104ED800B7FDD9F8003001369E42F6D384E703F1D6
:104EE8000802BA421D46B6D01346AFE70C285DD07B
:104EF8000A2877D00D2875D07F2800F01D81FF2E55
:104F08003FF672AFA0F12003DBB25E2B90D96BE7BE
:104F1800114C4FF0000B04F58C775D462DE000BF77
:104F28007163002045460020923D0020743900201E
:104F380000ED00E0EFBEADDE144B00207C500020F9
:104F4800A8220020BD030008242A0020A038030856
:104F58006C380308202A0020D81003086438030896
:104F6800FC9F00200400FA05282A0020282B002096
:104F7800E81103080834BC420DD032462168404687
:104F8800FFF7D6FD0028F5D1A346002DF2D125461E
:104F98000834BC42F1D1002D7FF45FAFBBF1000FA4
:104FA8003FF422AF8B4815F053FD7BE78A4815F094
:104FB8004FFD8A4815F04CFD16E714F8043C04F838
:104FC800030C5840052304F8023C04F8040C54F878
:104FD8000A3C51E6032204F8013C04F8022C54F878
:104FE8000A3C49E615F0B3FD23217D482BF0ADFAC4
:104FF80000283DD0A0EB0802C9F800209AB1531E42
:1050080018F80310202940F0DE80023A424405E0F7
:1050180012F80109202840F099800B46591E002BF0
:10502800F6D1C9F800304FF48072002140462BF0C9
:1050380075FA6C4B1B78002B3FF447AE674815F0A8
:1050480007FDD1E6511C202008F80200C9F800101D
:1050580008F801300A461EE709EB03014240013314
:1050680004F8063C04F8042C887254F80A3C03E659
:10507800D9F80020C2E75C4A14F8023CC2F80CA038
:105088005A4ACBF800209EE6062304F8023C14F89E
:1050980001CCBCF1000F0CD0BCF1010F6ED0002385
:1050A80004F8023CCC34444505F101057FF4DDAD3C
:1050B8000BE64F4B08940FCB0DF1300E0DF1100994
:1050C80089E80F0014F8053C4EF824CD14F8032C99
:1050D80001922344724609934FF0010EBDF8043043
:1050E800ADF82AC0494608A8ADF828308DF82CE05C
:1050F80023F052FB48B1CC20049A3E4B494600FBB2
:105108000570CDE9043219F065F8DDF80C9000233C
:1051180004F8023CB9F1000F3FF4D2AD54F80A0C80
:1051280019F038FECC3454F8D60CC847444505F17C
:1051380001057FF49AADC8E5013E00232E48C9F861
:10514800006008F8063015F083FC4DE6C9F8003019
:105158002A4C002204F58C7708F8032002E0083472
:10516800BC4232D0216840460CF0A2FB0028F6D0A1
:10517800BC422AD263689847002352E714F8053CDA
:1051880014F8032C0894234409936E2A4FF0000363
:10519800ADF82E30CDF82A30ADF828207FF47FAF57
:1051A80008A8FFF747FD08A8FFF738FD08A8FFF78C
:1051B80035FD08A8FFF732FD71E7094807F038FB0D
:1051C80083E5324666E61346C2E70D4815F040FC13
:1051D800D2E700BF64380308743803086C38030842
:1051E800282A00207163002000ED00E0EFBEADDE4C
:1051F800B80E0308686C00209C380308D810030810
:105208008038030838B50446006815462BF06CF85A
:1052180022682A44226038BD036810B40A0A5C1C5C
:1052280004601A7003685A1C026019705DF8044B18
:10523800704700BF03685A1C026010B419700368F5
:105248000A0A5C1C04601A7003680A0C5C1C04607F
:105258001A700368090E5A1C026019705DF8044B35
:10526800704700BF03685A1C026019700368090A76
:105278005A1C0260197070472DE9F043002489B068
:1052880006460D461F46A04605E025290CD03046A7
:105298000134A847039A531C039311780029F4D1C9
:1052A800204609B0BDE8F083931CCDE90338507857
:1052B800302842D0A0F13003DBB2092B4FF00009AF
:1052C80045D96C282AD0642873D019D9732858D0A6
:1052D80063D9752840F0828007F1040C386805AB63
:1052E80000220A216746FBF7CFF805AB049A009322
:1052F80029464B463046FBF7CDF9039A0444CAE7E2
:1053080025283CD051D958286BD06328C2D1397888
:105318003046A84704370134039ABCE7039B5A1C5C
:1053280003921B78642B52D016D8252B27D064D92A
:10533800582B18D0632BEAD0ADE7D31C0393907891
:10534800A0F13003DBB2092B4FF00109B9D804AA48
:1053580003A90FF027F8B4E7732B12D051D9752B96
:105368002DD0782B97D1A3F15802B2FA82F238687F
:10537800520905AB10210437FBF786F8B5E725215C
:1053880085E73B68049A0093294600233046FBF7DB
:1053980081F904370444039A7DE76E287FF47AAFD5
:1053A800039A3B6804371C6075E700283FF478AF20
:1053B80070E7386805A9FBF731F8043795E73868CE
:1053C80005AB00220A21FBF75FF804378DE73B1D88
:1053D800386805A91F46FBF721F886E778287FF487
:1053E80059AFA0F15802B2FA82F23868520905ABF7
:1053F8001021FBF749F8043777E7002B3FF450AF4B
:1054080049E76E2BCDD046E70EB400B584B005ABA6
:10541800019053F8042B0649039301A8FFF72CFFCA
:10542800019B00221A7004B05DF804EB03B07047CA
:10543800910600082DE9F04707468CB01E469246B3
:10544800002A5DD1154614460A8840F2B1739A4283
:1054580036D98B78581E0B2832D891F803C00CF136
:10546800FF301E282CD891F804E0BEF1170F27D87A
:1054780091F80590B9F13B0F22D888793B281FD8BD
:10548800B1F80880B8F57A7F1AD24FF001085EBBF0
:1054980009890491002CB4BF2D212B21002CB8BF01
:1054A8006442CDE90290CDE905140795CDE900CE17
:1054B80038462B49FFF7A8FF40460CB0BDE8F087F7
:1054C80000232849ADF828304FF0010C18468DF814
:1054D8002A30ADF82C3099469E461A4698460991CE
:1054E800634609A9002ED3D0CDE90290CDE900CEBC
:1054F80038461D49FFF788FF40460CB0BDE8F087E5
:105508001A4C84FB0234A318D417C4EB6314C4EBFD
:105518000415A2EB85052DB2002D0846B8BF6D42D3
:10552800FFF7D6FA4FF47A720023804689462AF0AC
:10553800ABFB3C230AFB030A4FF47A720023404674
:1055480049462AF0A1FB4FF47A7192B20023C1FBBD
:105558000A2309A8FAF7E4FF24B209A974E700BFEF
:10556800C838030800000101A8380308898888881A
:105578000FB430B583B006AB0A490B4853F8042B77
:10558800096800680193FFF777FE084C0546A06993
:10559800FCF7FCFE0028FAD0284603B0BDE83040EE
:1055A80004B070479C520020A0520020A82200207E
:1055B800DFED2B7AB4EEE70AF1EE10FA4ADDDFED03
:1055C800296A9FED297A01E0B0EE670AB4EEC70AAE
:1055D800F1EE10FA70EE667AF6DC9FED247AF4EEBE
:1055E800C77AF1EE10FA38D5DFED1E6A9FED207A02
:1055F80001E0F0EE407AF4EEC77AF1EE10FA37EEF9
:10560800A60AF6D4DFED1B7AB4EEE70AF1EE10FA3B
:1056180014DDDFED137A37EEC00A60EE006A9FED05
:10562800166A9FED167ADFED167AA6EE867A20EED8
:10563800266AE6EE877AA6EE270A7047DFED117A2A
:10564800B4EEE70AF1EE10FA44BFDFED087A37EE60
:10565800C00AE2E7F0EE407ABFE7B0EE670AD1E7AA
:10566800DB0F4940DB0FC940E4CB1641DB0F49C0D3
:10567800E4CB16C1DB0FC93F92E741B99730083C2C
:1056880015A82ABEDB0FC9BF09B909E0194690FB66
:10569800F1F301FB13030846002BF7D108467047C6
:1056A80001460846704700BF07EE901AF8EE677A81
:1056B8009FED837A27EE800A20EE070AFDEEC07A76
:1056C80017EE903A2033402B00F28180DFED7D7A8F
:1056D800B4EEE70AF1EE10FA40F3E680B0EE407A55
:1056E8009FED796ADFED796A01E0B0EE677AB4EE92
:1056F800E67AF1EE10FA77EE467AF6DC9FED747AE8
:10570800F4EEC77AF1EE10FA40F1D1809FED6E6A9F
:10571800DFED706A01E0F0EE477AF4EEE67AF1EE3A
:1057280010FA37EE867AF6D4DFED6B7AB4EEE77AC4
:10573800F1EE10FA40F3A780DFED627A37EEC77A10
:1057480027EE076ADFED655ADFED657ADFED656AFA
:105758009FED655AE6EE257A67EE065AE6EE276A69
:10576800F7EE007AA5EEA67AF0EE675AE7EE055A4C
:10577800E7EE457A87EEA55ADFED577A30EE277ABD
:10578800FDEEC76A16EE903A2033402B24D99FEDE0
:10579800577AF6EE006AB7EE006AF7EE004AC4EEF2
:1057A800A57A0023836143610362C36180ED045AD3
:1057B80067EEA66A27EE866A27EE877AC0ED006A4A
:1057C800C0ED026A80ED016A80ED037A7047B7EE9A
:1057D800005AF0EE455ACFE7B4EEE70AF1EE10FAB8
:1057E8006BDD9FED396ADFED396A01E0B0EE677A6B
:1057F800B4EEE67AF1EE10FA77EE467AF6DC9FED33
:10580800347AF4EEC77AF1EE10FA53D59FED2E6A8A
:10581800DFED306A01E0F0EE477AF4EEE67AF1EE79
:1058280010FA37EE867AF6D4DFED2B7AB4EEE77A03
:10583800F1EE10FA33DCDFED2E7AB4EEE77AF1EE12
:1058480010FA44BFDFED227A37EEC77A27EE076AEF
:10585800DFED224ADFED226ADFED227AE6EE246AE6
:1058680067EE064AE6EE267AB7EE006AA4EEA77A55
:10587800F6EE006A36EE476AF8EE007A27EE277AE7
:1058880066EE266A89E7DFED1A7AB4EEE77AF1EE7A
:1058980010FA44BFDFED0E7A37EEC77A50E7DFED36
:1058A800097A37EEC77AD1E7F0EE407A26E7B0EE0C
:1058B800677A39E7B0EE677AB6E7F0EE477A9EE79F
:1058C80027D4D236DB0F4940DB0FC940E4CB164161
:1058D800DB0F49C0E4CB16C1DB0FC93F92E741B9E2
:1058E8009730083C15A82ABEF304353F0000000095
:1058F800DB0FC9BF70B406688E4217D90139751E0F
:10590800002311F8014F0822634013F0800F4FEA7B
:10591800430318BF83F0D503013ADBB2F5D18D42BA
:10592800EFD1721C0260337070BC7047721C002388
:105938000260337070BC704710B44C09012250F8F3
:10594800243001F01F0102FA01F10B4340F8243022
:105958005DF8044B704700BF2DE9F04F2DED068B25
:10596800904B914A1C7800F59C4720379BB006461F
:105978001760002C01F0E4808C498D4A0968079271
:10598800884284BF04F1FF341C708A4B1268069366
:10599800894B0593894B099302F48052002A41F000
:1059A8007980874B1B78022B01F08280042B01F051
:1059B8007A82012B00F0F285824B099A9E429278F6
:1059C80000F23686002A40F036867F4B0893079B04
:1059D8001E68059B16F48057B3F9064040F0E88628
:1059E800069BDFF800825D8BA542CCBF0025012510
:1059F800764A089B12681B7812F0805203F0010364
:105A080000F05985002B40F00A85714C002184F87C
:105A18006011002D00F011856E4901200870002BDF
:105A280040F01C856C4B1B78002B40F0A280069B35
:105A3800059A598BB2F900009A8B654C8142B4BF24
:105A48008023002382420598B0F90200C8BF43F0C2
:105A580040039B088142BCBF63F07F03DBB28242F4
:105A68000598B0F90400C8BF43F040039B08814281
:105A7800BCBF63F07F03DBB282420598B0F9060031
:105A8800C8BF43F040039B088142BCBF63F07F035B
:105A9800DBB2824294F86221C8BF43F040039A42C5
:105AA80001F0C9824D4A84F8623111780022A4F8C5
:105AB800642184F86621002901F095835F2B58D072
:105AC8006F2B56D0089A079B12781B68D20703F0F1
:105AD800040301F17B8394F86611002941F0768371
:105AE800B4F96421322A41F3718394F862210120C8
:105AF800572A84F8660101F05B830BB15A2A27D034
:105B08005D2A01F08E875B2A01F073875E2A01F017
:105B18008C87562A01F0F187972A02F01180A72A6C
:105B280001F0C387DFF8C0A0BAF800309B0742F045
:105B38003480A2F1B703072B02F20E80DFE813F0DE
:105B4800FA100C100C100C10F1100C10E810DF10EB
:105B580094F8852094F86831002A41F0C38783F0CF
:105B6800010384F86831002B42F0B2800C2021F048
:105B78004DFC079BDFF870A01B6803F00403002BA3
:105B880041F01E80164DDDF814B00DF158090023C0
:105B9800C9F80430CDE9183316932C46CDE90A5AD2
:105BA80030E000BF54310020AC27002050310020E5
:105BB800183D00204839002048630020285B002059
:105BC80030290020404B4C0045460020BC2B0020CB
:105BD800A82200200C520020C0670020D802002014
:105BE800BC310020203200205C490020314618A832
:105BF800FBF7CAFA054670B95745C2F07D800534EF
:105C0800A04537D02678272EF9D82379A77894F895
:105C180003A0012BEAD1574580F0F3820125AC4659
:105C28006178043140F6330E3BF911007045A8BF86
:105C38007046B0F5617F4FF0190140F2833EB8BF5E
:105C48004FF4617011FB07E7874280F2E18211FB94
:105C58000AE28242B4BF00270127BCF1000F40F0DE
:105C6800D282BD42CBD0314648460534FFF764FEA8
:105C7800A045C7D19DF859009DF861109DF858605E
:105C88009DF860309DF8622041409DF85A008DF8DB
:105C98005910734042408DF858309DF85B009DF8CC
:105CA80063308DF85A2043408DF85B30484B494AA1
:105CB8001B7899E80300DDE90A5A82E80300002B03
:105CC80040F08286444B1B78002B00F0A985434B9B
:105CD8000A9340480121FBF757FABAF8006020B947
:105CE800099BDB78002B00F095823D4B1B689A07D7
:105CF80040F19082F30741F1EB8233B223F00203C3
:105D08009BB2B342AAF800300AD0364B41F20241A6
:105D1800FF2219800E209A7021F078FBBAF80060F3
:105D2800314B1978314BB607586801F0020100F081
:105D38007083003118BF0121FCF72CFF242125486E
:105D4800FBF722FA30B9089A1378580744BF23F0B2
:105D5800040313700C211F48FBF716FABAF8003039
:105D6800002800F0358343F480729A42AAF8002094
:105D780008D01C4B41F20241FF2219800E209A7074
:105D880021F044FB1A4B1B78082B00F02E830E2BB6
:105D980000F02B83079BD3F8008018F4806F60D045
:105DA800144B1B79002B40F08D83089B1B78D90777
:105DB80000F18F8327F07AF9012021F07FFA00287B
:105DC8004CD0DFF834900B9400264FF0CC0B18E041
:105DD80086410020BC2B002071630020644900200C
:105DE8000849002054350020DC370020E037002027
:105DF800A02D002028470020883D0020DEB2032E79
:105E08002BD00BFB06F8731C59F80870002FF5D13E
:105E1800032290F9023002970192C278E44951F8BE
:105E28002220009218463A463B46012121F0F4F818
:105E380006EB460202EB0212044609EB820240B16D
:105E4800101D3946C8222AF069FB013649F8084076
:105E5800F6B20EF03BFB0028D1D10B9C079BD3F880
:105E68000080089B93F800B0D24B1BF0010B00F0A8
:105E7800368201221A700A9BCF481A68059B5189FD
:105E8800B3F9063001268B42067080F21082CB4AA5
:105E98004FF07E511160069AC94E178B059A96F9F4
:105EA8000410B2F90020307896F801E00029A2EB3E
:105EB800070614BF01214FF0FF31002EB8BF76420C
:105EC800B6F5FA7FA8BF4FF4FA768642C6BF361AEF
:105ED80007EE906ADFEDBB7ABB4EC8BFF8EEE77AF3
:105EE800BA42059AC6ED007AB2F902C0B8BFF1EE1F
:105EF800677AACEB0702B8BFC6ED007A002AB8BFD4
:105F08005242B2F5FA7FA8BF4FF4FA729042BCBF72
:105F1800121A07EE902A059AA8BFDFEDAA7AB2F9FD
:105F28000400B8BFF8EEE77A6745A0EB0702C6EDB4
:105F3800017AC4BFF1EE677AC6ED017A002AB8BFCC
:105F48005242B2F5FA7FA8BF4FF4FA72964580F232
:105F5800AB81A2EB0E0201FB02F107EE901AF8EEFC
:105F6800E77A8742C6ED027A9849C4BFF1EE677AAC
:105F7800C6ED027A18F48058087800F08281B3F5EB
:105F8800FA6FA8BF4FF4FA63B3F57A7FB8BF4FF43E
:105F98007A73A3F57A73002841F008808C49DFF8FA
:105FA80044C281FB0320DA17C2EB6012501C6FF069
:105FB800630E3CF910003CF912C00EFB0233A0EB53
:105FC8000C0003FB00F381FB0321DB17C3EB611318
:105FD8009C440FFA8CFC07EE90CAF8EEE77AC6EDFF
:105FE800037AB8F1000F40F01585BAF800305A0668
:105FF80040F1FC807749784A91ED018A92ED027A66
:1060080092ED014AD1ED033AD2ED006AD1ED028A50
:1060180092ED036AD1ED005AD6ED011A96ED002AE9
:106028006E4A6F4938EE635A74EE470A76EE867AFE
:1060380065EE200A75EEE84A36EEC69A75EEA89A1D
:1060480064EEA74AB0EE603AA9EE893A13F003036A
:10605800B0EE645A38EE231A74EE077AA9EE895A1C
:10606800A1EE273AB0EE600A91EE270AA1EE675A30
:1060780033EE243AF0EE407AB6EE000A35EE88AAFE
:10608800B0EE671A20EE433A35EE605A76EE840A8F
:10609800A9EEC91AAAEE203A77EEE47A77EE460A14
:1060A80033EEE8AA25EE005AE9EE897AAAEE205ADC
:1060B80071EE244A36EEC44A63EE036A73EEA83AD8
:1060C80064EE804A75EEC85A37EE066A67EE807A43
:1060D800B0EE667AE3EE844A95EE057AE5EE056A57
:1060E800E5EE867AB1EE648AF0EE665AF0EE476A1B
:1060F800B1EE674AE8EE246A63EE270A67EEA43A2F
:10610800E4EE275AB1EE450AB0EE606AB0EE631AC3
:10611800A4EE277A23EE244AE7EEA76AA5EE246ABE
:10612800A0EE031AE8EE245AB0EE448A31EEA19AA2
:10613800E0EE240AA5EE278A66EEA16A72EE028ACC
:10614800E5EE033A61EE211A26EE096AA4EEA47A76
:10615800A0EE274A0CBFD6ED022ADFED1A2A82EDFF
:10616800005AA2EE256AE8EEA06AE2EE081A73EE7B
:10617800A33A27EE227A34EE044AF0EE005AE2EE11
:10618800A36AA2EE846AA1EEA57AC6ED016AC1ED02
:106198005C6A81ED5B6A86ED006A81ED5D7A82ED6D
:1061A800013AC2ED027AC2ED034AFBB91CE000BF16
:1061B80078360308464600203C520020C051002093
:1061C800582D00200000000038470020844D002092
:1061D8001F85EB51DC02002090020020C80200203D
:1061E800A8220020E44F002086ED027ABBF1000FC0
:1061F80040F0478218F070F81BB0BDEC068BBDE884
:10620800F08F00270125314618A8FFF795FB28E5F0
:10621800002722E526F001039BB2B342AAF800301A
:106228000AD0C24B41F20241FF2219800E209A7017
:1062380021F0ECF8BAF80060BD480221FAF7A4FF93
:1062480033B200283FF45AAD23F001039BB2B342A6
:10625800AAF800300AD0B54B41F20241FF2219805A
:106268000E209A7021F0D2F8BAF80060B7073FF50F
:1062780057AD46F00203B342AAF800307FF445ADAB
:106288004EE5069A528B934280F23C8143460028A1
:106298003FF484AE4A78A74903FB02F381FB03125B
:1062A800DB17C3EB621379E6DFEDA37A59E6B3F5A2
:1062B800FA6F127A9FEDA17ABFBF581A4243C1F50F
:1062C800FA6192FBF1F2C2F1640207EE902AF8EE4D
:1062D800E77A9B4A67EE877AC2ED007ADBE593F8A6
:1062E8000090B9F1000F7FF4C6AD964B1B68002BE8
:1062F8003FF4C1AD944B954A13F8030C0793194624
:10630800DE1E577816F03AF8079B002801F06C80DB
:10631800002F41F07F8306F10801707916F02EF8FE
:10632800002841F07A838A49B07A16F027F80028C5
:1063380001F06C80022F41F080838649F07B16F0D3
:106348001DF8002841F075838349307D16F016F852
:10635800002801F06C80042F41F07F837F49707E14
:1063680016F00CF8002841F074837D49B07F16F0D0
:1063780005F8002801F06C80062F41F06683794902
:1063880096F8230015F0FAFF002841F05A83764961
:1063980096F8280015F0F2FF002801F06C80082F0D
:1063A80041F07F83714996F82D0015F0E7FF00282A
:1063B8003FF461AD0923994603EB83031E44634808
:1063C8006B4B7178B27880F8019019705A7052E569
:1063D80023F4807292B29A42AAF800207FF4C9ACE2
:1063E800644B1B78082B7FF4D2ACBAF8002022F05B
:1063F80040039BB29A42AAF800303FF4CBAC4B4B17
:1064080041F20241FF2219800E209A7020F0FEFF0F
:10641800C0E4B1FA81F14909FCF7BCFB8EE40699A6
:10642800498CA14240F3EF85002D7FF4F5AA524C28
:1064380094F8601100297FF4EFAA50485049006889
:1064480090F82D0000240C604C608C6000287FF4CC
:10645800E3AA4C490870002B3FF4E4AAF1067FF543
:10646800E1AA494B1B78DB063FF5DCAA002F7FF435
:10647800D9AA002A7FF4D6AA77023FF5D3AA434BBC
:106488001B78002B01F05883414B9B78002D41F07D
:1064980043833BB13F4A404B12681B689B1A002B51
:1064A800C1F219841020344C20F0B0FF012384F885
:1064B8006131FFF7B7BA70027FF5A7AA002BAED1FA
:1064C800FFF7A3BA14211A48FAF75EFE00283FF432
:1064D80071AC4FF40F700FF043FA00283FF4BEACD4
:1064E80018F00AFD4FF40F700FF0F8F900283FF488
:1064F800B5AC18F001FD4FF40F700FF0EFF900285C
:10650800EED1ABE4B3F5FA6FD4BFC2EB030CC2F51E
:10651800FA6C4FF47A73C2F5FA6203FB0CF3B3FB1F
:10652800F2F300283FF43AADB4E600BF543500203A
:10653800BC2B00201F85EB51000000000AD7233C2C
:10654800C0510020484600202F2B002000000020CA
:10655800392B00203E2B0020432B0020482B002005
:106568004D2B0020522B0020572B00205C2B0020A5
:106578004C460020A02D0020A822002060490020C1
:10658800E42800200C52002095690020D802002041
:10659800802D0020F0350020945000208D4CD4F838
:1065A8005C31F31A002BFFF607AA8B4A8B4B527CFF
:1065B800DFED8B7A33F812309FED8A6AC4F85C718C
:1065C80006EE903A069B9A7DD97D07EE102AF8EEE2
:1065D800E66AB8EEC77A66EE866A27EE277A40F250
:1065E800FF32C6EE877AFCEEE77A17EE903A9BB256
:1065F800934228BF13461D4609B1D31A9DB27A4C5F
:106608007A4922787A4F31F81230386821F81250D6
:10661800C31A2B4477493B6001321B0902F00F0271
:106628000B80754B2270099A9E4292787FF6CAA910
:10663800002A00F0FB84714B099A1C7892F82150CB
:1066480008931B2015F0D2FE012D04F001078146A6
:1066580000F0118604F00204099A694E92F820307D
:10666800DFF8B0A1DFF8B0810A949346052B00F259
:10667800C184DFE813F06F003305130085001705A8
:106688003605604B1978604B01F001011868FCF77A
:1066980081FA1BB0BDEC068BBDE8F08F012D04BF5D
:1066A80005238BF8203097B1069B3088B3F9181072
:1066B8000022134661F30F0361F31F4361F30F02D6
:1066C800059960F31F420B6003234A600A934F4CFD
:1066D800DBF814102268914280F0418647F230516D
:1066E8000322CBF81C108BF82020022022F04CF853
:1066F80016F058FD2168DBF81C200A440421CBF869
:1067080018208BF82010012D41F0B4812268DBF8A5
:106718001810914280F06E849AF80000002800F06A
:106728006484D8F8002022F00202C8F80020226809
:106738007388642101FB03234FF480600022CBF8A7
:1067480010308BF820208BF8032021F0EDFF9BF808
:1067580020308BE7002F01F0978116F0CDF9012842
:1067680000F0AE84B9F1000F0CD0B37953B115F035
:10677800C3FD03224FF47A738BF82020CBF81C302A
:10678800224CB2E7012D00F03584204CDBF81010C4
:1067980022689142C0F0898401238BF82030F37974
:1067A800012B00F0D08515F0A7FD9BF820305DE7A0
:1067B8001D211748FAF7E8FC002800F0DF85DFF80C
:1067C8005C80069B5D8BA542CCBF00250125FFF7A9
:1067D8000FB900BFA822002088400020A840002050
:1067E8000000C842000080443129002038290020D8
:1067F80034290020205B0020404B4C0045460020F7
:10680800B04F0020DC370020E0370020F0350020B2
:10681800BC2B0020D802002058490020203200203C
:10682800DFF814B3DFF81493B34E0A930BF15A0749
:106838004FF0010859461BF8010C15F09FFDE8B10F
:106848009BF804009BF8023000EB400106EB810145
:10685800013B8A6A03EB43034B4493420ED096F8FC
:1068680069218B6208FA00F022EA00009BF80330E5
:106878000A9ACA6286F8690181F824300BF1060B7E
:10688800BB45D7D19D4B9E4A0A9319469D4B9E4EB8
:10689800D2F800B009681B780C910B93A6F1240874
:1068A8004FF000095F467368002B00F0838093F86F
:1068B80000B0BBF1000F7DD0B168791A00290BDB5D
:1068C80098F86911012000FA09F021EA000107F59A
:1068D800FA7088F86911B0600B9A002A6AD031788A
:1068E80058780431C9B2002840F01883069A108BF2
:1068F800059A32F911C098F8691100F1C80EF445EB
:1069080040F3878341FA09F1C8079B7852D4002BDA
:106918000CBF012002200D9320F056FE0BF1FF3131
:106928000D9B16293AD8DFE811F05F077407430773
:10693800170031071707FD06E306CD06B706A106BF
:10694800390017002B001707FD06E3063A068B06E9
:1069580050060906F10520060C9A6C489179807852
:1069680019446429A8BF642121EAE171917120B119
:106978000D200D9316F0DEF90D9BBBF10D0F0DD018
:106988000C9A62485179807819446429A8BF642117
:1069980021EAE1715171002841F09D80D8F8540036
:1069A80015F02CF998F86911012303FA09F30B4340
:1069B80088F8693109F10109B9F1040F06F10C06EB
:1069C8007FF471AFFFF785B9514B03E005339C4263
:1069D8003FF478A919782329F8D19878DA78904281
:1069E800F4D24C48FAF7D0FB00283FF46BA94A4B85
:1069F8001B689E0300F1EA87484B00221946087875
:106A0800142801F10C0100F030870132182AF6D160
:106A1800FFF758B91D213F48FAF7B6FB28B100F037
:106A2800BEBC0535A5423FF4E0AA29782629F8D14D
:106A3800AA78EB789A42F4D2099BDB78002B7FF492
:106A4800D4AA3448FAF7A0FB9FED357A354A77EE99
:106A5800C77AFDEEE77A17EE903A1BB21B0382FB6A
:106A68000312DB17C3EBA213002800F05B87C7F5FE
:106A78007A7212B203FB02F343F30F333B4407EE7F
:106A8800903A294BF8EEE77A0122C6ED037A1A709C
:106A9800FFF7ABBA00211F48FAF776FB00287EF40F
:106AA80080AF16F07FFB214B1B78022B7EF47EAF64
:106AB800069A0599537DD27D013B31F913301AB1FD
:106AC800C3F53B6308331BB2A3F57A7307EE903A1C
:106AD8009FED177A174AF8EEE77A40F2FF3167EE32
:106AE800877AFCEEE77A17EE903A9BB28B4228BF82
:106AF8000B461380FEF760BFA822002064490020DF
:106B0800F0350020195B0020CC2200207A6200209A
:106B1800BC310020BC2B0020AC32002060230308CD
:106B280000007A44D34D62103052002030290020F2
:106B38006F12833F205B0020602B0020C80E0308E3
:106B4800324B1D78002D00F0C084DFF8D4B0304DF2
:106B5800DFF8C8A00695DFF8CC90D84626E0295D76
:106B68009847032C034629DCC8B109EB840339F89C
:106B780024105A88401A4FF47A7303FB00F0521A13
:106B880040F6CA0390FBF2F000F57A709842A8BF6D
:106B9800184640F2EE239842B8BF184600B21B4B85
:106BA8002AF8020B1B7801349C423DDA072C404638
:106BB800DBF80430D3DDE1B29847034618B2EEE7BC
:106BC800144C94F868315BB1089B1B78DF0707D534
:106BD800059BB3F90620069B5B8B9A4200F38884D9
:106BE80011210D48FAF7D0FA002800F0EC8194F84A
:106BF80084302BB994F8853013B93223A4F868305F
:106C0800012384F88430FEF7BDBF00BF9532002011
:106C180048390020A8220020BC2B00207C2300201B
:106C2800982700209A3200201D46A64BA64A0793B3
:106C38001B68A2FB061242F2010B920913EA0B0B26
:106C48000E9200F0BC81A14CA149A248A24A94F836
:106C580000C0097880F800C01170BCF1000F04D0A2
:106C68009D4A92F800C08CF0010C9C4C4FF00F0923
:106C780084F8F890002D00F0C4820699984A109282
:106C88001078CA8C09920A8B1492964A0592964AF1
:106C9800B1F824E00F90A2FB0021490801EB410163
:106CA800411AC9B203F48053681E0C9115934B0026
:106CB8000E99DFF8608294F8F9A0CDF82C9003289B
:106CC800A8BF032001F59672CDE911750A92854D8A
:106CD8000D930246A1466046002377461396089115
:106CE8005C469446002800F02D82804A32F9132031
:106CF8001FFA82FEBE454FEA430103D3099EB645FB
:106D080040F2F48158F82320089E964280F02482AD
:106D18006A5E002C40F0F081013363456A52E1DD80
:106D2800129D139EAB42A346BE468446119F4C4615
:106D380060DA6F4A1295580000EB030902EB490923
:106D480048320D920E9A119602F5967165460A918F
:106D58000E97089277460599DDF848C0A6465C4626
:106D6800CDB1624A125E1FFA82FB5F4502D8099EC6
:106D78005E4513D258F82320089E964280F006827A
:106D88000A5E84B9013363450A5209F106092ED017
:106D98005800002DE5D1002FECD13A460A9E48F85C
:106DA8002360002CEED00C9E29F81620BAF1000FB3
:106DB80002D10F9E022EE5D9B9F80220B9F800B029
:106DC800B9F804A05A4492444A4A0FFA8AFA82FB54
:106DD8000A62A2EBEA720D9E013312B2634526F8ED
:106DE80000A009F106094FF0010A0A52D0D10E9FFE
:106DF800119E74460B99404B84F8F9A00F290CBFDB
:106E08000122002284F8F8101A7000F001823B4C2D
:106E18002F49314ADFF800B10994012304200B708F
:106E2800137021F0B1FCDBF80030A1686268E36000
:106E38005B1A934202D9002384F82130304B18782A
:106E4800079B1A6802F4805238B3069B254DB3F8A5
:106E58002480B3F818E02B49002A40F056821346E4
:106E68000CE09CF8014004EB840404EB840404F275
:106E7800EE240133984225F8024B0ED011F8134046
:106E880001EB430C002C00F0A581022CE9D0013362
:106E98002C8825F8024B9842F0D110990B780133D1
:106EA8000B70FEF77BBDFBF7E1F8174B174A1B6821
:106EB800C31A93427EF780AD154B00221A80FEF765
:106EC8007BBD00BF183D0020D34D62107427002001
:106ED80020000020195B002021000020A8220020AB
:106EE8007131002048630020ABAAAAAA7C230020A5
:106EF800A423002056555555C42B0020285B00209C
:106F0800953200202D3500201859002060E3160026
:106F1800205B002074310020F035002001287FF428
:106F280041AD059A987832F9111040F63303994229
:106F3800A8BF1946B1F5617FB8BF4FF46171BBF1C5
:106F48000C0FA1F561714FF4966393FBF0F391FB7D
:106F5800F3F100F0BE84BBF1180F7FF423ADC9B282
:106F6800D8F85400C8290B4690F817E0A8BFC823E2
:106F78005FFA83FCF4453FF415ADB3EB0E0348BF4D
:106F880007334FEAE30BBD4B80F817C09B780BF132
:106F9800010B5FFA8BFB002B40F0FD82BBF1000F69
:106FA8003FF400AD584620F00FFBFBE44A78B449A3
:106FB80003FB02F3A1FB03235B09FEF7EFBFB14A12
:106FC80092F800C049E694F88530002B3EF4DAAD1B
:106FD800089B1B7813F001037EF4D4AD012284F8DA
:106FE800853084F88620FEF7CDBD15F0FFF900281E
:106FF8003FF497AB0A9C002C3EF4E9AC204620F005
:1070080005FAFEF7E4BCA04C012184F86011FEF7F4
:1070180003BDC838844580F2118441FA09F1C907D3
:107028009B783FF5C7AC5B42012074E4099A0123C1
:107038009370FFF700BB954895490068B4F96461FF
:10704800C76981FB07018911FF17781A00F5FF400E
:107058007F30864240F3FE838E490978002900F08C
:10706800C2805F2A00F04A846F2B7EF42BADB6F500
:10707800FA7FFEF67EAD94F86621002A7EF479AD9B
:10708800089B1B78012184F86611D90700F1A784B1
:1070980017F0A2FA079BDFF834A21B6803F0040379
:1070A800FEF76DBD7C4CFFF72EBB15F025F90321CB
:1070B80040F6B8328BF82010CBF81C20FFF715BB30
:1070C800754C72882368642101FB0233CBF81030B9
:1070D800B9F1000F3FF456ABFFF747BB012D7FF422
:1070E8005EAB6D4CFFF723BB3A4659000A9E48F841
:1070F8002360002C3FF410AE684E01EB030B06EB47
:107108004B0E0D9E2EF80620BAF1000F03D10F9EEC
:10711800022E7FF601AE614EBEF80220BEF804E0F2
:1071280036F81BA0724492445D4A0FFA8AFA82FB31
:107138000A625C4EA2EBEA7226F801A012B24FF086
:10714800010AE9E5002FCFD058F82320089E96427F
:107158004FEA4301FFF4DCAD534E725C06EB010EBF
:10716800002A7FD0022A40F084809EF8012002EB9A
:10717800820202EB820202F2EE22012606FA03FEE6
:107188000B9E26EA0E0612B20B96C2E5464E325CFC
:1071980006EB000B002A5CD0022A61D19BF8012083
:1071A80002EB820202EB820202F2EE2212B2E8E560
:1071B8003E4A3F4910684FF47A72B2FBF0F2C2EBD4
:1071C800421002EB8002D200A1F8A820DFF8FCA050
:1071D800FEF7D5BCDCB2022C40F26781032C7FF4A9
:1071E80056AE444645E600213248F9F7CDFF00285F
:1071F80000F04E81002384F8673117F0EDF9FEF7AF
:1072080061BC2D4B2D4A109201221A702C4B05930C
:107218001B212848F9F7B8FF00287FF4F8AD294862
:10722800DFF874B0C168DBF80030079A8360126831
:1072380009905B1AC82B02F480527FF62EAE2249C1
:107248000B6823F004030B601E4B012083F8210018
:1072580023E6DAB2022A40F20683032A00F03F81CD
:107268000A5AA3E7DAB2022A40F2FB82032A00F0A4
:1072780030816A5A81E70024FFF7EEB97A6200206C
:107288001F85EB51195B0020A8220020646C0020A8
:10729800D34D6210D8020020F0350020A42300202E
:1072A80056555555EC2300202D350020083D00206B
:1072B800903A0020BC2B0020C42B00207131002004
:1072C80048630020285B0020584900205C490020C2
:1072D80046F00103B342AAF800303EF40EADC64BA7
:1072E80041F20241FF2219809A700E2020F08EF898
:1072F800BAF8006033B223F002039BB2B342AAF893
:1073080000307EF402ADFEF70BBD00230DE09CF8C3
:10731800014004EB840404EB840404F2EE240133FA
:10732800834225F8024B3FF4B8AD11F8134001EB46
:10733800430C1CB1022CEAD02C88F0E7DCB2032CF9
:10734800FAD87446EBE714F0D7FF032240F6B833B7
:107358008BF82020CBF81C30A84CFFF7C6B9A84AF8
:107368001278002A7FF4BAA9002F3FF4B7A9012D9B
:107378007FF440AE9BF82030FFF778B9A14B03F1BA
:10738800640803E00533984500F091801A78262AAE
:10739800F8D19978DA789142F4D2FFF712BA099BBA
:1073A800DB78002B7FF441AB9FED977A974977EE16
:1073B800C77AC7F5FA63FDEEE77A1AB217EE903A84
:1073C8001BB21B0381FB0301DB17C3EBA11302FBF9
:1073D80003F343F30F333B4407EE903AF8EEE77AB2
:1073E800C6ED037AFFF721BB591D707914F0C6FF6B
:1073F80000283EF498AF012F40F00F8306F10D01ED
:10740800B07A14F0BBFF002840F017838049F07B66
:1074180014F0B4FF00283EF497AF032F40F009831F
:107428007C49307D14F0AAFF002840F016837A4981
:10743800707E14F0A3FF00283EF497AF052F40F0AC
:1074480008837649B07F14F099FF002840F0FD8248
:10745800734996F8230014F091FF00283EF497AF83
:10746800072F40F0EE826F4996F8280014F086FF47
:10747800002840F016836C4996F82D0014F07EFF22
:1074880000283EF4F8AC092F3EF4F5ACFEF792BFA5
:10749800089B664A1B781060DE0700F1FD81079B98
:1074A8001B6803F00403FEF716BB7446E1E4604A68
:1074B800069BD5881B8B5A1BA24216DA2B44A34283
:1074C800CCBF00250125FEF793BA5A4B0693FFF768
:1074D800ACBBDDE91426002E08BF3A464DE6DDE9CF
:1074E8001426002E08BF3A4660E60125FEF780BA4A
:1074F80000215148F9F748FE00287FF471AB322388
:1075080084F86801A4F86830FFF76ABBD8F854001B
:107518004A4A90F8371092781944FE29A8BFFE21EC
:1075280021EAE17180F83710002A3FF439AA1620C1
:1075380015F000FCD8F85400FFF732BA0C9A5178CD
:107548001944B1F5967FA8BF4FF4967121EAE1710D
:107558003A4B51709B78002B3FF420AA152015F068
:10756800E9FBD8F85400FFF71BBAD8F85400334A9F
:1075780090F83610927819446429A8BF642121EA4A
:10758800E17180F83610002A3FF40AAA172015F096
:10759800D1FBFFF703BA182015F0CCFBFEE4D8F8AE
:1075A800540001781944C829A8BFC82121EAE1710B
:1075B800224B01709B78002B3FF4F2A9122015F0A2
:1075C800B9FBD8F85400FFF7EBB9D8F85400817824
:1075D8001944C829A8BFC82121EAE171174B817055
:1075E8009B78002B3FF4DCA9142015F0A3FBD8F8F6
:1075F8005400FFF7D5B900BF54350020F0350020FE
:1076080004520020BC31002000007A44D34D62109F
:107618003E2B0020432B0020482B00204D2B002020
:10762800522B0020572B00205C2B00209850002064
:10763800D44C002048390020BC2B00207A6200205E
:10764800D8F8540041781944C829A8BFC82121EAAC
:10765800E171BD4B41709B78002B3FF4A1A9132029
:1076680015F068FBD8F85400FFF79AB9D8F8540019
:10767800B54A017A92781944C829A8BFC82121EAD5
:10768800E1710172002A3FF48BA90B2015F052FB1F
:10769800D8F85400FFF784B9D8F85400AA4AC17939
:1076A80092781944C829A8BFC82121EAE171C1719B
:1076B800002A3FF475A90A2015F03CFBD8F85400BD
:1076C800FFF76EB9D8F854009F4A81799278194427
:1076D800C829A8BFC82121EAE1718171002A3FF4B5
:1076E8005FA9092015F026FBD8F85400FFF758B910
:1076F800D8F85400944A417992781944C829A8BF07
:10770800C82121EAE171417132B111200D9315F0C0
:1077180011FBD8F854000D9BBBF1110F7FF457AF44
:10772800FFF73EB9D8F85400874A0179927819448E
:10773800C829A8BFC82121EAE171017132B110201E
:107748000D9315F0F7FAD8F854000D9BBBF1100F04
:107758007FF478AFFFF724B9D8F854007A4AC17893
:1077680092781944C829A8BFC82121EAE171C170DB
:1077780032B10F200D9315F0DDFAD8F854000D9BA7
:10778800BBF10F0F7FF40DAFFFF70AB90C9A6E48E3
:10779800D1798078194481F30801D17100283FF428
:1077A800FDA8052015F0C6FAD8F85400FFF7F8B878
:1077B8000C9A92F804B09B44BBF1640FA8BF4FF039
:1077C800640B2BEAEB7B82F804B015F0CDFA5E4B24
:1077D8009B78002B3FF4E2A80320594615F0AAFA3B
:1077E800D8F85400FFF7DCB80C9A11781944FA2934
:1077F800A8BFFA2121EAE171534B11709B78002B45
:107808003FF4CCA8012015F095FAD8F85400FFF7FA
:10781800C7B80C9A917819446429A8BF642121EA51
:10782800E171494B91709B78002B3FF4B7A8022077
:1078380015F080FAD8F85400FFF7B2B8012303FA1C
:1078480009F321EA030107F5FA7388F86911B360AF
:10785800FFF7B0B8C91B0E4436B2A4F86461FFF74D
:10786800FBBB149A89E4149AA0E4384807685100CD
:107878003FB18E1803EB86067F787678BE42BEF459
:1078880021AA0A44324E334903EB820300220360E3
:1078980032800A60FEF716BA2F4B1B78002B3EF495
:1078A80068A9099BDB78002B7EF463A994F86731FB
:1078B8000133DBB2032B84F867317EF65AA9274BD4
:1078C8005B7813B9002D7EF454A915F06BFCFEF714
:1078D800F9B8234B5878CBB298423FF463A81846BE
:1078E8000D9316F0F7F9184B99780D9B002940F085
:1078F800E98001335FFA83FBFFF750BBB6F5FA7FE7
:10790800FEF637A994F86631002B7EF432A9089B5D
:107918001B780122DD0784F8662125D515F042FC85
:10792800FEF727B9C7F5FA6212B203FB02F343F375
:107938000F333B4407EE903A0A4BF8EEE77A18709B
:10794800C6ED037AFEF751BB7A620020FC4F002097
:107958000050002004500020195B0020802D0020DA
:10796800144B002030520020C84B1B68980378D471
:10797800C74B00211A4610780F2802F10C0210D0CC
:1079880001311829F7D1079BDFF840A31B68FA3E9D
:107998000022A4F8646103F0040384F86621FEF76A
:1079A800EEB8BC4807684A0037B1551803EB85059F
:1079B8007F786D78BD42E6D20A44B74DB74903EBEC
:1079C8008203002203602A800A60DCE7B44B1B783C
:1079D800032B7FF411A81FF0FDFCFEF773B9079B7A
:1079E800B0491B680A6003F00403DFF8E0A2FEF761
:1079F800C6B8AD4B01220220AC49AD4C0B602270D9
:107A08001FF0E2FD079BDFF8C4A21B6803F0040324
:107A1800FEF7B5B84B46FEF7CFBC01239946FEF7F3
:107A2800CBBC00220120A34BE6E7A34B0222032094
:107A3800E2E703239946FEF7BFBC02239946FEF707
:107A4800BBBC07239946FEF7B7BC06239946FEF749
:107A5800B3BC05239946FEF7AFBC04239946FEF74D
:107A6800ABBC8F4B1B78032B82D11FF0B3FCB4F94E
:107A7800646188E7A3460999DBF80020CB690A9C72
:107A880013448B61FFF7B7BA0A9C4FF48060B9F1D1
:107A9800000F1DD020F060FE099A00231361FFF744
:107AA800AABA08239946FEF787BC8449079B0A7837
:107AB8001B68DFF818A242F004020A7003F00403FE
:107AC800FEF75DB81946584615F034F90D9B10E7D6
:107AD80020F02AFEE0E70E2015F02CF9D8F8540023
:107AE800FEF75EBF84F8851084F88600DFF8DCA115
:107AF800002B3FF475A8FFF767B807F0EDFAFCF71D
:107B08000DFB07F08FFAFCF71DF901201FF05CFD53
:107B180094F86221FEF700B8002B40F0E480684C2E
:107B280094F86131002B3DF47DAF1FF053FC002326
:107B380084F86131FDF776BF002DF0D1FEF7B2BCB5
:107B4800079B604A1B68DFF884A14FF4C871118055
:107B580003F00403FEF713B89E2A50D09D2A7ED066
:107B6800AE2A75D0AD2A00F08A80EF2A00F0848012
:107B7800FD2A7ED0FB2A79D0FE2A66D0F72A52D079
:107B88007B2A04D14FF4FA61022015F0B9FF079B54
:107B98001B6803F00403FDF7F2BF0023BB2A189308
:107BA8003DD0B72A36D0BE2A30D0BD2AD4D14FF620
:107BB800FE73ADF86030444BBDF862009989DA89EC
:107BC800BDF86050024429449981DA8107F084FAAB
:107BD800FCF7A4FA07F026FAFCF7B4F801201FF026
:107BE800F3FC079BB4F864211B68FA3A0021A4F857
:107BF800642103F0040384F86611FDF7C0BF002177
:107C0800012028F051FB94F86221A7E70223ADF880
:107C18006030D0E74FF6FE73ADF86230CBE7022351
:107C2800ADF86230C7E70021042015F069FF079B13
:107C3800B4F864211B68963A0021A4F8642103F083
:107C4800040384F86611FDF79ABF00210320ECE7CE
:107C58000121002028F028FB94F8622182E7002106
:107C6800FF2028F021FB94F8622179E70021022007
:107C7800DBE700210120D8E700210846D5E7FF21EE
:107C8800002028F011FB94F862216EE7AC32002046
:107C980060230308FC4F00200050002004500020FF
:107CA80094590020985000208461002060490020E9
:107CB800144B002036610020D26100209569002015
:107CC800A82200208E500020602D00205C49002052
:107CD8000B20FDF74CBF1C4C15F064FA002384F808
:107CE8006131FDF79FBE1949194A09684FF47A7046
:107CF80000FB0313136012E78446FDF791BF0220CF
:107D080015F0E8FF079B1B6803F00403FDF737BF76
:107D1800032015F0DFFF079B1B6803F00403FDF742
:107D28002EBF002015F0D6FF079B1B6803F0040345
:107D3800FDF725BF012015F0CDFF079B1B6803F059
:107D48000403FDF71CBF00BFA8220020F035002067
:107D58009450002008B540F2E93300E09BB1028955
:107D6800013B12F0020F9BB2F8D0017340F2E933E5
:107D780000E043B10289013B12F0010F9BB2F8D039
:107D8800007BC0B208BDFBF7DDF8C0B208BD00BF7C
:107D980038B50D4A0D4C00F0EF03C02B0CBF012184
:107DA800002105461068FBF74BF8D4F8E030B4F82A
:107DB800E4201A8506482946FFF7CCFFD4F8E030BE
:107DC800B4F8E4209A6138BD044500201838002032
:107DD800003800402DE9F041454CC37A94F88C21D5
:107DE800444F9A423B70884604D004F5BC7142481F
:107DF800F8F7CAFD414D1E23002605F1480085F815
:107E08004E3085F84F600BF04BF905F15003052211
:107E1800184685F8562085F85760C4F890310BF05D
:107E28009FF8D4F89001FAF7A9FE3B780B2B47D0BE
:107E38000823334D88F800307D600EF03DFE05F1D3
:107E480010000BF011FE31462E48FAF709FF10B169
:107E5800D4F87831FBB9002384F898312A4B1A7882
:107E68000AB903221A700F2015F02CFEC020FFF764
:107E78008FFFFAF7FBF87A68D4F8C0315268C4F873
:107E8800B82101330022C4F8B401C4F8C031C4F8E1
:107E9800BC21BDE8F0811D4DC4F89C31A5F1240337
:107EA8000FCB85E80F0094F8B03103F00F03E11809
:107EB800012291F8A01184F8B03184F89821CDE717
:107EC8000E22134B134988F80020134A09681B68CF
:107ED8001268124D7D604B405340C4F894310EF047
:107EE800EBFD05F110000BF0BFFD0D21ACE700BF65
:107EF800A822002000000020807303081838002002
:107F0800540F03086038002030290020482400203E
:107F1800ACF7FF1FB0F7FF1FB4F7FF1F100F0308E0
:107F2800F8B5114F114E0446F0200D46FFF730FF0B
:107F3800D7F8E030B7F8E4201A8545213046FFF736
:107F480009FF013D54FA85F5013CFF213046FFF752
:107F580001FF04F8010FAC42F7D1D7F8E030B7F8C9
:107F6800E4209A61F8BD00BF1838002000380040AE
:107F78002DE9F047C74C94F820308AB0002B53D035
:107F8800814600254020D4F81CA084F820500BF02E
:107F980051FD00F00303022B94F8986100F0D7809C
:107FA80010F0210840F0EA80BB4F3B780B2B00F023
:107FB800F780002E00F0E68015216846FFF7B0FF35
:107FC8009DF80030552B00F0FA81C0204546FFF798
:107FD800DFFE94F8986194F8C631002B4ED1002E3C
:107FE8005CD1FAF743F8D4F8D031AC4AC01A9042C1
:107FF80016D994F8A0319BB1D4F89C3183B1A84E1E
:10800800C4F8783106F124030FCBA34D2D7884F8FA
:108018008C51012586E80F0084F89851FCF75AFB2B
:1080280028460AB0BDE8F08703F0FF05B4F8C4316C
:1080380001339BB2B3F57A7FA4F8C431C9D940F2B1
:10804800E933A4F8C431FAF711F8964B0246A3FBBA
:1080580002129209A3FB02139B094FF47A7101FBE8
:108068001323B3F5FA7FD4F8900177D9FAF786FD90
:1080780094F8C63194F89861002BB0D0F9F7F6FF60
:10808800D4F8CC31C01AB0F5FA7FA8D9D020FFF7C0
:108098007FFE002384F8C631002EA2D07E4FF9F768
:1080A800E5FF7E680246D6F800C0D4F8D401652101
:1080B80001FB0CF1101A88420ED9D4F8C011C4F88B
:1080C800D42163299ABFC1F1640189B20021002338
:1080D800A4F8C811C4F8C031D4F8D811F368511AFB
:1080E800994204D90123C4F8D82184F8C731D4F8B7
:1080F800B401D4F8B811131A8B4291D9B3FBFCF62A
:10810800012E98BF4218A020C4F8B421FFF740FE02
:1081180094F8B031334403F00F03E2180F2092F8BB
:10812800A01184F8B03115F0CDFCC020FFF730FE67
:10813800D4F8BC311F2B14D87A681268C4F8B82157
:1081480001332846C4F8BC310AB0BDE8F087002ED8
:108158003DD1C020FFF71CFE00253CE7FAF714FDCF
:1081680037E7514B7A681B789268C4F8B821032B1B
:108178007FF456AF4D4B00221A8051E7C020FFF71D
:1081880007FE28E705216846FFF7CAFE9DF800307C
:10819800AA2B00F08D80C0203546FFF7F9FD18E7BF
:1081A8002EB3E84640462521FFF7BAFE9DF8003079
:1081B800582B00F0C980AA2B00F0C680562B00F07F
:1081C800C38094F8C651002D60D0002501E794F8CB
:1081D800B031013303F00F03E2180F2092F8A01119
:1081E80084F8B03115F06EFC94F89861B1E7E84670
:1081F80040461B21FFF794FE9DF80030AA2B00F0A3
:10820800A38040F29C80BB3B012BDAD87A68D4F873
:10821800C0315268C4F8B8219DF80B20C4F8B4A145
:108228000133FF2AC4F8BC61C4F8C03100F00681EC
:108238000AAD04F5D07655F81D0D6968AA68EB6893
:108248000FC64FF0FF33D4F89421DDF80110CDF8B4
:108258000520CDF80B3001226B60AB60EB602B6121
:108268006B612B83E020C4F89C1184F8C621C4F804
:10827800D0A1C4F8CCA1FFF78BFD414625220520EB
:1082880015F0F8FB94F8C651002D9ED1C020FFF7D9
:108298007FFD9EE6A822002000000020400D03007C
:1082A80024240020D34D621030290020205B0020B8
:1082B80035467868DDF801604068D4F8C031C4F804
:1082C800B801C6F3031001309449954AC4F89C617B
:1082D80006F00F0C013300270928C4F8B4A128BF01
:1082E800092001EB0C11C4F8C03102F11006C4F8E2
:1082F800BC7111F8013B1B1A02F8013FB242F8D1D8
:1083080094F8B03103F00F03E2180F2092F8A0118F
:1083180084F8B03115F0D6FBC020C4F8D0A1FFF71F
:1083280037FD022D7FF455AE0023D4F89001A4F850
:10833800C4310225FAF728FC94F898614BE6562BCD
:1083480002D0582B7FF43DAFDDF80520D4F89431E6
:108358009A427FF436AFDDF80120D4F89C319A4276
:108368007FF42FAFF8F7BEFED4F8C03179689DF8D6
:1083780000204968C4F8B4A101330025582AC4F87C
:10838800B811C4F8C031C4F8BC515AD094F8C631F9
:10839800002BC6D194F8B031013303F00F03E21873
:1083A8000F2092F8A01184F8B03115F08BFB94F8E7
:1083B800C631002BB5D1C020FFF7EAFCB1E7DDF8E4
:1083C8000120D4F89C319A427FF4FFADF8F78AFE79
:1083D800D4F8C0317A68C4F8B4A15268C4F8BC8132
:1083E8000133C4F8B821C4F8C031B9F1000F0DD079
:1083F8000AAB53F8232DC9F8002059689A68DB683E
:10840800C9F80410C9F80820C9F80C3094F8B0313C
:10841800013303F00F03E2180F2092F8A01184F83B
:10842800B03115F04FFB94F898311BB99DF8003026
:10843800AA2B25D0C020FFF7ABFC75E70DF10B0583
:10844800FFE6B9F1000F16D00AAB53F81F0DC9F8B3
:1084580000009A685968C9F80820DA68C9F8041051
:108468001869C9F80C2059699A69C9F81000C9F83F
:108478001410C9F8182094F8C7311BB9022585E7EC
:10848800022516E7274BA18A1B88B4F8C8213E7A33
:108498008DF80F1003EB83035B009BB28DF80B3054
:1084A8001B0A080A402E4FEA12218DF80C304FF0B3
:1084B800FF334FF0000528BF40268DF813208DF8B4
:1084C8001000FC228DF81410CDF81930AA21CDF82F
:1084D8001530CDF81D30CDF82130E020FE238DF881
:1084E80011308DF800108DF80D208DF809508DF899
:1084F8000A508DF80E508DF81250FFF749FC32469D
:108508004146052015F0B6FA1522012384F8C75113
:10851800C4F8CCA13A7284F8C63105E7980F03086D
:108528004724002094370020F8B584894FF6FF7659
:108538004FF47A742BB311B30F78013101E0B442D0
:1085480017D00589013CAD07A4B2F8D507734FF4DD
:108558007A7402E0BCB2B4420BD00589ED0704F18D
:10856800FF37F7D5057BEDB20AB115700132013B33
:10857800E0E7FAF7E7FC003018BF0120F8BDFF2755
:10858800DFE70120F8BD00BF028822F04002120494
:10859800120C0280038823F038031B041B0C69B1FA
:1085A80041F48071002991FAA1F1B1FA81F108BF73
:1085B8004FF0FF31013943EAC1039BB203800388BE
:1085C80043F04003038070472DE9F84F314ADFF844
:1085D800D4A03148DFF8D0B0304F01230421137004
:1085E800FFF7D2FFDAF80000FAF7C8FA05212A489F
:1085F800FFF7B0FB00212848FFF7ACFB062126480F
:10860800FFF7A8FB00212448FFF7A4FB9BF80040D4
:108618002148042144F00104FFF79CFB21461E4831
:10862800FFF798FB3B88B3B1DFF880801C4D1A4EEA
:10863800444615F8019F07213046FFF78BFB494652
:108648003046FFF787FB2B7804F8013B3A88A4EB08
:1086580008039A42EDDC07210F48FFF77BFBFF2157
:108668000D48FFF777FB9BF800400B480421FFF704
:1086780071FB21460848FFF76DFBDAF80000FAF7AE
:1086880083FA02210448FFF77FFF024A0023137090
:10869800BDE8F88F7263002000300140CC03002051
:1086A800575B002098390020B867002080630020BD
:1086B800F8B5114D114FC1F1030646EA80060421B1
:1086C8002846FFF761FF3868FAF758FAF6B210241F
:1086D800E1B22846FFF73EFB013431462846FFF752
:1086E80039FB202CF4D13868FAF74EFA02210248F7
:1086F800BDE8F84048E700BF003001409839002045
:10870800F8B5424C42480421FFF73EFF2068FAF7CB
:1087180035FA404B1B78012B6CD057D3022B4ED126
:108728003D4D08232B704FF4C3733C4E3C4F3380B0
:1087380002210020FFF7BCFF04213548FFF724FF82
:108748002068FAF71BFA2D7831480021FFF702FB61
:1087580029462F48FFF7FEFA324B2D481D78022193
:10876800FFF7F8FA29462A48FFF7F4FA2E4B28486B
:108778001D780321FFF7EEFA29462548FFF7EAFAA4
:108788002A4B23481D7804210D43FFF7E3FA2946B5
:108798001F48FFF7DFFA2068FAF7F6F902211C48AC
:1087A800FFF7F2FE32882248002127F0B7FE7B7AD5
:1087B80023B1204B1B781BB300237B72F8BD164DE9
:1087C8002B785B06AFD54FF4F073AEE7A0211048C5
:1087D800114DFFF7BFFA00210D48FFF7BBFA00F073
:1087E8000603022B03D000F0050001280BD0082354
:1087F8002B7098E7084D48232B704FF4F07394E7DB
:10880800FFF7E2FED8E748232B70DCE79839002011
:10881800003001409C390020B5050020CC03002021
:1088280000000020A3390020A4390020B8670020E8
:10883800806300207263002070B50F4C0F4DC0EBB1
:10884800C00004EB8004686926693043686182B01F
:108858009209667BA1600025012101A863618DF85A
:1088680004608DF805208DF806508DF807100EF07D
:108878008BF802B070BD00BFCC0000200010024091
:10888800074BC0EBC00030B403EB8000054C056912
:1088980063692B4363610176427630BC704700BF41
:1088A800CC000020001002402DE9F04F5F4C54F836
:1088B800204083B0002C71D0A66DA16098467368E3
:1088C800236504F15E0363614FF48073C4E90333E5
:1088D8009146574A226004F5AF72A2610746307E7E
:1088E8000AF020FBF068A8B1524B00215A68904268
:1088F80003F11C0300F0928001310C29F6D100200D
:108908007A1CD2B20C21FFF7BBFF236DF2686263B9
:108918002433E364B068D8B1464B00215A689042CA
:1089280003F11C037CD001310C29F7D100257A1CF6
:10893800D2B20B212846FFF7A3FF2346F27E3E4919
:108948002846FFF779FF236DB268A2632833A36432
:1089580094F85D00F9F7F4F9054694F85C00F9F726
:10896800EFF918F0080F824696F819B01AD0CDB171
:1089780018F0110F4FF00B0307F1010714BF4E2138
:108988003E21EF715A46AB712846F8F77DFE18F084
:10899800010F47D0636B6BB3A36B5BB3204603B087
:1089A800BDE8F08F18F0010F0CBF4FF02E084FF004
:1089B8004E0819F0020F09D045B10B227B1CAA7191
:1089C800EB7128465A464146F8F75EFE19F0010F4A
:1089D800E0D0BAF1000FDDD00C2301378AF8063059
:1089E8008AF807705A4641465046F8F74DFE636BC1
:1089F800002BD1D1337FB27E8DF804209B09002152
:108A0800012201A88DF805308DF806108DF8072091
:108A18000DF0BAFF204603B0BDE8F08FC8B26FE78B
:108A2800CDB284E72846FAF7A9F8B3E7085500203D
:108A380098100308CC0000207108000800B970479E
:108A4800F0B595B006460AF0ABFC614DC368026804
:108A58002A600446002B00F0AD803046F9F770F923
:108A68005C4BC3F8DC0118B1292200238271C37161
:108A7800227A594E2E21F8F707FE2868F9F788F967
:108A88000AF050FA2868554A038823F001031B04AA
:108A98001B0C03800F211E233380118000262D23F9
:108AA80001A90127CDE9017303960AF02BFCE379AC
:108AB800059660229907CDE90666089604927BD54B
:108AC800DB0003F008030422ADF81E30ADF81620D1
:108AD800002304AA617928680693F8F729FC6179CC
:108AE80028683F4F0AF0EEFB2B685A6C42F40042AC
:108AF8005A641A8842F080021A80E2796079196A09
:108B080092074CBF04220122824021EA0201196225
:108B1800196A0A431A621A8842F001021A80207CF4
:108B280000222921FFF7ACFE2E49207C0023602279
:108B3800FFF782FEE06838600DF096F93868036840
:108B48004FF6FE72134003600DF08EF909A80DF080
:108B58005DF92B686279244938680A9134331344E3
:108B6800099380221023002609A940F22A3C0E927C
:108B78000B934FF400724FF400530D961096139612
:108B880011960F921293ADF830C00DF04DF962793D
:108B98002B680C2A98BF1549D86898BF31F812601D
:108BA8003A6813490643DE601368012043F0020364
:108BB8001360087015B0F0BD5B0003F002034FF4BA
:108BC8008072ADF81C30ADF81470ADF820207FE746
:108BD800AC600020A8220020765D0020745D002093
:108BE800A860002061090008785D0020902903082A
:108BF800A66000200348D0F83C3113B100F59A7004
:108C080018477047CC0000200348D0F8203113B132
:108C180000F58C7018477047CC0000200348D0F846
:108C280004310BB1FC301847704700BFCC0000205E
:108C38000348D0F8E8300BB1E0301847704700BF60
:108C4800CC0000200348D0F8CC300BB1C430184712
:108C5800704700BFCC0000200348D0F8B0300BB1FB
:108C6800A8301847704700BFCC0000200348D0F850
:108C780094300BB18C301847704700BFCC000020EF
:108C88000248836F0BB1703018477047CC00002042
:108C98000248C36D0BB1543018477047CC00002010
:108CA8000248036C0BB1383018477047CC000020DD
:108CB8000248436A0BB11C3018477047CC000020AB
:108CC8000248836803B11847704700BFCC000020F2
:108CD800F8B50501594C5A4B625961199A4204EB8F
:108CE800050704BF01230B730646387A0AF01AF900
:108CF8003B7A03F01F015B090122022B02FA01F201
:108D080075D0032B6ED0012B64D063190136187906
:108D1800F9F716F8F6B2074610B11223C671837137
:108D280063195879F9F70CF810B11323C6718371D8
:108D380063199879F9F704F810B11423C67183718F
:108D480066190E21F2793846F8F79EFC7079F8F723
:108D5800F7FFF2790E21F8F797FCB079F8F7F0FFF2
:108D6800F2790E21F8F790FC6359364A934243D0C2
:108D7800334A934256D0344A934248D02C44227BFB
:108D88006ABB012102209A8822F480521204120C34
:108D98009A809A8842F480529A801A8802F4415242
:108DA80042F445720A4302431A809A8822F4706298
:108DB8001204120C42F4E0629A809A8B22F4006248
:108DC8001204120C07219A8319821A8842F0400271
:108DD8001A80F8BD1D4B996A0A439A6295E70021EB
:108DE8000846D0E7194B19690A431A618DE7174BF2
:108DF800D9680A43DA6088E702F56042D16841F42D
:108E08008051D160D16821F48051D160B6E702F574
:108E1800EA32116941F400411161116921F40041FC
:108E28001161ABE702F5EC32116941F4804111613F
:108E3800116921F480411161A0E700BF2C55002081
:108E48000038004000300140003C00400010024063
:108E58001749184B184A194810B4D1F8884044F4F7
:108E68007004C1F888401C6844F001041C605C6808
:108E780022405A601A6822F0847222F480321A6002
:108E88001A6822F480221A605A6822F4FE025A6094
:108E9800DA6A22F00F02DA621A6B002410404FF0EF
:108EA800006218639C608A605DF8044B704700BFDD
:108EB80000ED00E0001002400CC07FF8CCFC00FF81
:108EC80000230122C2708370038003714371837190
:108ED800C37103724372704700230A220360436020
:108EE800C381C0F80630C0F80A300280704700BF5E
:108EF800634B5B68C3F3080370B4B3B9EFF3118332
:108F08009BB9604A604D1368AC6800BF11688B421A
:108F1800F9D15E4A15684FF47A7101FB05F2121B0C
:108F2800B2FBF5F201FB032220E0EFF311841023DA
:108F380083F3128803F1E02355499D681A68D20328
:108F480042BF01220A609D684E4BE4B21E680B685E
:108F580084F311884D4A14684FF47A7202FB04F1C5
:108F68003344491BB1FBF4F102FB0312494B0021C6
:108F780019705978012913D9596840F6AC54511A17
:108F8800A1420DDD444909781B2907D11989434CB1
:108F9800013189B2012519816180A58000215970AC
:108FA800C0B27E2822D05A78F2B15A781B2A4DD8FE
:108FB80093F86C20002A5DD0002280F0200083F80E
:108FC8006C205A78022A03D1012808BF83F8600070
:108FD8009A7A5C785978C2EBC20203EB8202224487
:108FE8000131C9B2D072597070BC704759780129E3
:108FF80027D9997A2A48DC7A0131A0FB0150400828
:1090080000EB4000091AC9B28C4209D05C78987A02
:109018009972C0EBC00003EB8000611E80F8271036
:1090280093F8601029B101200021187083F86010AE
:109038005A66194909781B2917D000219A6683F8BE
:109048006C10012159705A6070BC7047124A12782E
:1090580000211B2A5970C7D11A891049013292B2CE
:1090680002201A814A808880BEE7996E0B48511AFF
:109078000180E2E77D28A4D1012283F86C20B3E7C0
:1090880000ED00E0F035002010E000E0143800208A
:1090980010380020D8240020104B0020084B002056
:1090A800ABAAAAAA03788B4283BF034B03EB410107
:1090B800B1F8700000207047D8240020044B93F8C2
:1090C800880018B1002283F888200120704700BF6B
:1090D800D8240020F0B4C24D95F8AF6005F18C0299
:1090E8000244B41E1444A24200F07881013A013CC3
:1090F800002341F2210112F8017F83EA07231FB2FE
:10910800BBB2002FACBF5B0081EA43039BB21F04D4
:1091180054BF5B0081EA43039BB21F0454BF5B004A
:1091280081EA43039BB21F0454BF5B0081EA4303F7
:109138009BB21F0454BF5B0081EA43039BB21F0428
:1091480054BF5B0081EA43039BB21F0454BF5B001A
:1091580081EA43039BB21F0454BF5B0081EA4303C7
:10916800A2429BB2C7D10644B21E013E2A442E44F5
:1091780092F88C1096F88C2002EB012292B29A4257
:1091880001D0F0BC704795F8B020002A00F021818A
:10919800431CDBB25C1C2C442B444FF4AF6193F8A6
:1091A8008C6094F88C3003EB06239BB201FB03F32D
:1091B8001B1303F54873012AA5F8703000F00981E4
:1091C800C31CDBB25C1C2C442B44022A93F88C6031
:1091D80094F88C3003EB06239BB201FB03F34FEAB0
:1091E800233303F54873A5F8723000F0F280431D6D
:1091F800DBB25C1C2C442B44032A93F88C6094F853
:109208008C3003EB06239BB201FB03F34FEA2333B5
:1092180003F54873A5F8743000F0DB80C31DDBB29A
:109228005C1C2C442B44042A93F88C6094F88C30F2
:1092380003EB06239BB201FB03F34FEA233303F549
:109248004873A5F8763000F0C48000F10903DBB25A
:109258005C1C2C442B44052A93F88C6094F88C30C1
:1092680003EB06239BB201FB03F34FEA233303F519
:109278004873A5F8783000F0AC8000F10B03DBB23E
:109288005C1C2C442B44062A93F88C6094F88C3090
:1092980003EB06239BB201FB03F34FEA233303F5E9
:1092A8004873A5F87A3000F0948000F10D03DBB222
:1092B8005C1C2C442B44072A93F88C6094F88C305F
:1092C80003EB06239BB201FB03F34FEA233303F5B9
:1092D8004873A5F87C307CD000F10F03DBB25C1C2E
:1092E8002C442B44082A93F88C6094F88C3003EBB8
:1092F80006239BB201FB03F34FEA233303F54873BC
:10930800A5F87E3065D000F11103DBB25C1C2C445B
:109318002B44092A93F88C6094F88C3003EB0623CD
:109328009BB201FB03F34FEA233303F54873A5F817
:1093380080304ED000F11303DBB25C1C2C442B446C
:109348000A2A93F88C6094F88C3003EB06239BB2BE
:1093580001FB03F34FEA233303F54873A5F8823082
:1093680037D000F11503DBB25C1C2C442B440B2ACC
:1093780093F88C6094F88C3003EB06239BB201FBC6
:1093880003F34FEA233303F54873A5F8843020D05C
:1093980000F11703DBB25C1C2C442B440C2A93F815
:1093A8008C6094F88C3003EB06239BB201FB03F32B
:1093B8004FEA233303F54873A5F8863009D000F146
:1093C8001903DBB25A1C2A442B4493F88C3092F8C8
:1093D8008C30012385F88830F0BC70470023C2E642
:1093E800D8240020794B5B68C3F3080370B5B3B980
:1093F800EFF311839BB9764A764D1368AC6800BFCA
:1094080011688B42F9D1744A15684FF47A7101FBDF
:1094180005F2141BB4FBF5F401FB034320E0EFF362
:109428001181102383F312886A4C6C4AA56823685B
:10943800DE0344BF01231360654B48BFA5681E685F
:109448001368C9B281F31188634A14684FF47A71BA
:10945800334401FB04F2521BB2FBF4F201FB032379
:109468005F4CD4F8B420C4F8B4309B1AB3F5FA5F53
:109478001AD9002384F8B83084F8B930A1282FD03D
:10948800A22800F09C8094F8B92094F8AF30002509
:10949800A2B16A1C6119D5B2C0B29D4281F88C0094
:1094A80084F8B8500CD070BD94F8B850002DE5D0B1
:1094B80094F8B92094F8AF30002AEAD19D42F2D14D
:1094C80094F8BA30052B72D0062B03D194F88D305E
:1094D8001E2B0DD0002384F8B83084F8B93070BD45
:1094E80001221B2384F8B92084F8AF300025D0E787
:1094F8006A1E002A4FF0000150DD08460B4623443F
:10950800013093F88C30DBB283EA0105ED074FEAAE
:10951800530348BF83F08C0383EA5105EE074FEAF3
:10952800530348BF83F08C0383EA9105ED074FEAA4
:10953800530344BF83F08C03DBB283EAD105EE0703
:109548004FEA530344BF83F08C03DBB283EA11155F
:10955800ED074FEA530344BF83F08C03DBB283EA81
:109568005115EE074FEA530344BF83F08C03DBB277
:1095780083EA9115ED074FEA530344BF83F08C0348
:10958800DBB283EAD1155908EB0748BF81F08C019B
:10959800C0B248BFC9B290420346B0DB224492F839
:1095A8008C308B4296D10320FFF794FD92E7002080
:1095B800FFF790FD94F88D301E2B8BD198E7012290
:1095C800232384F8B92084F8AF308FE700ED00E05A
:1095D800F035002010E000E014380020103800209A
:1095E800D824002007299DBF034B03EB8101B1F864
:1095F800BC000020704700BFD82400201A4B93F805
:10960800DC2032B193F8E0200021A82A83F8DC108E
:1096180001D00020704793F8F320002AF9D110B444
:10962800DFED126A03F1E00103F1B80003F1F00283
:10963800B4EE047ACC780B7903EB042307EE903A66
:10964800F8EEE77AB0EE666AA7EE876A02318A42D8
:10965800FCEEC67A17EE903A40F8043FEAD10120B2
:109668005DF8044B704700BFD82400200080BBC3BE
:1096780010B50446F8F7FAFC0F4BD3F8F820C3F8F6
:10968800F800801A41F288329042E4B205D983F892
:10969800E040012283F8FC2010BD93F8FC209918C3
:1096A800142A81F8E04003D1012283F8DC2010BDA0
:1096B8000132D2B2EEE700BFD8240020034B03EBFF
:1096C8004101B1F80001C008704700BFD82400204C
:1096D800724B93F82021002A00F0C28070B493F8EE
:1096E8002141B3F8225103EB4401002091F827618E
:1096F80091F8282183F8200142EA0622954202D0F7
:10970800002070BC704793F82521012A00F0AA8038
:10971800812AF6D10320102C40F2A68093F8294123
:1097280093F8275193F8281193F82A2141EA052143
:1097380042EA04221024A3F80011A3F8022183F8B6
:10974800214193F82B1193F82C21032C42EA012292
:10975800A3F80421D5D093F82D1193F82E21042CC9
:1097680042EA0122A3F80621CBD093F82F1193F8EF
:109778003021052C42EA0122A3F80821C1D093F830
:10978800311193F83221062C42EA0122A3F80A216A
:10979800B7D093F8331193F83421072C42EA012209
:1097A800A3F80C21ADD093F8351193F83621082C85
:1097B80042EA0122A3F80E21A3D093F8371193F8B7
:1097C8003821092C42EA0122A3F8102199D093F8F4
:1097D800391193F83A210A2C42EA0122A3F81221FE
:1097E8008FD093F83B1193F83C210B2C42EA0122CD
:1097F800A3F8142185D093F83D1193F83E210C2C41
:1098080042EA0122A3F816213FF47BAF93F83F11F7
:1098180093F840210D2C42EA0122A3F818213FF4C5
:1098280070AF93F8411193F842210E2C42EA0122BD
:10983800A3F81A213FF465AF93F8431193F8442134
:10984800102C42EA0122A3F81C217FF45AAF93F8A6
:10985800451193F8462142EA0122A3F81E2150E758
:1098680000207047104656E7002C3FF44AAF93F8A3
:10987800271193F82821012C42EA0122A3F800219C
:109888003FF43FAF93F8291193F82A21022C42EABA
:109898000122A3F802217FF454AF32E7D824002034
:1098A800654B5B68C3F3080370B4B3B9EFF3118376
:1098B8009BB9624A624D1368AC6800BF11688B425D
:1098C800F9D1604A15684FF47A7101FB05F2141B4F
:1098D800B4FBF5F401FB034320E0EFF311811023FF
:1098E80083F31288564C584AA5682368DE0344BFA0
:1098F80001231360514B48BFA5681E681368C9B29D
:1099080081F311884F4A14684FF47A71334401FB8C
:1099180004F2521BB2FBF4F201FB03234B49D1F8CA
:109928004C219A1AB2F57A6F17D891F85021C1F8DC
:109938004C31BAB1022A20D0242A91F8213178D9A1
:1099480001320233D2B25B009A4281F850211CDB0B
:1099580001339A4265D070BC70470022C1F84C317F
:1099680081F85021A828F6D1002281F82021A1F8F9
:10997800222191F82131044603E0C4B281F8214143
:1099880023468D1885F82441DAE7B1F82231C0B2B0
:1099980083EA002000B20028B8BF41F2210283B256
:1099A800B4BF82EA43035B009BB2180446BF41F28E
:1099B800210282EA43035B009BB21A0446BF41F2CC
:1099C800210282EA43035B009BB21E0446BF41F2B8
:1099D800210282EA43035B009BB21D0446BF41F2A9
:1099E800210282EA43035B009BB21C0446BF41F29A
:1099F800210282EA43035B009BB2180446BF41F28E
:109A0800210282EA43035B009BB21A0446BF41F27B
:109A1800210282EA43035B009BB2A1F8223170BCA9
:109A280070470022012381F8502181F8203170BC51
:109A38007047C4B2A5E700BF00ED00E0F035002094
:109A480010E000E01438002010380020D82400204E
:109A5800F8B5124D95F8692102B9F8BD104B1C688C
:109A68002368DE693EB1204605F5AA71B047002398
:109A780085F86931F8BD05F5AA77BE1800E02368B6
:109A88009B68204698470028F9D0236817F8011BDF
:109A98001B6820469847B742F1D1E8E7D824002050
:109AA800B468002003788B4210D9094B03EB81017D
:109AB80093F89C31D1F86C011BB900F5777080B22E
:109AC8007047400800F5777080B2704700207047F3
:109AD800D8240020324B5B68C3F3080370B4B3B9D1
:109AE800EFF311839BB92F4A2F4D1368AC6800BF61
:109AF80011688B42F9D12D4A15684FF47A7101FB30
:109B080005F2141BB4FBF5F401FB034320E0EFF36B
:109B18001181102383F31288234C254AA5682368F2
:109B2800DB0344BF012313601E4B48BFA5681E68B2
:109B38001368C9B281F311881C4A14684FF47A710A
:109B4800334401FB04F2521BB2FBF4F201FB032382
:109B5800184AD2F8A011C2F8A0315B1A41F2883134
:109B68008B420AD9C0B2012382F8A80182F8A43135
:109B7800002382F8B83170BC704792F8A4310F2BDB
:109B8800F9D8D1180133DBB2C0B2102B81F8A80183
:109B980082F8A431ECD1012382F8B83170BC704747
:109BA80000ED00E0F035002010E000E0143800205F
:109BB80010380020D8240020C36833F8110000EBC7
:109BC8008000C01000F55C7080B27047036993F89C
:109BD8002320002A00F0C3802DE9F043714ADC7D80
:109BE800127800211A2A04F0040604F0080583F804
:109BF800231000F0B680002E40F0BE801DB11A8CF4
:109C080042F001021A8493F80290997993F801C0FE
:109C1800C268DE7893F80480DF7909F0070001F064
:109C28000F014FEAC11E4CEA002106F03F06187AE0
:109C38001180997893F80AC0760146EAD106D97856
:109C480056804FEA880848EA911193F805809E7B70
:109C580008F0010841EA8821918059794EEA5101BA
:109C6800D18007F07F07997993F807E03F0147EA29
:109C78001117597A1781400040EADE1001F00301FC
:109C880040EA41205F7BD97A50810CF01F0C587A4A
:109C98004FEA8C1C4CEA90009081187B93F80AC01C
:109CA80007F0070740EA072006F03F065F7B1082AF
:109CB800C90041EA5C117601D18146EAD701518297
:109CC800D97B93F80E8093F810E093F811C0DE7CEE
:109CD8009F7C587D890041EA98110EF0010E41EAF7
:109CE8008E21918293F812E0197C0CF00F0C76000B
:109CF8004FEACC1C46EADE1E4CEA51011E7D93F861
:109D080011C0D18207F07F073F01997D47EA1C17F0
:109D180006F0030693F814C017834EEA46265F7DC3
:109D2800568314F0010F40F2147300F01F0014BFA3
:109D38001E46AD26800114F0020F4FEAC10140EA29
:109D48009C0008BFAD2341EA5711002D9083D183B1
:109D5800168453840CBF01200320BDE8F08310460D
:109D6800704711491F8C0C8066B147F002021A84B3
:109D780012B29DB94A8046E71A8C4DB942F00202E8
:109D88001A8440E745B147F001021A8412B2F1E79C
:109D980042F003021A8436E73AB2EBE747F00302CF
:109DA8001A84F3E7104B0020084B0020394B5B68FE
:109DB800C3F30803F0B413BBEFF31183FBB9364ABE
:109DC800364E1368B56800BF1468A342F9D1344A07
:109DD80016684FF47A7404FB06F2551BCA69B5FB82
:109DE800F6F504FB03539A1A40F6AC54A2422DDC54
:109DF80091F822406CB3182C37D9F0BC7047EFF3B8
:109E08001184102383F31288244D264AAE682B68E8
:109E1800DB0344BF012313601F4B48BFAE681F68B4
:109E28001368E4B284F311881D4A15684FF47A74F4
:109E380004FB05F23B44921BB2FBF5F204FB03233F
:109E4800CA6940F6AC549A1AA242D1DD002281F8C0
:109E580022200F28D1D10122CB61087081F822205D
:109E6800002381F82330F0BC7047631CDBB2192B48
:109E780081F822300855F3D10B4B1B781A2B08BFF9
:109E88000A4B4FF0010081F8230008BF9A80F0BC0C
:109E9800704700BF00ED00E0F035002010E000E062
:109EA8001438002010380020104B0020084B0020E8
:109EB800094BDFED0A6ADFED0A7A03EB810191EDC8
:109EC8006F7AB8EE477AE7EE267AFCEEE77A17EE75
:109ED800903A98B2704700BFD824002001F11F3F84
:109EE80000405C44714A92F8FC3133B192F8023276
:109EF8000021162B82F8FC1101D00020704792F83F
:109F08000132022BF0B440F2CE8002F50070184402
:109F180002F20221D32311F8014F634013F0800F9E
:109F28004FEA430318BF83F0D503DBB213F0800F69
:109F38004FEA430318BF83F0D503DBB213F0800F59
:109F48004FEA430318BF83F0D503DBB213F0800F49
:109F58004FEA430318BF83F0D503DBB213F0800F39
:109F68004FEA430318BF83F0D503DBB213F0800F29
:109F78004FEA430318BF83F0D503DBB213F0800F19
:109F88004FEA430318BF83F0D503DBB213F0800F09
:109F98004FEA430318BF83F0D5038842DBB2BAD136
:109FA80092F81912994202D00020F0BC704792F83A
:109FB800080292F8076292F80C1292F8103292F89E
:109FC800144292F80452B2F804C2D2F8047200F0B3
:109FD8000F00C00140EA560001F01F0192F80B6221
:109FE800C2F8C801890141EA960103F03F0392F8DB
:109FF8000F6292F81302C2F8D4115B0143EAD60348
:10A0080092F80312C2F8E03104F07F04B2F8083283
:10A01800D2F80862240105F0070544EA101041EA65
:10A028000521C3F30A13C2F8EC01B2F80C52C2F8C6
:10A03800BC11B2F80E42D2F81002B2F81212C2F8ED
:10A04800CC31D2F81432C0F38A10C1F34A01C3F3F9
:10A05800CA13CCF3CA0CC7F38A37C6F3CA366D09DC
:10A06800C4F30A04C2F8E401C2F8E811C2F8C0C196
:10A07800C2F8C471C2F8D061C2F8D851C2F8DC4144
:10A08800C2F8F03192F8183292F81702B2F81612A4
:10A09800DB0043EA5013C1F38A01C2F8F831C2F871
:10A0A800F411012081E7D3237AE700BFD8240020E8
:10A0B800944B5B68C3F3080370B443BBEFF311839D
:10A0C8002BBB914A914D1368AC6800BF11688B4255
:10A0D800F9D18F4A15684FF47A7101FB05F2141B08
:10A0E8008C4AB4FBF5F401FB0343D2F8401201F2A9
:10A0F8004C41994233D201240021C2F8403282F8FF
:10A10800000282F8444282F8FC1170BC7047EFF3F9
:10A118001181102383F312887C4C7F4AA568236839
:10A12800DE0344BF01231360774B48BFA5681E6850
:10A138001368C9B281F31188754A14684FF47A71AB
:10A1480001FB04F23344521BB2FBF4F201FB03237C
:10A15800704AD2F8401201F24C419942CBD392F89E
:10A1680044120029C7D002298ABF92F80142052467
:10A1780002348C42C9DD4B1CDBB29C421144D4BF73
:10A188000125002582F8443281F8000282F8FC514A
:10A19800BBDC92F802520023162D82F84432B4D068
:10A1A8006B00290648BF83F0D503DBB213F0800F9C
:10A1B8004FEA430318BF83F0D503DBB213F0800FD7
:10A1C8004FEA430318BF83F0D503DBB213F0800FC7
:10A1D8004FEA430318BF83F0D503DBB213F0800FB7
:10A1E8004FEA430318BF83F0D503DBB213F0800FA7
:10A1F8004FEA430318BF83F0D503DBB213F0800F97
:10A208004FEA430318BF83F0D503DBB292F801028B
:10A2180013F0800F4FEA430318BF83F0D5030228D9
:10A22800DBB247D93D490844023111F8016F734048
:10A2380013F0800F4FEA430318BF83F0D503DBB256
:10A2480013F0800F4FEA430318BF83F0D503DBB246
:10A2580013F0800F4FEA430318BF83F0D503DBB236
:10A2680013F0800F4FEA430318BF83F0D503DBB226
:10A2780013F0800F4FEA430318BF83F0D503DBB216
:10A2880013F0800F4FEA430318BF83F0D503DBB206
:10A2980013F0800F4FEA430318BF83F0D503DBB2F6
:10A2A80013F0800F4FEA430318BF83F0D5038142B0
:10A2B800DBB2BAD1224492F8FF219A427FF425AF4B
:10A2C8007A2D08D07C2D06D0282D7FF41EAF144B94
:10A2D80001221A7019E7134A136E572B3FF715AF6F
:10A2E800114912480D684C680821995413440121FA
:10A2F800C3F80150C3F80540136E017009331366A3
:10A3080003E700BF00ED00E0F035002010E000E0BA
:10A3180014380020D824002010380020D826002027
:10A32800A8680020B8680020DD260020A968002061
:10A3380010B5064CD4F8683204F512709847022814
:10A3480006BF012084F86C02002010BDD82400202C
:10A3580038B503788B4213D90A4C94F86C320D4601
:10A368004BB1D4F8943204F5127104F51C70984777
:10A37800002384F86C3204EB4504B4F8700238BD4D
:10A38800002038BDD824002070B5404D404C2B78B3
:10A3980006461BB1D4F89832834232D93D4B1B682C
:10A3A800DA070FD594F89D3294F89E229A422DD15F
:10A3B80094F8BC0228B9D4F8D402B0428CBF00206B
:10A3C800012070BD13F400532ED1D4F8C8223248AE
:10A3D80084F8BC329047C307EAD5D4F8A0322F4A94
:10A3E80000F0020000281E4413BF012100210123B0
:10A3F8000023012051702B70C4F8986284F8BC02C5
:10A4080070BD00232B7084F89C32C7E7D4F8A022D3
:10A41800224984F89E32324400200123C4F898224D
:10A42800087084F89C32C3E7B4F8A4320BBBB4F8C4
:10A43800A632F3B9B4F8A832DBB9B4F8AA32C3B972
:10A44800B4F8AC32ABB9B4F8AE3293B9B4F8B032B0
:10A458007BB9B4F8B23263B9B4F8B4324BB9B4F8D2
:10A46800B63233B9B4F8B8321BB9B4F8BA32002BE3
:10A478009ED0D4F8A0320949334400200122C4F800
:10A488009832087084F89C2292E700BF195B00207C
:10A49800D8240020183D0020982700202000002004
:10A4A8000020704700207047024B03EB4101B1F8D0
:10A4B800D8027047D8240020044B93F8FC0218B146
:10A4C800002283F8FC220120704700BFD824002016
:10A4D800024B03EB8101B1F800037047D824002038
:10A4E80003788B4283BF034B03EB4101B1F8380378
:10A4F80000207047D824002038B5394C0546F7F7B6
:10A50800B5FDD4F88C33C4F88C03C01AB0F57A7F43
:10A518001CDD0023282284F8903384F8923384F8D1
:10A52800933384F891233D2D42D03E2D0DD12D4AF1
:10A53800C4F89423012384F892330123157084F816
:10A54800903394F891239A4220D038BD94F8902300
:10A55800002AE8D0531CDBB2D4F8941384F8903363
:10A56800062B8D54EDD194F89233012B27D094F813
:10A578009333012B27D00023282284F8903384F8C2
:10A58800923384F8933384F8912338BD94F8923346
:10A59800012B04BF022384F8923394F89333012BE0
:10A5A80015D00022282384F8902384F8913338BDED
:10A5B8000D4AC4F89423012384F89333BDE78B78BC
:10A5C800282BD4D8F1E78B78092BD4D8EDE70223D0
:10A5D80084F89333F7F74AFDC4F89803E1E700BF1E
:10A5E800D82400203C2800203028002030B402461F
:10A5F800002305251E2400E00232032BD4BF0021CE
:10A60800012100F813100133042B04D0122B5470CD
:10A61800F2D130BC70475570EEE700BF024B0360C3
:10A6280043608360C3607047E803D007024B03EBC5
:10A638004101B1F8A4027047D8240020024B03EB73
:10A648004101B1F8A4027047D824002030B4264C48
:10A6580094F89233022B02D0002030BC704794F853
:10A668006653EDB1013D04F2653353FA85F504F5FF
:10A678005970002210F8013B534083EA0313DBB200
:10A68800120AD90042EA0322854281EA131382EAB8
:10A698000302EFD122B1002084F8920330BC704746
:10A6A800B4F864335BBA9BB243F60162934209D0B3
:10A6B80043F60362934205D0002384F892330120C5
:10A6C80030BC7047094AA2F12E0102F12005D07969
:10A6D8009379023203EB0023C3F3CC03AA4221F897
:10A6E800023FF4D1E8E700BFD82400203C2800202E
:10A6F8004E4B5B68C3F3080370B4B3B9EFF311832F
:10A708009BB94B4A4B4D1368AC6800BF11688B422C
:10A71800F9D1494A15684FF47A7101FB05F2141B07
:10A72800B4FBF5F401FB034320E0EFF311811023A0
:10A7380083F312883F4C414AA5682368DB0344BF72
:10A74800012313603A4B48BFA5681E681368C9B255
:10A7580081F31188384A14684FF47A71334401FB45
:10A7680004F2521BB2FBF4F201FB0323344AD2F881
:10A778009C13591AB1F5FA7F14D90021C2F89C33F9
:10A7880082F8A01382F8A113C3B2042B26D0202B81
:10A7980024D092F8A41309B9552838D0814216D18B
:10A7A800002109E092F8A11399B992F8A013C2F810
:10A7B8009C33C3B20029E8D092F8A2035418013898
:10A7C800814284F8AC331DD0013182F8A01370BCEB
:10A7D8007047013982F8A11370BC70470021022428
:10A7E8004FF6FF7082F8A843A2F8A6035418581E23
:10A7F800814282F8A43382F8A23382F8A31384F842
:10A80800AC33E1D1012382F8CC3370BC704701240A
:10A818001F2582F8A403A2F8A61382F8AC3382F8A5
:10A82800A34382F8A84382F8A253CDE700ED00E0E5
:10A83800F035002010E000E0143800201038002027
:10A84800D824002070B540F2014444EA8004F7F7A8
:10A858000DFC0C4E054696F8F03306EB8303D3F84F
:10A86800D003E3070AD5F8F78FF9640805F1340532
:10A8780007D0F7F7FBFB8542FBD8ECE7F8F77EF942
:10A88800F3E770BDD82400200D49B1F8F13330B595
:10A8980008224AF2010580EA030414F0010F4FEA86
:10A8A800530318BF6B4002F1FF3218BF9BB212F07E
:10A8B800FF024FEA5000EED1A1F8F13330BD00BFDE
:10A8C800D8240020084623F0D5BC00BF0FB400B53B
:10A8D80083B004AB054953F8042B01930020FAF721
:10A8E800CBFC03B05DF804EB04B07047CDA80008BA
:10A8F8000EB470B583B007AC0646482054F8045B24
:10A9080023F0B8FC202023F0B5FC304623F09EFC51
:10A918003A2023F0AFFC2A46234609490194002037
:10A92800FAF7AAFC04460A2023F0A4FC054A136897
:10A9380003341B1B136003B0BDE8704003B07047BD
:10A94800CDA8000874690020F8B50F4BD3F8F4536C
:10A95800D3F8F843D3F8FC63A9B1831E00EB410791
:10A9680027441E4404441D4434F9022B36F9023F9F
:10A9780035F9020F134403EBD373A0EB630023F004
:10A9880035FDA742F0D1F8BDD82400202DE9F04FBD
:10A99800DFF80C913949D9F8F453394B2C4685B076
:10A9A80005F1300B05F1100244F8040B5E460292E3
:10A9B80009F5806A09F20C4809F58367FAEC016A1F
:10A9C800B8EC017AF7EC017AB1EC010A0193FDEEDB
:10A9D800E66ABDEEC77AFDEEE77AE4EC016A84ED3B
:10A9E800027AC4ED057A0091039125F071FF019B6D
:10A9F800029A26F8020B944253F8040BB08000998F
:10AA0800DCD1204905F12803F1EC017AFDEEE77A63
:10AA180017EE902A23F8022B5B45F5D11A4B1B4AF7
:10AA2800588811781A88AA879A88DB88E887A5F851
:10AA38004020A5F8423071B105F14403144A03EBF4
:10AA48004101F2EC017AFDEEE77A17EE900A23F85D
:10AA5800020B8B42F5D10F490F4A104BB9F84E043F
:10AA6800498852681B88A5F85E00A5F86410A5F807
:10AA78006620A5F8683005B0BDE8F08F0C3D0020D1
:10AA88004449002038470020084B00206C40002033
:10AA9800FC2800209437002080370020205B00200D
:10AAA800D82400202DE9F041814CE27AA37A9A4219
:10AAB8005BD0E27AE37AC2EBC20204EB8202C3EB18
:10AAC800C30304EB830392F827101E7B8B1E9E4260
:10AAD80026D0784BD4F854141B781B2B61D0002057
:10AAE800E37A754A0133A2FB0352520802EB420291
:10AAF8009B1ADBB2E37209B9BDE8F0816F4B1B68A2
:10AB0800591AB1F5FA7FF7D994F85834032B02D1C2
:10AB18006B4B00221A800023C4F85434BDE8F0813E
:10AB2800E37A04F10C07C3EBC30307EB830361B1BA
:10AB38001944002213F8015B2A44994292B2F9D1D0
:10AB4800D3B203EB1222FF2A39D05A4BD4F854144B
:10AB58001B781B2BC3D123895A4A01339BB204208B
:10AB68009080238153800020BAE7F7F77FFA94F8A2
:10AB7800803403B32378F3B1636EC31AB3F5FA7F55
:10AB880019DB636EC31AB3F5FA6FC4BF00232370D1
:10AB9800237803F0FF02002B48D11046D4F8541450
:10ABA800A9E72389474A01339BB203209080238178
:10ABB8005380002094E7D4F8541400209BE7E37AEC
:10ABC80001221C2101FB0323FA18FB5CDBB1012BDA
:10ABD80012D1082ED4F854144BD0364B1B781B2BAB
:10ABE8007FF47DAF2389374A01339BB206209080DA
:10ABF80023815380002073E72E4B1B781B2B2CD00E
:10AC0800D4F854146BE7192E60D02A4AD4F8541497
:10AC180012781B2A7FF463AF22892A4D013292B23F
:10AC28000626184622816A80AE8059E7214B1B7898
:10AC38001B2B03D1626E234B801AD88094F888347A
:10AC4800D4F8840403B918B1002219490DF0C4FAE4
:10AC58000020D4F8541420704DE72389194AD4F8F9
:10AC6800541401339BB20520908023815380002027
:10AC780036E794F8800400283FF432AF5378002573
:10AC8800102BC4F8845400F0F78040F2F280303B77
:10AC9800012B3FF624AF52F8010F0B4BC4F88C047C
:10ACA8009088927998809A712846C4F8843417E776
:10ACB800D8240020104B0020ABAAAAAAF035002007
:10ACC800205B0020084B00206429002092F80280B5
:10ACD8005778C36892F803E011799579D67992F894
:10ACE80008C008F0070047EA00200EF03F0E977AE8
:10ACF800188090784FEA4E1E4EEAD00E907BA3F84B
:10AD080002E092F803E0890041EA9E1192F805E01A
:10AD18000EF0010E41EA8E21998005F00F05517958
:10AD280092F807E0ED0145EA5101557AD9804FEADA
:10AD38004C0C4CEADE1C05F0030592F806E0D17ACB
:10AD480006F07F064CEA452C3601557BA3F80AC06D
:10AD580046EA1E161E8105F00706957A92F809C084
:10AD6800C90041EA5511157B07F01F0745EA06257A
:10AD780000F03F00567BD9814001BF0140EAD6016F
:10AD880047EA9C079F811D825982D17B92F80EC0A9
:10AD9800D67C92F812E0577C957C507D890041EA78
:10ADA8009C1192F810C076000CF0010C46EADE16F1
:10ADB80007F00F0792F810E041EA8C21FF0192F8A2
:10ADC80014C0998247EA5E07917DDF8205F07F050E
:10ADD800577C0CF0030C46EA4C262D0145EA171562
:10ADE8005E83177D567D1D8300F01F008001C9001A
:10ADF80041EA561140EA9700D9839883D07D94F8A8
:10AE0800585410F0010F40F2147114BF0E46AD26CD
:10AE180010F0020F08BFAD2110F0080F0CBF012081
:10AE28000320032D1E8459841ED1137E94F85914CF
:10AE3800144ED4F85C24642B04EB4105A8BF6423AA
:10AE48009B02A6FB0363B5F8606401315B0901F05E
:10AE58000F01921B1A4484F859140B49A5F8603461
:10AE68001309C4F85C240B80084B1968C4F85414FF
:10AE780036E6002B7FF433AE012384F888340020B3
:10AE88002EE600BF1F85EB51205B0020F035002027
:10AE9800F0B5174E002383B004460821D6F8940471
:10AEA800737002ADF7F782FAD6F894048121F7F7A8
:10AEB8007DFA8923D6F8946425F8023DE71D14F835
:10AEC800010B324629460DF0B7FBBC42F7D1BDF85D
:10AED80006301A0A52FA83F3C3F1FF039BB23246D3
:10AEE800D8B20021ADF806300DF0A6FB03B0F0BDD6
:10AEF800D824002038B50D4C05460146D4F89804EE
:10AF0800F7F754FAB4F89C04082380EA052041F2C4
:10AF1800210210F4004F4FEA400018BF5040013B97
:10AF280080B2F6D1A4F89C0438BD00BFD824002014
:10AF38002DE9F84388460178A9B10C4E04468146AC
:10AF4800354606F10807284625F0FFFA38B1B84219
:10AF5800A0EB06003CBFA9EB040308F8003019F881
:10AF6800011F0029EFD1BDE8F88300BFC010030816
:10AF78002DE9F8432C228146002125F0CFFA0B2336
:10AF88001D4D1E4ADFF87C8089F80B3019240120FA
:10AF9800292140F26C7389F8124089F814000224C0
:10AFA800132089F81610C9F818201549A9F81C307B
:10AFB80040F643020E2389F81E40C9F8221089F88A
:10AFC8002000A9F8262089F8283044462E4605F1A5
:10AFD80008074121304625F0B8FA38B1B842A0EB4D
:10AFE80005003CBFA4EB080309F8003014F8011F62
:10AFF8000029EFD1BDE8F883C0100308DC051A0466
:10B0080046057503B03F03082DE9F04FE24C94F86C
:10B01800CC338BB023B9002318460BB0BDE8F08FB2
:10B0280094F8A33394F8A2030022012B84F8CC23CC
:10B0380044D0861E00F0AB8104F2AA35054404F51D
:10B048006B714FF6FF7311F8012B9B1AA9429BB243
:10B05800F9D11A0A204490F8AB139142DBD1264467
:10B06800DBB296F8AC239A42D5D194F8A433202BBE
:10B0780040F0868194F8A8138B1C09938B1D0193CB
:10B0880001F10803029301F10A03039301F10C0390
:10B09800049301F10E03059301F11003069301F1E6
:10B0A8001603079301F1180301F1040A01F11208CC
:10B0B80001F11407089301F11A0BAFE094F8A813F3
:10B0C800B4F8A6E38B1C671854FA83F6099301F1C8
:10B0D800040A97F8AC3397F8ADC396F8AC5396F8D2
:10B0E800AD7354FA8AF673448A1D96F8ADE301925B
:10B0F8001D4496F8AC3354FA82F605EB0C2501F1A1
:10B10800080296F8ADC302922B4496F8AC5354FA51
:10B1180082F603EB072301F10A0254FA82F72B4463
:10B1280096F8AC53039203EB0E2301F10C0297F847
:10B13800ADE396F8AD6304921D4497F8AC3354FA26
:10B1480082F705EB0C2501F10E0254FA82FC1D442E
:10B1580097F8AC33059205EB062501F110029CF82F
:10B16800AC6397F8AD739CF8ADC306922B4454FAC0
:10B1780082F503EB0E2301F1120895F8ADE3334491
:10B1880095F8AC6354FA88F503EB072301F114072B
:10B1980095F8AD93334495F8AC6354FA87F501F10B
:10B1A800160203EB0C23334495F8ACC3079254FA08
:10B1B80082F603EB0E2301F1180295F8AD530892BD
:10B1C800634496F8ACE396F8ADC303EB092354FA4D
:10B1D80082F6734401F11A0B96F8ACE396F8AD6366
:10B1E80003EB052354FA8BF52044734495F8ACE33C
:10B1F80090F8AB9395F8AD5390F8AA0303EB0C23A2
:10B208009E440EEB062E0EEB052E00EB09291FFAC5
:10B218008EFE1FFA89F9F1457FF4FDAE9DF82430C2
:10B2280054FA83F29DF8043054FA83FC9DF80830F0
:10B238009CF8AD939CF8ACC354FA83F301939DF842
:10B248000C3054FA83F69DF8103054FA83F59DF8C3
:10B25800143054FA83F09DF8183054FA83F30293AB
:10B2680054FA88F303939DF81C3092F8AD8392F852
:10B27800AC2354FA83F3214405939DF8203054FA03
:10B288008AFE54FA87F791F8ADA391F8AC130497A6
:10B2980054FA83F39EF8AD7306939EF8ACE3019BD2
:10B2A80001EB0A2102EB08220EEB072E93F8AD837F
:10B2B80093F8AC73C4F8001396F8AD3301930CEB14
:10B2C8000921C4F80C1395F8ADC396F8AC6395F84A
:10B2D800AC53019BC4F8042306EB0326049B029A93
:10B2E800C4F808E393F8ADE393F8AC3392F8AD9360
:10B2F80092F8AC13039A019603EB0E23C4F8283393
:10B30800059B90F8ADA3019E90F8AC03C4F81463B4
:10B3180007EB082701EB092192F8AD8392F8AC23DB
:10B3280093F8AD63C4F8201354FA8BFB93F8AC136D
:10B33800069BC4F8107305EB0C2500EB0A2002EB02
:10B348000822C4F81853C4F81C0393F8AD539BF8AB
:10B35800AD03C4F8242393F8AC239BF8AC3301EB7A
:10B36800062103EB0023C4F82C13C4F8343301235B
:10B3780002EB05221846C4F830230BB0BDE8F08F65
:10B3880006480CF0B7FC002384F8A10344E6FF222A
:10B398004FF6FF735EE600BFD82400208428002003
:10B3A800F8B5F6F763FE274E054600F1FA0734466E
:10B3B80096F8F03306EB8303D3F8D003F7F750FC85
:10B3C80038BB94F8F03304EB8303D3F8D003F7F7D2
:10B3D80047FC28B3F6F74AFED4F8A434401B984239
:10B3E800C4F8A0042BD805F5FA7594F8F03304EBEB
:10B3F8008303D3F8D003F7F733FCB0B994F8F033EC
:10B4080004EB8303D3F8D003F7F72AFC90B10020AC
:10B4180005E0F6F72BFEB842CAD94FF0FF30F8BD69
:10B42800F6F724FEB842CCD9F7E7F6F71FFEA84294
:10B43800DBD9F2E7F6F71AFEA842DFD9EDE70120DB
:10B44800EDE700BFD824002038B500240546047075
:10B45800FFF7A6FF431C11D0012803D12B78A04089
:10B46800184328700134082CF2D1054A2B7892F839
:10B47800A8144B4082F8A834012038BD0020FCE70E
:10B48800D82400202DE9F843204C214D2668074692
:10B498000236A84695F8F03305EB8303D3F8D003BA
:10B4A800F7F7DEFB10BBF6F7E1FD00F12706F6F72C
:10B4B800DDFD8642FBD800252C464FF0010998F89F
:10B4C800F03308EB8303D3F8D003F7F7C9FB18B1BF
:10B4D80009FA05F31C43A4B2092D06F134060BD072
:10B4E800F6F7C4FD8642FBD80135E8E723689E429B
:10B4F800D0D80020BDE8F88340F201232340B3F5FB
:10B50800007FF6D164083C700120F3E7F035002095
:10B51800D824002037B502ADFF2305F8013D0446C5
:10B528002846FFF7AFFF00B91CB99DF8070003B024
:10B5380030BD013CF4E773B5204C002284F8F123B8
:10B5480084F8F22384F8A92484F8AA240144FF2269
:10B558008DF807200546CEB22846FFF793FFF8B1CD
:10B5680015F8010BFFF790F9EBB2B342F4D194F858
:10B57800AB34EBB11248FFF785FF88B11148FFF7EC
:10B5880081FF68B10DF10700FFF77CFF40B1B4F807
:10B59800F123B4F8A9349A4202D0C2238DF80730B7
:10B5A8009DF80700A0F130035842584102B070BD21
:10B5B8000DF10700FFF766FFF2E700BFD82400206F
:10B5C800812900208229002070B5194C94F8F033A5
:10B5D8000D4604EB8303013D0646EDB2D3F8D003D4
:10B5E80007F0BEFC0135002384F8F13384F8F23308
:10B5F80035443078FFF726F916F8010BFFF744F9C0
:10B60800AE42F6D194F8AB343BB194F8F103FFF7AE
:10B6180019F994F8F203FFF715F994F8F03304EBED
:10B628008304D4F8D003BDE8704007F039BD00BFEB
:10B63800D824002013B5FE23ADF8043000238DF87C
:10B64800063003788DF80730044613B901238DF8C6
:10B65800063004210DEB0100FFF7B6FF0220FFF7CB
:10B6680059FFFF280CD121786068FFF7ADFF28202B
:10B67800FFF750FFA0F130035842584102B010BD07
:10B688000020FBE737B5054608461446FFF7D2FF0A
:10B6980078B10123022101A88DF805308DF80450F6
:10B6A800FFF792FF2046FFF735FFA0F1300358421D
:10B6B800584103B030BD07B50E4B0268934317D00D
:10B6C800FF230421ADF8043043788DF806308378E1
:10B6D8008DF807300DEB0100FFF776FF0220FFF72A
:10B6E80019FFA0F130035842584103B05DF804FB3C
:10B6F8000120FAE700FFFF0037B5054608460C466B
:10B70800FFF7D9FF60B123788DF80450022101A812
:10B718008DF80530FFF758FF21786068FFF70BFFB9
:10B7280003B030BD10B5064CD4F89804F6F73AFECD
:10B738000028F9D0D4F89804BDE81040F6F72ABEDE
:10B74800D824002010B5FFF7EDFF0A4AB2F8AF344D
:10B7580083EA00239BB2082141F2210413F4004F2D
:10B768004FEA430318BF634001399BB2F6D1A2F8F0
:10B77800AF3410BDD824002038B5064D002455F844
:10B78800340001340FF064F90FF0E1F9232CF6D1FD
:10B7980038BD00BFD81003082DE9F04F82468FB09E
:10B7A80091460E4615460027337808937378099317
:10B7B800F3780A9396F904300B9396F9028096F978
:10B7C80005300C93B3790D93B8F1000F4AD0B9F155
:10B7D800000F4ED02B78089C6A7895F90210E8780B
:10B7E80095F904C095F905E095F806B09C423ED15C
:10B7F800099C94423BD1884539D10A9C844236D170
:10B808000B9C644533D10C9C744530D10D9C5C4530
:10B8180014BF00240124CDE90121CDE9030C0093D4
:10B82800CDE905EB3B46144A214650460FF066FA2F
:10B838000D9B06930C9B05930B9B04930A9B0E4A46
:10B84800CDE90283099B0193089B009321463B465F
:10B85800504601370FF068FA102F06F1070605F178
:10B868000705A1D10FB0BDE8F04F0FF070B9002463
:10B87800D1E74C46DCE700BFF63803082DE9F04F66
:10B88800DFF820B189B08046894616460D46144631
:10B898004FF0000A002E71D06A6863689A426BD133
:10B8A800AF68A368FB1A5F425F4194F90B300493B9
:10B8B80094F90A300393B4F908300293B4F90630C6
:10B8C8000193B4F9043000935A465346394640462A
:10B8D8000FF014FA95F90B30049395F90A30039395
:10B8E800B5F908300293B5F906300193B5F904307B
:10B8F80000935A465346394640460AF1010A0FF06A
:10B9080013FABAF1080F05F10C0504F10C04C1D1C2
:10B918000024DFF894A0254696B30027012303FAF4
:10B9280007FB325959F8043053403BEA030314BF6C
:10B938000123002312EA0B0F079306D000972B462A
:10B948005246079940460FF0D9F959F804301BEAD6
:10B95800030F06D000972B465246079940460FF032
:10B96800E3F901370E2FD9D10135082D04F10C0464
:10B97800D2D109B0BDE8F08F002796E73746A9E78E
:10B988003746012359F80420BB40134206D00097DC
:10B998002B465246012140460FF0C6F901370E2FBB
:10B9A800EFD1E1E7133903082B3903082DE9F04FEC
:10B9B800064685B0884614468946924600270025E3
:10B9C80009EB050393F8C0300393002C64D00AEB0D
:10B9D8000503039A93F8C030D01AD0F1000B4BEB53
:10B9E800000BCDE900532E4A3B46594630460FF02E
:10B9F80085F9039B2A4ACDE9005359463B46304610
:10BA080001350FF091F9062DDAD10137062F09F12A
:10BA180006090AF1060AD2D1DFF884B008F1E40A6F
:10BA280000251AF8019B002C38D063195A4693F860
:10BA3800E430A9EB03014F424F41CDE900533946A9
:10BA4800062330460FF05AF9CDE900590623144A67
:10BA58003946304601350FF067F90B2DE1D198F8DA
:10BA6800F0506CB194F8F0300193EA1A5442544102
:10BA7800002300930A4A0723214630460FF03EF977
:10BA88000023009301950723054A214630460FF00D
:10BA98004BF905B0BDE8F08FA346AAE72746D3E7E0
:10BAA800403903082DE9FF47DFF86CA0814690462E
:10BAB8000E4615460027B8F1000F2AD02B88328889
:10BAC8009A4224D174886A88A21A54425441EA7866
:10BAD8000292AA782146CDE9003248463B465246B2
:10BAE8000FF00CF9F3780293B378019336F8043B1E
:10BAF800009352463B462146484601370FF014F959
:10BB0800102F05F10405D6D104B0BDE8F087002454
:10BB1800DDE74446E6E700BF543903082DE9F3475B
:10BB2800DFF868A081460F46904602260024B8F147
:10BB3800000F28D038F8243037F8241038F80620B9
:10BB480099421ED1BD5BA91A4D424D41CDE9003243
:10BB580029462346524648460FF0D0F8BB5B01936E
:10BB680037F8243000935246234629464846013484
:10BB78000FF0DAF8042C06F10406D8D102B0BDE8BB
:10BB8800F0870025E2E74546E8E700BF6639030885
:10BB98002DE9F04F834687B092460C46164600279B
:10BBA8004FF019094FF46178BAF1000F4DD0307891
:10BBB80025787378B27896F803C096F804E071791E
:10BBC800854240D165789D423DD1A57895423AD1CC
:10BBD800E578654537D12579754534D165798D4244
:10BBE80014BF0025012519FB028219FB0383CDE947
:10BBF800010303920091CDE904CE3B46144A29463D
:10BC080058460FF07BF823790593E3780493A378DB
:10BC18000F4A19FB03830393637819FB0383029389
:10BC2800237801936379009329463B4658460137A8
:10BC38000FF07AF80F2F04F1060406F10606B3D1C7
:10BC480007B0BDE8F08F0025CDE75546DBE700BF1C
:10BC5800773903087FB5094B0493094B0393094BC4
:10BC68000293094B0193094B0093094A094B0A496E
:10BC78000A480EF0F1FF07B05DF804FBD639030857
:10BC8800DB390308E5390308EE390308FA390308F4
:10BC9800953903081A4B0020A0390308AB3903086B
:10BCA80038B50B4B03EBC0040D4694F8F82109484E
:10BCB80003EB8203D3F830110EF0ABFE94F8FE319B
:10BCC8002BB1691C0448BDE838400EF0A2BE38BD4F
:10BCD800C0100308BD3E0308975E03082DE9F04F26
:10BCE800324C87B00746324A2378608802EB8303D8
:10BCF800D3F83081F8F70CF8D0E901A304932D4B61
:10BD080093F8B13413B9CDF810A09A4607F0400360
:10BD1800DFF8ACB005930025A379002B08BF0123F9
:10BD28009D4206DB244B08349C42DCD107B0BDE8B9
:10BD3800F08FA388049A2B440135D65C1AF8033097
:10BD4800F21AD2F1000949EB020993B9009543466A
:10BD58005A46494638460EF0D1FFC6B9059B002B16
:10BD6800DAD1009543465A46494638460EF0DCFF7C
:10BD7800D2E703F00F021B0940330292CDE90053CA
:10BD88000E4A4346494638460EF0B8FFE5E706F046
:10BD98000F03360940360293CDE900564346074A59
:10BDA800494638460EF0C0FFB6E700BFB812030890
:10BDB800C0100308D824002050130308143A0308BD
:10BDC800003A03082DE9F04F91B00025DFF88CA167
:10BDD800DFF88C91DFF89CB10795A84608A9E8B26E
:10BDE80012F0ECF89DF82830002B64D0012D0C9C43
:10BDF80040F09180002C00F0858007EE904ADFED3E
:10BE0800546AF8EEE77A86EEA77AFDEEC77A17EE5F
:10BE1800906A99F8B244089B012C75D996FBF4F402
:10BE28001A4601214B480EF0F4FD0D9A002A00F045
:10BE3800868041F2883002FB04004FF47A73B0FB2D
:10BE4800F3F00F9B002B7CD041F2883103FB0411E7
:10BE58004FF47A7CB1FBFCF1052D03D0079F0F440A
:10BE6800804407979AF803C0BCF1000F6BD04FF4D9
:10BE78007A7C0E9FB7FBFCFCCDF810C04FF00A0C83
:10BE880091FBFCFE0CFB1E11CDE902E190FBFCF1DD
:10BE98000CFB1100CDE9001021462F480EF0DCFE06
:10BEA800012D08D199F8B234012B04D932460999E9
:10BEB80058460EF0D1FE0135122D8FD1274BDB7875
:10BEC800EBB12749D1F8B824D1F8B404D1F8BC149F
:10BED80052094FF47A73B0FBF3F322480EF0BCFE1C
:10BEE8000798079B0A2293FBF2F302FB130798FBC0
:10BEF800F2F1009702FB11821B480EF0ADFE11B063
:10BF0800BDE8F08F264684E7099A184801210EF00B
:10BF180080FD344689E75CB107EE904ADFED0C6A94
:10BF2800F8EEE77A86EEA77AFDEEC77A17EE904A22
:10BF3800089A084829460EF06CFD002675E7104659
:10BF48007FE7194688E7214609480EF085FEA7E7EE
:10BF5800002474492A3A03084C3A0308144B002079
:10BF6800D8240020803A0308A03A0308393A030885
:10BF78007C3A0308703A03082DE9F0475D4B5E48A8
:10BF8800196890B04FF47A73B1FBF3F10EF064FEC8
:10BF980005A8F8F779FD58B1584A05A90023B2F960
:10BFA800002008A8F9F746FA08A955480EF054FEEB
:10BFB800544B554E1B78554A5549127809885548AF
:10BFC800DFF8A0A106EB830306F52979D3F89032B0
:10BFD8000EF042FE482150480EF01BFD4F4BD3F89F
:10BFE8000080002406F5317659F82470A300CFB1FB
:10BFF8000125A54015EA080F12D02A0710D01AF813
:10C0080004209B59464853F8222039460EF001FD7A
:10C01800022D05D1434B197F11B143480EF0F9FCAD
:10C028000134E1E70EF093FD404A41494148424C52
:10C038000EF012FE414A424B4248D31A3946B4F830
:10C04800C0240EF009FE40490A6D002A42D007EECE
:10C05800902ADFED3E6AB8EEE77AC6EE877AFDEE03
:10C06800E77ACDED037AD1F8EC305BB107EE903A80
:10C07800DFED366AF8EEE77A86EEA77AFDEEC77A44
:10C0880017EE903AC96959B107EE901ADFED2F6A99
:10C09800F8EEE77A86EEA77AFDEEC77A17EE901AE1
:10C0A800B4F8C2042A4E2B4F6428CDE9003101466A
:10C0B800039B2948A8BF64210EF0CEFD27480EF047
:10C0C800C7FC274B1C68012534B90EF040FD10B0A1
:10C0D800BDE8F0870392C6E794FAA4F3B3FA83F3B2
:10C0E80005FA03F256F82310384624EA02040EF043
:10C0F80090FCE9E7F0350020CE3A03081C690020DF
:10C10800E83A030894590020C01003083647002075
:10C1180094370020F93A03081F3B03080849002018
:10C128002F3B030814490020373B03080020001068
:10C13800000800003B3B0308D82400200000040846
:10C1480000F003085F3B0308D4050020002474496D
:10C15800D8360308BC3E0308993B0308DF3B0308B5
:10C1680058490020240000202DE9F84F184EDFF828
:10C17800689000250746AA4606F535780D246C43D5
:10C1880033193946D3F8D4B2584624F01AFA88B18C
:10C198004444594648460EF03CFC002120460EF027
:10C1A800CBFC0EF0D4FC20460EF06AFD0EF0CFFC5E
:10C1B8000AF1010A0135B5F5807FDFD1BAF1000F28
:10C1C80004D10448BDE8F84F0EF026BFBDE8F88F4B
:10C1D800C0100308F53B0308655E030838B50C4D2D
:10C1E800044620460EF0ACFB30B10A4B0A48597899
:10C1F800BDE838400EF030BD204624F071F8022822
:10C2080004D8C0B211F066FD2C46EAE738BD00BF7D
:10C218002B5E0308144B0020023C0308022810B5CB
:10C228000C460CD811F056FD0548FFF7D7FF0EF065
:10C238008EFC21460820BDE810400EF08DBC10BDD4
:10C248002B5E030870B50B4E0B4D044620460EF0CE
:10C2580077FB30B1074B09481978BDE870400EF0FC
:10C26800FBBC204624F03CF8022802D830702C464B
:10C27800ECE770BD144B00202B5E0308063C030856
:10C28800022810B50C460CD8F4F762FF0548FFF7F2
:10C29800D9FF0EF05CFC21460420BDE810400EF0EA
:10C2A8005BBC10BD2B5E0308F0B585B005460EF0EB
:10C2B80047FB002863D033490022012005B0BDE8C0
:10C2C800F040FFF7DBBA2D2B03D0A3F13002092A87
:10C2D80050D8052C04DD05B0BDE8F0400EF0A2BE34
:10C2E800284623F0FDFF04AB621C03EB440424F84A
:10C2F8000C0C15F8013F303B092BFAD914462B7862
:10C30800002BE0D1062CE6D1BDF904309AB2072AF9
:10C31800E1D8BDF90600A0F2EE2292B240F2DC5458
:10C32800A242D8D8BDF90810A1F2EE2292B2A242D8
:10C33800D1D8BDF90A209042CDDC9142CBDBBDF9C2
:10C348000C5005F16404A4B2C82CC4D8BDF90E4041
:10C35800112CC0DC0C4E0C2707FB0363A3F8C804A0
:10C36800A3F8CA14A3F8CC2483F8CE5483F8CF4496
:10C3780005B0F0BD202BAED101352246BEE70446FC
:10C38800BDE700BF9C290020D82400202DE9F341F7
:10C3980005460EF0D5FA044620B10EF043FE02B071
:10C3A800BDE8F081284601AA2949DFF8A48023F0D6
:10C3B800D0FF27460546264675B9022CEDD1A7F5CC
:10C3C8007A73B3F57A7F1ED94FF4FA624FF47A7113
:10C3D80020480EF04EFCE2E74CB1012C0ED001AA29
:10C3E8004146002023F0B5FF01340546E4E728461E
:10C3F80009F02EFC431C0646F1D1D0E7284623F06D
:10C408006FFF0746EBE7B8B20FF04EFDFF2EBCEE0C
:10C41800C00A114B0BD1114AF8EE407A1278AA42A1
:10C4280012DC10EE101A0E480EF016FCB7E7F8EE04
:10C43800407A03EB860310EE102A31460948C3ED13
:10C44800007A0EF009FCAAE7E3EC017A0135E6E789
:10C458000B3F03088F3E0308FC2900206C40002096
:10C468001E3C0308113C03082DE9F04F014691B02A
:10C47800854D064685480EF0EFFB002385F84435C8
:10C48800834B062219783046402485F8454510F03C
:10C49800D5FF0A20F5F790FE95F84435DBB20C2B52
:10C4A80040F2ED809DF80C90B9F1FE0F2ED0B9F155
:10C4B800FF0F15BF0F241524002601269C4240F0CB
:10C4C800DE80611EC9B268460BF0ECFB10AB1C4461
:10C4D80014F8413C834240F0CE8006F1FF38B8F1B1
:10C4E800010F9DF80D4013D904F01F076509613746
:10C4F8004C4668480EF0ACFA022E71D0013D042D6E
:10C508006AD8DFE805F00A5D616965000226D5E7AB
:10C518009DF80E709DF80F50EBE75F480EF07CFD1C
:10C528005E48DFF8CC91DFF8CCB10EF091FA002527
:10C538004FF0030A1DF80510484601350EF069FA58
:10C548000C2D55D10EF003FB022E5BD06422B4FBF8
:10C55800F2F102FB11423B46D2B2C9B250480EF08A
:10C568007BFB5FFA88F8B8F1010F7BD84D4A4E4B38
:10C578009DF810104D484E4D00290CBF1146194624
:10C588000EF06AFB9DF811104A4B4B4800290CBF6E
:10C59800294619460EF060FB022E63D19DF8124021
:10C5A80046480EF055FA9CB3FF2C41D00A22B4FB42
:10C5B800F2F102FB1142D2B241480EF04DFB2AE0E3
:10C5C80040480EF029FDABE73F480EF025FDA7E7F0
:10C5D8003E480EF021FDA3E73D480EF01DFD9FE704
:10C5E80000230DF11F008DF83F300EF015FD97E781
:10C5F80095FBFAF303EB43039D429BD158460EF09B
:10C6080027FA97E73A46214632480EF025FBA8E775
:10C6180028460EF001FD9DF813402F480EF018FA39
:10C6280054B1FF2C21D021462C480EF015FB06E012
:10C638002B480EF0F1FCEEE71D480EF0EDFC1C4D0A
:10C648001C4E274F00240DEB04031A7D8AB1FF2AE4
:10C6580014BF32463A462146224801340EF0FCFA0D
:10C66800042CF0D111B0BDE8F08F1D480EF0D4FCB9
:10C67800E5E72A46EFE71C480EF0CEFCF2E71B4838
:10C688000EF0CAFCEEE700BFD8240020503C030897
:10C698006C400020613C03086C3C03089A3C03088A
:10C6A800B13C0308363C03082D3C0308E83C03086A
:10C6B800403C03083D3C0308FF3C0308063D0308D3
:10C6C8001A3D0308733C03087B3C0308833C0308BA
:10C6D800923C0308CD3C0308223D0308985E0308FA
:10C6E800443C0308323D03083D3D03084D3D030823
:10C6F800AC3C0308E96403082DE9F34705460EF04E
:10C708001FF9044618B9324B9B78042B04D80EF055
:10C7180089FC02B0BDE8F08701AA2E49DFF8B8907D
:10C72800DFF8B8A0DFF8B880284623F012FE01270A
:10C73800264610B910F026FDEBE75EB909F088FA35
:10C74800431C0446E5D001AA22490020013623F003
:10C7580000FEEEE723F0C4FD2F28054630D807B3C6
:10C7680010F0E5FC062D08D10520F5F725FDFF2C76
:10C7780024D0E0B2FFF778FE08E00120F5F71CFDB1
:10C78800EAB298F80010E0B210F058FE2946504678
:10C798000EF062FA052D18DC1420F5F70DFD0027C0
:10C7A800D1E70628E3D0EBE7FFF75EFE98F8003004
:10C7B800F8B2834207F10107F6D8E7E70027F5E763
:10C7C8002F2148460EF048FABDE70027BBE700BF17
:10C7D800704100200B3F0308673D0308563D0308DE
:10C7E8006C40002038B50C4C05460C480EF030F96A
:10C7F800D4F84805F7F732FAD4F84C0512F0CAFA1B
:10C808000FF0C6FB064B074A25B1074907480860E1
:10C81800DA6038BDDA60FCE7D8240020873D0308D9
:10C8280000ED00E00400FA05FC9F0020EFBEADDE3D
:10C8380038B50A4DD5F84805F7F710FA084B002423
:10C848001C7085F85045C5F850460FF0E1FC2046AD
:10C85800FFF7C8FFC5F8484538BD00BFD8240020F9
:10C868007163002008B5F7F735FF0020BDE80840E0
:10C87800B8E70120B6E770B5064622F037FD124C3E
:10C88800054690B111220021204623F047FE2A4692
:10C898000E49304623F06EFE38B1102D2A46314637
:10C8A80028BF1022204623F077FE2378064A002B63
:10C8B80008BF0121054B1CBF002113460120044A73
:10C8C800BDE870400EF030BA7D690020E9640308C5
:10C8D800933D03082DE9F04188B080460EF030F80A
:10C8E800074608B33E4CDFF80481002519274FF4AA
:10C8F8006176237917FB03630493E37817FB0363DB
:10C908000393A37802936378019314F8053B00938B
:10C9180042462B460021012001350EF005FA0A2D6A
:10C92800E7D108B0BDE8F081404623F0D9FC0928DA
:10C9380005464FDC8400261808F101008DF81F70A9
:10C948000EF006F8074660B123F0CAFC0D2808D897
:10C95800244B334483F854069DF81F3001338DF877
:10C968001F3038460DF0F4FF074670B123F0B8FCCD
:10C97800431E042B09D81B4B6219134483F8550630
:10C988009DF81F3001338DF81F3038460DF0E0FF59
:10C99800074670B123F0A4FC431E072B09D8114B9E
:10C9A8002C441C449DF81F3084F8560601338DF83A
:10C9B8001F300B4CF11C0DF11F02214438460DF0BD
:10C9C800D4FF9DF81F30052BABD0A2190023A3512B
:10C9D8001371A6E70922394603480EF04AF9A0E781
:10C9E8002C2B0020D8240020B13D03089B3D0308D0
:10C9F8002DE9F34107460DF0A3FF064638B10022A2
:10CA080039490120FFF7C4F802B0BDE8F081384683
:10CA180023F066FC0E2804465FDC06254543781C97
:10CA28008DF807600DF094FF304F064658B123F09B
:10CA380057FC032807D87B1983F88C069DF8073024
:10CA480001338DF8073030460DF082FF804668B11B
:10CA580023F046FC0D2809D8062303FB047383F84A
:10CA680087069DF8073001338DF807301E4E691C84
:10CA78000DF10702314440460DF077FF0DF068FFD5
:10CA8800804668B123F02CFC182809D8062303FB3C
:10CA9800047383F88A069DF8073001338DF8073050
:10CAA80040460DF055FF68B123F01AFC0D2809D84F
:10CAB800062303FB04749DF8073084F88B060133C2
:10CAC8008DF807309DF80730062B9DD0721900238A
:10CAD800735193800EF0A6FA96E70E223146044869
:10CAE8000EF0C7F890E700BF5F2B0020D824002085
:10CAF800B13D03087FB505460DF022FF044630B16D
:10CB0800002218490120FEF751FF04B070BD2846E5
:10CB18006A461549144E23F01CFC01AD78B1032C6C
:10CB280002D10EF07FFAF0E723F0DAFB6A4645F807
:10CB380024003146002023F00CFC0134EEE7032CDE
:10CB4800EFD1DDE90145039E29463246E0B220F0E7
:10CB580067FD0028E5D033462A46214603480EF0F3
:10CB68007BF8D2E79C5900200B3F030840390308A3
:10CB780070B506460DF0E4FE044630B100221049B7
:10CB88000120BDE87040FEF78DBF304623F0A8FBBA
:10CB98000F2805460BDC30460DF0DAFE0146284624
:10CBA80020F066FD50B9BDE870400EF03BBA214652
:10CBB8000F220448BDE870400EF05BB870BD00BF9E
:10CBC8001C5A0020B13D03082DE9F04FDFF86880BA
:10CBD8008FB007468A46164600240DF124095AF8F4
:10CBE80024300293494602A808F0E4FF16B356F829
:10CBF8002430029D0393EB1A5D420DF1100B5D4149
:10CC0800594603A808F0D6FFCDF800B0234642469F
:10CC1800294638460EF072F82346CDF80090424671
:10CC28002946384601340EF07FF8202CD7D10FB0B2
:10CC3800BDE8F08F3546EFE7B73D030870B5064607
:10CC48000DF07EFE044628B100220F490120BDE800
:10CC58007040B9E7304623F043FB1F2805460BDC3C
:10CC680030460DF075FE0146284620F0D3FD50B938
:10CC7800BDE870400EF0D6B921461F220348BDE832
:10CC880070400DF0F6BF70BD9C590020B13D0308FF
:10CC98002DE9F04F2DED088BDFF80C9193B080460D
:10CCA80092460D461446002695ED008AB5EE408A58
:10CCB800F1EE10FA70D0D5ED019A95ED029AD5ED06
:10CCC800038ABAF1000F3ED094ED000A94ED01BA40
:10CCD800D4ED02AA94ED03AAB4EE408AF1EE10FA5C
:10CCE8005FD1F4EE4B9AF1EE10FA5AD1B4EE6A9A8B
:10CCF800F1EE10FA55D1F4EE4A8AF1EE10FA0CBFB3
:10CD0800012700270FA8F7F7DDFDB0EE4B0A834691
:10CD18000CA8F7F7D7FDB0EE6A0A059009A8F7F74F
:10CD2800D1FDB0EE4A0A049006A8F7F7CBFD059BA3
:10CD3800049A03900292CDE900B34A463346394635
:10CD480040460DF0DBFFB0EE480A0FA8F7F7BAFD32
:10CD5800B0EE690A07460CA8F7F7B4FDB0EE490A29
:10CD6800834609A8F7F7AEFDB0EE680A049006A856
:10CD7800F7F7A8FD049B0390CDE901B3009733466C
:10CD88004A460021404601360DF0CEFF082E05F137
:10CD9800100504F1100487D113B0BDEC088BBDE871
:10CDA800F08F0027AEE700BFC13D03087F2810B50C
:10CDB800044607D964F07F00C0B2E40921F05AFAAA
:10CDC8007F2CF7D8E0B2BDE8104021F053BA00BF7D
:10CDD800F0B52B4C2B4DD4F8F076D4F8F4662A49EC
:10CDE8002A48D4F8E43694F8EC262D78097890F897
:10CDF8002000B74285B027DB84F8FC56C4F8F83623
:10CE080084F8FD0684F8FE1684F8FF2601AD532049
:10CE180021F030FAD4F8F806FFF7C8FF94F8FC06BA
:10CE2800FFF7C4FF94F8FD1694F8FE2694F8FF3631
:10CE380003932846CDE9011221F024FA0023C4F80F
:10CE4800F036012005B0F0BDD4F8F8668DF808502A
:10CE5800B3428DF80B2001938DF809008DF80A1064
:10CE680001AD04F5DF6204D095E8030082E8030011
:10CE7800CDE7696853689942F6D10020E2E700BF20
:10CE8800D824002095690020195B0020285B002029
:10CE98001E4A1F4B116800221F29C3F80027A3F858
:10CEA8000427A3F80627A3F80827C3F8F02623D0F9
:10CEB8003F291CD04FF4FA42B2FBF1F1A3F80A174C
:10CEC8001448B3F90A27018829B1914201DD1F2AC4
:10CED80017DC92FBF1F1A3F80C1781780E480031AA
:10CEE80018BF01211202C3F8F426017070474FF4ED
:10CEF8000072A3F80A27E3E74FF48062A3F80A2731
:10CF0800DEE70121A3F80C17E7E700BF083D002082
:10CF1800D82400207A62002078620020084B10B5DF
:10CF2800B3F90A47B3F90C172046F8F7ADFB054BE0
:10CF38001B88C0B200FB03F090FBF4F0C0B210BD38
:10CF4800D82400207A6200202DE9F04F784CB4F8FC
:10CF580004378BB00546002B40F0F880754B1B88D2
:10CF6800002B00F09E802846FDF710FDD4F8F463EE
:10CF78004920354621F07EF9D4F80007FFF716FF5F
:10CF880055F8040BFFF712FF284608F0DDFD06F1FF
:10CF9800100008F0D9FDD4F81037DA0300F19D80AD
:10CFA800D4F810379B0300F18F80D4F810375F0353
:10CFB80000F1BA80032106F1280021F009FA5E4B3E
:10CFC800B6F92E001B8AC01AFFF7F0FED4F8103706
:10CFD800DD0400F19A80980400F18D80190400F1B5
:10CFE8008580032106F1300021F0F2F9D4F81037DA
:10CFF800DA025FD49F0257D4B6F9443007EE903A6C
:10D008004E4BF8EEE77A93ED007A77EEC77AFCEEAE
:10D01800E77A17EE900AFFF7C9FE494B1B78012BF8
:10D028000ED906F1440707EB430706F1460535F923
:10D03800020BB6F94430C01A21F0D8F9AF42F6D144
:10D04800D4F810379D0525D4D4F8F4133D483E4A4A
:10D05800C4F8F8130B1A9B1003EBC30503EB450345
:10D06800C3EB432303EB8343C3F1010382FB035266
:10D07800A2EBE37202EB42029B1A6C2202FB03034F
:10D088000122C4F8FC13C4F8F43384F860280BB008
:10D09800BDE8F08FB6F95E00A0F2DC5021F0A6F9E9
:10D0A800D2E7FFF795FE5EE7042106F13C0021F088
:10D0B8008FF9A1E7032106F1360021F089F9D4F8A8
:10D0C80010379F0298D5EFE7306A21F08FF9D4F82E
:10D0D80010375F037FF56EAF26E0F06921F086F91F
:10D0E800D4F810379B037FF560AFEDE7B6F868001A
:10D0F800FFF75CFE75E7B6F86600FFF757FED4F851
:10D10800103719047FF56DAFF0E7B6F86430B4F85E
:10D118001407C01AC0F30D00FFF748FED4F8103703
:10D1280098047FF55BAFE6E7706A21F05FF941E7A5
:10D13800D82400207A62002070410020F02B0020C3
:10D148006C400020F42B002056555555D4F86468DF
:10D15800D4F86838B34207D0C84BC4F868681B785D
:10D16800093B012B40F27481D4F86C78D4F8E4665A
:10D17800B74207D0C14BC4F86C681B78093B012B38
:10D1880040F25981B4F80837002B80D1BC4B1B887A
:10D19800002B3FF47CAFFFF71BFE2846FDF7F6FB9C
:10D1A8005020D4F8F483D4F8F89321F063F8D4F835
:10D1B800F433D4F8FC23D4F8F81312681B68086811
:10D1C8001344A3EB400002AE21F010F909F1040268
:10D1D80008F10401304608F08FFA304608F0B4FC34
:10D1E80009F1100208F11001304608F085FA3046BE
:10D1F80021F048F810250127D4F8103707FA05F26E
:10D208001A4240F0C6800135132DF5D108F12802E5
:10D2180009F12800B24608F13007314632F9023BDD
:10D2280030F9025B9742A3EB050341F8043BF5D1C3
:10D2380006AA002552F8043DAD0003F10801EDB23D
:10D2480033B10F2903F1800300F29C8045F00105FA
:10D258009642EFD14FF0000B284621F00BF85F46BD
:10D268005A4605F00303022B00F08380032B71D08C
:10D27800012B64D00137042F4FEA9505F1D1002A1C
:10D2880040F03081D4F81037D80403F4005203F486
:10D29800004100F19780002A40F0FA8059B1B8F8AF
:10D2A8006830B9F868209B1A0293029BD81780EA65
:10D2B8004300FFF77BFD03213020FDF745FBD4F841
:10D2C8001037D90200F1FF809A0200F1F7806D4B08
:10D2D80044201978FDF738FBD4F810379B0506D59C
:10D2E800B8F95E00B9F95E30C01A21F07FF8D4F8B9
:10D2F800F4136548654A0B1A9B1003EBC30503EB4F
:10D308004503C3EB432303EB8343C3F1010382FBD0
:10D318000352A2EBE37202EB42029B1A6C2202FB5D
:10D328000303D4F8F823C4F8F4330123C4F8F8133A
:10D33800C4F8FC2384F860380BB0BDE8F08F56F8C9
:10D348002710002A40F0C6804FEA011B5FFA8BFBCA
:10D358001A468FE756F827000192002A60D1C0F3D9
:10D36800072020F087FF16F8270020F083FF019A96
:10D3780080E756F827000192BAB9C0B220F07AFFC8
:10D38800019A77E7FF2B94BF45F0020545F00305A6
:10D398005EE7AB0008EB03024B4452F8240C53F849
:10D3A800243CC01A21F022F82DE7C0F3031040EA0C
:10D3B8000B0020F05FFF56F82730019A1B015FFA37
:10D3C80083FB57E7B8F86430B9F864001B1A029376
:10D3D800002A47D0B8F86630B9F866209B1A03933C
:10D3E800022500295ED1AD007319002053F8042DE1
:10D3F8004000C0B20AB140F001009E42F6D120F0D0
:10D4080039FF2E4402E056453FF455AF5AF8043B25
:10D41800002BF8D0D81780EA4300FFF7C7FCF2E7E3
:10D42800C0F3033040EA0B0020F024FF56F8270031
:10D43800C0F30710BDE7452020F01CFF1E2020F098
:10D4480019FF3046FFF7B2FC3846FFF7AFFC99E604
:10D45800452020F00FFF002020F00CFF3046FFF79A
:10D46800A5FC81E600293FF421AFB8F86830B9F887
:10D4780068209B1A03930225B5E700BF7862002055
:10D488007A6200206C400020F42B00205655555538
:10D49800B8F86630B9F866209B1A0293012500296E
:10D4A8003FF403AFB8F86830B9F868100AAA02EB7D
:10D4B80085025B1A42F8203C013594E704213C20A0
:10D4C800FDF742FA03E703213620FDF73DFAD4F8C9
:10D4D8001037F9E601F00F0141EA0B0020F0CAFE0F
:10D4E8000022C7E6584620F0C5FECBE6194BB3F834
:10D4F8000427D3F8F006D3F8001710B40132B3F9B3
:10D508000A4792B201300131A242C3F8F006C3F8CB
:10D518000017A3F804270FDAB3F80827B3F90C1794
:10D528005DF8044B013292B28A42A3F80827A4BFDF
:10D538000022A3F808277047B3F806275DF8044BC4
:10D5480000210132A3F80627A3F80417A3F8081747
:10D55800704700BFD8240020F0B5A44C04F5E3635D
:10D568008FB093ED000A23F0B3F904F5076393ED48
:10D57800000A054623F0ACF90646402020F016FEC6
:10D58800002855D19A4AD4F8743857784C2B00F2B1
:10D59800D984DFE813F00204F403EA03D603CD03C9
:10D5A800C303B003A60329041F0415040B043A049B
:10D5B800330444049C0395038B03810377036A03B4
:10D5C8005C034E0340033203240316030803F702E7
:10D5D800E9029E02900282027402660258024A021E
:10D5E8003F02310225021A020F020402F901ED017D
:10D5F800E101D501CA01BF01B301A7019C01910155
:10D6080086017B0171016701200116010C010101EE
:10D61800F600E000D600CC00C200B800AE00A300BF
:10D6280099008F0085007B00710067005E00500044
:10D6380000200FB0F0BD6F4B6F491A686F48FDF7B7
:10D6480057F9D4F8743801330020C4F874380FB08F
:10D65800F0BD927868496A48FDF74AF9D4F87438F9
:10D668000133F1E7674B6449DA896748FDF740F908
:10D67800D4F874380133E7E7624B5F491A88634886
:10D68800FDF736F9D4F874380133DDE75D4B5A49B4
:10D698009A785F48FDF72CF9D4F874380133D3E74A
:10D6A800584B55491A795B48FDF722F9D4F8743874
:10D6B8000133C9E7584B50491A7A5848FDF718F909
:10D6C800D4F874380133BFE7534B4B495A8C54484C
:10D6D800FDF70EF9D4F874380133B5E74E4B4649D7
:10D6E80093F820204F48FDF703F9D4F87438013334
:10D6F800AAE7494B40499A7F4B48FDF7F9F8D4F817
:10D7080074380133A0E794F8A8283B494748FDF747
:10D71800EFF8D4F87438013396E794F89B28364923
:10D728004348FDF7E5F8D4F8743801338CE7414BEA
:10D7380031495A794048FDF7DBF8D4F87438013399
:10D7480082E794F88B282C493C48FDF7D1F8D4F8A7
:10D758007438013378E7B4F888389FED397A264968
:10D76800384807EE903AF8EEE77A67EE877AFDEEEA
:10D77800E77A17EE902AFDF7BBF8D4F8743801332E
:10D7880062E7314A3149138A31489289FDF7B0F886
:10D79800D4F87438013357E72B4A2C49D3892D48DC
:10D7A8005289FDF7A5F8D4F8743801334CE7264BB5
:10D7B80011495A792848FDF79BF8D4F87438013391
:10D7C80042E7214B0C491A792448FDF791F8D4F81F
:10D7D8007438013338E71C4B0749DA782048FDF7DD
:10D7E80087F8D4F8743801332EE700BFD824002016
:10D7F800144B0020BC670020985E0308704403089F
:10D80800644403087041002050440308404403085E
:10D818002C4403081844030848390020044403082A
:10D82800E8430308CC430308B8430308A0430308AC
:10D8380090430308546C0020804303087043030896
:10D848000000C842644303087C3A0020884003086B
:10D858005043030840430308304303081C430308AC
:10D868001043030894F88128A149A248FDF740F81D
:10D87800D4F874380133E7E694F880289C499E4828
:10D88800FDF736F8D4F874380133DDE69B4B984938
:10D898001B689B485A8DFDF72BF8D4F87438013370
:10D8A800D2E6964B92491B6896481A8DFDF720F8E8
:10D8B800D4F874380133C7E6904B8D491B689248F9
:10D8C8005A8FFDF715F8D4F874380133BCE68B4B42
:10D8D80087491B688D481A8FFDF70AF8D4F8743801
:10D8E8000133B1E6854B82491B68894893F8372094
:10D8F800FCF7FEFFD4F874380133A5E67F4B7C496A
:10D908001B68844893F83620FCF7F2FFD4F8743883
:10D91800013399E6794B76491B687F489A8EFCF764
:10D92800E7FFD4F8743801338EE6744B70491B68EE
:10D938007A485A8EFCF7DCFFD4F87438013383E652
:10D948006E4B6B491B68764893F82D20FCF7D0FF87
:10D95800D4F87438013377E6684B65491B68714819
:10D9680093F82C20FCF7C4FFD4F8743801336BE625
:10D97800624B5F491B686C4893F82720FCF7B8FF97
:10D98800D4F8743801335FE65C4B59491B68674823
:10D998009A8CFCF7ADFFD4F87438013354E6574B32
:10D9A80053491B6862485A8CFCF7A2FFD4F87438B4
:10D9B800013349E6514B4E491B685E48DA8BFCF748
:10D9C80097FFD4F8743801333EE64C4B48491B683E
:10D9D80059481A8CFCF78CFFD4F87438013333E6B5
:10D9E800464B43491B68554893F82620FCF780FFAF
:10D9F800D4F87438013327E6404B51491D68514823
:10DA08002B7FEA7E6D7F0095FCF772FFD4F874389F
:10DA1800013319E6394B36491B684B481A7EFCF727
:10DA280067FFD4F8743801330EE6344B44491D6857
:10DA38004648AB7D6A7DED7D0095FCF759FFD4F82B
:10DA48007438013300E62D4B3D491D684048EB7C96
:10DA5800AA7C2D7D0095FCF74BFFD4F87438013370
:10DA6800F2E5264B36491D683A482B7CEA7B6D7CEB
:10DA78000095FCF73DFFD4F874380133E4E51F4BFB
:10DA88002F491D6834486B7B2A7BAD7B0095FCF7DA
:10DA98002FFFD4F874380133D6E5184B28491D6890
:10DAA8002E48AB7A6A7AED7A0095FCF721FFD4F814
:10DAB80074380133C8E5114B21491D682848EB79B2
:10DAC800AA792D7A0095FCF713FFD4F8743801333E
:10DAD800BAE50A4B1A491D6822482B79EA786D790C
:10DAE8000095FCF705FFD4F874380133ACE500BFA6
:10DAF800985E0308004303080443030860490020B4
:10DB0800EC420308DC420308D0420308C042030881
:10DB1800A84203088C4203087842030860420308BD
:10DB28004C4203083C4203082C42030818420308ED
:10DB380008420308FC410308EC410308D8410308E4
:10DB48006C410308D0410308C8410308BC410308DD
:10DB5800B4410308AC410308A44103089C410308ED
:10DB68009441030888410308B34BB4491D68B4487D
:10DB78006B782A78AD780095FCF7BAFED4F874383B
:10DB8800013361E5AF4BAD49AF4807EB470703EBFE
:10DB98008707FD79BB797A790095FCF7A9FED4F857
:10DBA8007438013350E5A74BA849A94807EB470744
:10DBB80003EB87035A89FCF79BFED4F874380133CA
:10DBC80042E5A04BA149A34807EB470703EB8703AE
:10DBD8001A7AFCF78DFED4F87438013334E5994B82
:10DBE8009A499D4807EB470703EB87031A79FCF727
:10DBF8007FFED4F87438013326E5924B9349974851
:10DC080007EB470703EB8703DA78FCF771FED4F8D4
:10DC18007438013318E58B4B8C49914807EB47075B
:10DC280003EB87035A7AFCF763FED4F874380133A0
:10DC38000AE5844B85498B4807EB470703EB8703C5
:10DC48005A78FCF755FED4F874380133FCE47D4B60
:10DC58007E49854807EB470703EB87039A78FCF76B
:10DC680047FED4F874380133EEE4764B77497F48A1
:10DC780007EB470713F82720FCF73AFED4F8743867
:10DC88000133E1E494F8B22470497948FCF730FE96
:10DC9800D4F874380133D7E4764B6C499A787648CF
:10DCA800FCF726FED4F874380133CDE4734B67498A
:10DCB8001A687348FCF71CFED4F874380133C3E4BF
:10DCC800704B9B79012B00F030811123BCE4B4F830
:10DCD80014276D496D48FCF70BFED4F874380133EE
:10DCE800B2E46B4B59491A886A48FCF701FED4F82C
:10DCF80074380133A8E4FFF711F9B4F90C17054695
:10DD0800B4F90A07F7F7C0FC2A46C3B26249634868
:10DD1800FCF7EEFDD4F87438013395E4B4F90A271A
:10DD28004A495F48FCF7E4FDD4F8743801338BE4C2
:10DD38005C4A5D495D48FCF7DBFDD4F87438013373
:10DD480082E403A8F6F7A0FE594B03A9B3F9002013
:10DD580006A80023F7F76EFB06AA53495548FCF7B7
:10DD6800C7FDD4F8743801336EE4534B534A544911
:10DD78005448FCF7BDFDD4F87438013364E4524AC2
:10DD8800524B53495348CDE90032534B534AFCF7A1
:10DD9800AFFDD4F87438013356E4514A424951482A
:10DDA800FCF7A6FDD4F8743801334DE4B3B2AAB237
:10DDB8004D494E48FCF79CFDD4F87438013343E4D0
:10DDC8004FF07E524A494B48FCF792FDD4F874381C
:10DDD800013339E4484B1D495A8A4848FCF788FD05
:10DDE800D4F8743801332FE4434B18491A8A44484D
:10DDF800FCF77EFDD4F87438013325E4D4F81037E5
:10DE0800DB0400F1878010231EE43E4B1E499A8AEA
:10DE18003D48FCF76DFDD4F87438013314E4194813
:10DE28003A4983784278007800903948FCF760FDD9
:10DE3800D4F87438013307E4604900206C410308C2
:10DE4800804103084262002078410308985E030875
:10DE58005C41030850410308444103083C4103085E
:10DE680030410308244103081C41030814410308F6
:10DE7800004103087C3A0020F0400308083D0020D8
:10DE8800E4400308F84800204C5E0308CC4003082F
:10DE98007A620020544003084040030848400308C1
:10DEA800344003087D690020BD3E0308284003086C
:10DEB8001C69002014400308E5390308EE390308FB
:10DEC800FC3F03080440030895390308DB390308BD
:10DED800D83F0308E83F0308FA390308A0390308C4
:10DEE800BC3F0308C83F0308884003089040030864
:10DEF800744003087C400308704100206840030810
:10DF08005C400308144900209C400308B040030803
:10DF1800BC4003080D4B0E491A780E48FCF7E8FC84
:10DF2800D4F874380133FFF78FBBB4F97C38B4F9EF
:10DF38007E2809490948FCF7DBFCD4F8743801331A
:10DF4800FFF782BB0120FFF774BB00BF21610020EF
:10DF58004C5E0308A440030888400308D440030823
:10DF68002DE9F04F604D85B0D5F87848009390467C
:10DF780000290CBF04230623621C0F9F01936ED057
:10DF88000E9BA34247DDDFF874A157B1109BDA1B43
:10DF980004FB02F20123B95CD5F810278B40134229
:10DFA80031D0009BD5F874B8A3EB080304FB03F445
:10DFB80008EB0406BBF1000F3AD158F8040021F031
:10DFC80095F900F10509484620F0F0F8002836D107
:10DFD800DAF8000095F8AB18A0EB0900CAF80000C1
:10DFE800002936D1012385F8AB38BBF1000F2AD1BF
:10DFF80058F8040020F02AF996F904104B1C02D0B6
:10E008003A48FCF763FCD5F878480E9B01349C42EB
:10E01800C5F87848B9DB0E9BA3424ED0D5F87408F2
:10E02800019B834294BF0020012005B0BDE8F08F1A
:10E038004FF00309484620F0B9F80028C8D001205D
:10E0480005B0BDE8F08F5E4429483179FCF73EFC05
:10E05800D9E72C2020F00EF9D5F874B8C5E7D5F823
:10E0680074A89A4503D3002005B0BDE8F08F214B72
:10E07800039103EB8A030646D3F8D42F0292104685
:10E0880021F034F90B3020F091F8DDE90221044643
:10E098000028D4D1BAF1030F98BF31461648FCF7CF
:10E0A80015FC1649D5F878280B6885F8AB481B1A73
:10E0B800541C0B60C5F8784862E7012020F076F818
:10E0C8000028ABD10D4A13680A20013B136020F0E9
:10E0D800D1F8D5F874084FF0FF330130C5F874084B
:10E0E800C5F878389CE700BFD82400208C44030882
:10E0F800985E0308C01003087C4403087469002074
:10E108002DE9F04F8F4CA378032B18BF032387B05A
:10E118004FF0800018BFA37019F0D0F80746002808
:10E1280000F0A980802119F0BFF87E79864B97F915
:10E1380002C053F82620854D0092B2F5613F14BF06
:10E14800002702270023022185F8AC08CDE9011732
:10E158001A466046802118F05FFF0C3E7C4B032E68
:10E16800186040F28E80D5F8B0387A4A03EB430342
:10E17800A2FB03235B0900F0E380402BA8BF4023E8
:10E18800DBB2754A1370002875D0744B744993F844
:10E1980015E0744A744B0F68E67811689879734AE9
:10E1A80093F80590DFF8D4A192F8008095F8C82874
:10E1B8006F4BB4F800C0BAF80240DFF8C4B1A5F854
:10E1C8001447BEF1000FC7F3C03718BF0127003648
:10E1D80018BF012611F0020F08BF0026002110F019
:10E1E800FD0F14BF4FF0010A8A46B9EB0109A2F1ED
:10E1F800190E18BF4FF00109B8EB0108A3F5CC744C
:10E208005C48C5F8B41818BF4FF00108BEFA8EFE76
:10E21800012A4FEA5E1EA3F5967208BF4FF0010E61
:10E22800C5F8F4431CF1FF3CA3F1C004C3E9011194
:10E23800C3E90311DBF80030C5F8F823C5F8FC433F
:10E2480090F800B0049318BF4FF0010C0A460C4632
:10E2580001200596D3B2591E152918D8DFE801F018
:10E2680024242424242424242E1A1A42201A3E3238
:10E2780032324A15461A404B00221A7007B0BDE8E0
:10E28800F08F354B40221A707DE7059931B100FABD
:10E2980002F10C430133DBB2162B2FD80132D9E738
:10E2A80051460029F3D1F9E79B4534BF00210121EC
:10E2B8000029EFD000FA02F10C43EBE77146002980
:10E2C800E5D1EBE7049E02EB4201314411F82E1C24
:10E2D800003118BF01210029ECD1DBE739460029BC
:10E2E800D5D1DBE749460029D1D1D7E741460029F6
:10E2F800CDD1D3E761460029C9D1CFE71A20C5F8A7
:10E3080010470EF017F81C4CD5F86418D5F8E42619
:10E3180085F8CA08002302202070C5F80037A5F840
:10E328000437A5F80637A5F80837C5F8F03685F894
:10E338006038C5F86818C5F86C2807B0BDE8F08FD4
:10E3480001231EE77A62002078360308D8240020CB
:10E3580078690020D34D62107C690020483900207C
:10E36800183D002008490020F8480020104B0020E4
:10E378008C2D00206C40002078620020943700200B
:10E388006049002008B5084B9B78032B06D0FFF79F
:10E39800B7FE064B012283F8CB2808BD802007F082
:10E3A800DFFA0028F3D008BD7A620020D8240020C4
:10E3B8002DE9F04F2DED028B9F4B1B78DA1ED2B260
:10E3C800142A85B000F2FD8201209C4900FA02F26D
:10E3D8001140002908BF0023994A9A4982F8CC388D
:10E3E8000023C1E90033C1E9023397490C463D22B5
:10E3F80023208B6181F85520F3F7DEFE934BA0694B
:10E40800636102232374002800F0B4831C220023D4
:10E418008271C3710D21F4F737FA8B4B1C4698694A
:10E42800F4F7B2FB4FF480716069FAF7ADF8A369AD
:10E4380013B11A689B881385834B1C4658696B2156
:10E44800F9F788FC80216069F9F784FCA36913B1A6
:10E458001A689B88936106237D4CDFF804827D4D02
:10E46800DFF8009201937C4F4FF0960E4FF0100C9E
:10E478004FF47A767B68C3F30803002B40F0B8802A
:10E48800EFF31183002B40F0B3802168AA6800BF26
:10E4980023689942F9D1D8F8000006FB00F39A1ACC
:10E4A800B2FBF0F206FB01217B68C3F30803002BE3
:10E4B8007ED1EFF31183002B7AD12368A86800BFBF
:10E4C80022689342F9D1D8F800A006FB0AF2101A84
:10E4D800B0FBFAF006FB03035B1AB3F57A7FE3D3CC
:10E4E800BEF1010EC6D1584B9B6913B11A689B88BF
:10E4F8001385554B586940F2E93302E0002B00F0D0
:10E5080097800289013B12F0020F9BB2F6D0F523E7
:10E51800037340F2E93302E0002B00F0898002899E
:10E52800013B12F0010F9BB2F6D0037B464B5869B2
:10E53800838940F2E93301E0002B76D00289013B60
:10E5480012F0020F9BB2F7D0FF23037340F2E933B6
:10E5580001E0002B69D00289013B12F0010F9BB248
:10E56800F7D0037BDBB29B46374B986910B1036841
:10E5780082889A615B46682B00F0D082019B013B40
:10E5880013F0FF0301937FF46EAF2F49334C91F8DA
:10E598005320A37981F85C30032A4FF0000381F8F7
:10E5A800523061D0184605B0BDEC028BBDE8F08F43
:10E5B800EFF311808CF31288D5F808A02B68DB03E1
:10E5C80004D50123C9F80030D5F808A02368D9F884
:10E5D8000020C0B280F31188D8F80000134406FB6D
:10E5E80000F2A2EB0A02B2FBF0F206FB032373E788
:10E5F800EFF311828CF31288A8682B68D90303D52E
:10E608000123C9F80030A8682368D9F80010D2B2ED
:10E6180082F31188D8F80020194406FB02F31B1A6C
:10E62800B3FBF2F306FB01313EE7F4F78BFC9BE703
:10E63800F4F788FC7AE700BF104B00202100110096
:10E64800D8240020083D0020903A002000300140E6
:10E65800F035002010E000E000ED00E07C3A0020FA
:10E668001438002010380020DE49DF4E0A68DF48E1
:10E67800DF4DE37142F001020A60DE493160062194
:10E688000171E278DC4971600221F56186F8521067
:10E69800002A00F07782072A00F07482D2499FEDA1
:10E6A800D77A81F84F30012307EE903AF8EEE77AEF
:10E6B800CD4867EE877A013BFCEEE77A80F8503068
:10E6C800CF4B80F84E20C3ED007A0546F4F756FC90
:10E6D80023780BB185F8523006F0CEF8C94CCA4AF7
:10E6E800C74BA260A4F6D80620468032A261C74A6A
:10E6F8001D6840F81C2B4FF47A714FF4FA72C44B22
:10E70800B3FBF5F39BB2B3FBF1F3C6F8D038102393
:10E71800A6F8D428202186F8D638A6F8DC381422A2
:10E72800BC4BC6F8E438A6F8EC18A6F8E82800218F
:10E73800802221F0F3FE8022002104F19C0021F0C8
:10E74800EDFE002104F58E70802221F0E7FE9FED9A
:10E75800B25ADFEDB25ADFEDB23A9FEDB22ADFEDE1
:10E76800B22A9FEDB23A9FEDBE1ADFEDB11ADFED86
:10E77800BA6A04F5CE71002306E00133F6EE007A9A
:10E78800202BE1EC017A55D007EE903AB8EEE77A03
:10E7980027EE057A77EE257ABDEEE76A16EE102A9F
:10E7A8002032402AE9D8B4EEE57AF1EE10FA40F3C7
:10E7B80015819FEDA86A01E0F0EE477AF4EEC67A7B
:10E7C800F1EE10FA37EEE67AF6DCB4EEE37AF1EE23
:10E7D80010FA40F100819FEDA16A01E0B0EE677A7E
:10E7E800B4EEC67AF1EE10FA77EE267AF6D4F4EEA5
:10E7F800E57AF1EE10FA40F3E68071EEE77A27EE5B
:10E80800A76AB0EE624AA6EE024A0133202BF0EE68
:10E81800430AE4EE060AB7EE007A66EE674A77EE38
:10E82800677AB6EE007AE4EEA07A67EE877AE1ECD2
:10E83800017AA9D10C2303FB05F306EE103AB8EED2
:10E84800466ADFED7C7A9FED751A7B4BDFED783AEF
:10E858009FED734A9FED732ADFED732A9FED733A9C
:10E86800DFED766ABCEEC66AF0EE411AB8EE466A8B
:10E8780003F16C0226EE276A03F1D80EFDEEC67A84
:10E8880036EE011A17EE905AFDEEC17A203517EED2
:10E89800904A00212034F7EE004A0EEB0100C8260A
:10E8A800402D868000F2DE80B4EEE36AF1EE10FAC5
:10E8B80040F37381B0EE467A9FED675ADFED655AF3
:10E8C80001E0B0EE677AB4EEE57AF1EE10FA77EE91
:10E8D800457AF6DCF4EEC47AF1EE10FA40F15A818A
:10E8E8009FED5D5ADFED5D5A01E0F0EE477AF4EEF8
:10E8F800E57AF1EE10FA37EE857AF6D4B4EEE17ADD
:10E90800F1EE10FA40F3008133EEC77A67EE077A2A
:10E91800F0EE620AE7EE820A402CB0EE430AA0EE5F
:10E92800A70A27EE275ADFED465AA5EE007AF0EE41
:10E93800640AF0EE647AE7EE250AE7EE657A87EE78
:10E94800A00A40F29680B0EE667AF6EE005AB7EE6C
:10E95800005AC4EEA07A0831DFF8F4C0394F3A4EB5
:10E968003A48C2F800C018299760D660106103F1D0
:10E97800240302F1240203ED050A65EEA75A25EEE9
:10E98800275A67EE277A43ED095A43ED075A03EDF4
:10E99800085A43ED067A43ED036A43ED046A43EDF2
:10E9A800016A43ED026A42ED086A42ED036A42EDEC
:10E9B800046A42ED016A42ED026A7FF46EAF0120FB
:10E9C800F1E5002308E5F4EEC17AF1EE10FA48BF4C
:10E9D80073EEE77A13E7F0EE477A08E7B0EE677A66
:10E9E800F3E600BF08490020903A002020000020EC
:10E9F80090C1793D852F0008C93A000800007A4483
:10EA0800083D0020B02D0020D42003080000F84164
:10EA180040420F00AC2003083C8C4F3EDB0FC93F3F
:10EA2800DB0F49C092E741B99730083C15A82ABEC8
:10EA3800DB0F4940E5A6C539CC2F002000000000B7
:10EA4800F304353F00DFCDBEBA32BDBE0184483E77
:10EA580000DFCD3EE4CB1641DB0FC940E4CB16C145
:10EA6800DB0FC9BFB7EE000A402CF0EE400A3FF6B4
:10EA78006AAFB4EEE16AF1EE10FA40F39180B0EEBD
:10EA8800417A1FED0B5A5FED0D5A01E0B0EE677A3F
:10EA9800B4EEE57AF1EE10FA77EE457AF6DCF4EEAC
:10EAA800C47AF1EE10FA0FD5B0EE677A1FED165A58
:10EAB8005FED165A01E0B0EE677AB4EEE57AF1EE52
:10EAC80010FA77EE857AF6D4F4EEE17AF1EE10FAE0
:10EAD80046DD73EEE77A67EEA75AB0EE625AA5EE06
:10EAE800825AF0EE438AE5EE858A25EEA78AB8EECB
:10EAF800007AE8EE287AF6EE005A34EEE75A27EE66
:10EB0800877A65EE255A24E75FED2B7AB4EEE77A2B
:10EB1800F1EE10FA48BF34EE477AF7E6F4F72EF82C
:10EB2800214B1C468C215869F9F714F901230DF182
:10EB38000F0200216069F9F7F7FCA069F4F724F8DF
:10EB48009DF80F30142BFFF420AD182B03D9543B3C
:10EB5800062B3FF61AAD144A032382F8533014E506
:10EB68009FED127AF4EEC77AF1EE10FA48BF74EE10
:10EB7800677AB0E71420F3F7E3F8A06100283FF4C0
:10EB880049AC43E408499FED0A7A032381F84F30E2
:10EB9800A37889E5B0EE677AB0E6F0EE467A99E6B2
:10EBA800F0EE417A7BE700BF903A0020DB0FC9BF47
:10EBB8000000FA4270B502392DED048BD0E900232C
:10EBC800856806290CD8DFE801F04C52575D626A67
:10EBD800040059425342C0E900136D420A46856059
:10EBE8003149097AD1BB314E07EE903A06EE902AA8
:10EBF800B8EEE78A96ED030A96ED007AD6ED067A26
:10EC0800F8EEE68A28EE000A06EE905AA7EE280AE1
:10EC18000446B8EEE69AA7EE890A21F059FE96ED69
:10EC2800040A96ED017AD6ED077A206028EE000AEC
:10EC3800A8EE870AA9EE270A21F04AFE96ED050AF2
:10EC480096ED027AD6ED087A606028EE000AA8EE02
:10EC5800870AA9EE270A21F03BFEA060BDEC048BD1
:10EC680070BD5142C0E900311A460B46B8E752421E
:10EC78005B42C0E90023B3E75942C0E900121346DA
:10EC88000A46ADE752426D4202608560A8E7114628
:10EC98006D42C0E9012503601A460B46A0E75B42B6
:10ECA8006D42C0E901359BE720000020BC30002000
:10ECB800944B954AD96AB2F88838A2F8083C0029DA
:10ECC80000F00D8107EE903AB8EE676A07EE901AE9
:10ECD800F8EE677A9FED8D7A9FED8D0ADFED8D2A2C
:10ECE8009FED8D3A9FED8D1ADFED8D1A9FED8D2AE0
:10ECF8009FED8D5A26EE276AF0EE400A26EE076A47
:10ED08002DED028BFDEEC67A36EE000A17EE900A5C
:10ED1800FDEEC07A02F60C4317EE901A203020312F
:10ED280002F67842F7EE004A402800F2A580B4EED9
:10ED3800E26AF1EE10FA40F3DC80B0EE467ADFEDDD
:10ED48007B5ADFED7B6A01E0B0EE677AB4EEE67AD3
:10ED5800F1EE10FA77EE657AF6DCF4EEC37AF1EEAE
:10ED680010FA40F1BD80DFED715ADFED726A01E003
:10ED7800F0EE477AF4EEE67AF1EE10FA37EEA57A7D
:10ED8800F6D4B4EEE07AF1EE10FA00F3A280DFEDEB
:10ED98006A7AB4EEE77AF1EE10FA48BF33EE477AB2
:10EDA80067EE077AB0EE614AA7EE814A4029F0EE95
:10EDB800423AE7EE843A67EE275ADFED606AA5EE3D
:10EDC800A37AB0EE644AF0EE647AA7EE264AE7EE3C
:10EDD800667AC7EE843A55D8B4EEE06AF1EE10FAD6
:10EDE80040F38A80B0EE407ADFED505ADFED506A8A
:10EDF80001E0B0EE677AB4EEE67AF1EE10FA77EE5B
:10EE0800657AF6DCF4EEC37AF1EE10FA77D5DFED29
:10EE1800475ADFED486A01E0F0EE477AF4EEE67A09
:10EE2800F1EE10FA37EEA57AF6D4B4EEE07AF1EE08
:10EE380010FA51DCDFED407AB4EEE77AF1EE10FA21
:10EE480048BF33EE477A67EE077AF0EE616AE7EE7D
:10EE5800816AF0EE428AE7EEA68A67EE275AB8EE94
:10EE6800008AA5EEA87AF6EE006A74EEC75A27EE75
:10EE7800087A65EEA66A0BE0F7EE003A4029B0EE94
:10EE8800634AA9D9B0EE457AF6EE006AF7EE005A61
:10EE9800C4EE847A243343ED053A67EEA66A67EE3A
:10EEA800A55A27EE877A43ED096A43ED076A43EDD1
:10EEB800085A03ED067A03ED035A03ED045A03EDED
:10EEC800015A03ED025A9A427FF42EAFBDEC028B31
:10EED800704732EEC77A63E732EEC77AB3E7704716
:10EEE800B0EE677AB4EEE07AF1EE10FA7FF74FAF42
:10EEF800EFE7F0EE467A30E7F0EE407A82E7B0EEE0
:10EF0800677A92E714490020D824002027D4D23603
:10EF1800DB0FC93FDB0F4940DB0F49C092E741B91E
:10EF28009730083C15A82ABE00000000DB0FC94036
:10EF3800E4CB1641E4CB16C1DB0FC9BFF304353F60
:10EF4800F8B5304C304E40220021204621F0E6FA38
:10EF58002E4B96F88C78B3F853509A6D6262103342
:10EF680093E80700A4F81F5096F88B5884F8287087
:10EF780004F10803072D83E8070004D92B46012B69
:10EF88004FF0000506D00123AB4013F0FD0F03D16D
:10EF9800002DF3D10020F8BDE37F032BF8D11C4AE4
:10EFA8001C4913681C4D216043F0020313601B4980
:10EFB8001448616002224FF480730727A277A38266
:10EFC8006F71F1F749FCB6F8083C4FF47A72E262C7
:10EFD8007BB1134D05F16C07B6F8083CE16A00EE09
:10EFE800103A2846B8EE400A2435F6F75DFBAF42E2
:10EFF800F2D196F88A3813B1A3770120F8BD012021
:10F00800F8BD00BF14490020D8240020903A002001
:10F01800084900206108000820000020793B00080A
:10F02800E4300020254B5B68C3F3080370B4B3B920
:10F03800EFF311839BB9224A224C1368A06800BFE2
:10F0480011688B42F9D120490D684FF47A7404FB9A
:10F0580005F1081AB0FBF5F004FB03031FE0EFF31A
:10F068001180102383F31288164A1849956813688B
:10F07800DB0342BF01230B609568114AC0B21668D2
:10F088000B6880F3118810490C684FF47A70334488
:10F0980000FB04F1491BB1FBF4F100FB03130C481E
:10F0A8000C49126882600124022280F8214081F80C
:10F0B8007C2CC1F8783C70BC704700BF00ED00E0C4
:10F0C800F035002010E000E014380020103800204F
:10F0D800285B0020D8240020274B5B68C3F3080373
:10F0E80030B4B3B9EFF311839BB9244A244C1368A5
:10F0F800A06800BF11688B42F9D1224A14684FF406
:10F108007A7101FB04F2101AB0FBF4F001FB03035F
:10F1180020E0EFF31181102383F3128818481A4A6C
:10F1280084680368DB0344BF01231360134B48BFA3
:10F1380084681D681368C9B281F31188114A106880
:10F148004FF47A712B4401FB00F2121BB2FBF0F270
:10F1580001FB03230D490E488A68022403F5B713FF
:10F1680003F5587302F2DC5280F87C4CC0F8783C06
:10F178008A6030BC704700BF00ED00E0F035002029
:10F1880010E000E01438002010380020285B002030
:10F19800D82400202DE9F04FA44C94F8B80189B088
:10F1A800002800F0D78094F8843C002284F8B82125
:10F1B800002B00F0D28094F8A8219D4E94F8855C2D
:10F1C80052B212F1630FB8BF96F90920002D40F032
:10F1D8000A81727294F8922C94F8AA11D4F8943C8B
:10F1E80094F8980C1B78114101F00F018B4210D94B
:10F1F8000B290ED80DB18D420BD094F8AAC194F802
:10F20800AB7104EB810100EA0C0C07EB0C27C1F889
:10F218006C7194F8AC11114101F00F018B4210D9B7
:10F228000B290ED80DB1A9420BD094F8ACC194F8B3
:10F23800AD7104EB810100EA0C0C07EB0C27C1F857
:10F248006C7194F8AE11114101F00F018B4210D985
:10F258000B290ED80DB1A9420BD094F8AEC194F881
:10F26800AF7104EB810100EA0C0C07EB0C27C1F825
:10F278006C7194F8B011114101F00F018B4210D953
:10F288000B290ED80DB18D420BD094F8B0C194F86B
:10F29800B17104EB810100EA0C0C07EB0C27C1F8F3
:10F2A8006C7194F8B211114101F00F018B4210D921
:10F2B8000B290ED80DB18D420BD094F8B2C194F839
:10F2C800B37104EB810100EA0C0C07EB0C27C1F8C1
:10F2D8006C7194F8B411114101F00F018B4210D9EF
:10F2E8000B290ED80DB18D420BD094F8B4C194F807
:10F2F800B57104EB810100EA0C0C07EB0C27C1F88F
:10F308006C7194F8B61141FA02F202F00F029342BE
:10F3180001D90B2A58D994F8B41194F8B55194F836
:10F32800B63194F8B7212D0445EA0165154345EA3D
:10F33800032505F0F023B3F1E02F7DD094F8843C49
:10F348003BB194F8693123B194F8AA311B0600F156
:10F358003281012009B0BDE8F08FF2F787FE344E04
:10F36800344BB27AA3FB00135B0CAAB194F8A82122
:10F3780094F8A911C9B2122918BF0129D2B200F014
:10F388003A8101F0EF01A1F1A201B1FA81F1490935
:10F39800002940F03081B17294F8A81194F8A9219D
:10F3A80002EB012292B2D4F88C1C94F8855C31B13E
:10F3B80099423FF40FAF591A012900F01E81A4F8B1
:10F3C800902CC4F88C3C05E70DB1AA42A3D094F860
:10F3D800B61194F8B73104EB8202084003EB002021
:10F3E800C2F86C0197E712F1310F80F2988012F1A0
:10F3F800380F80F2FC8012F13D0F80F22C8112F15F
:10F40800420F80F2368112F1450F80F2388112F1F5
:10F41800470F80F23C8112F1490F80F23C8112F1D2
:10F428004A0F40F03C81174608237BE0D82400208F
:10F438002000002083DE1B43A74FDFF8B892B9886D
:10F448003A7A97F800C097F801E097F802A08DF88B
:10F4580008C00023CDF80A30CDF80E308DF809E049
:10F4680002AB8DF80AA0ADF80C108DF8102093E8C7
:10F47800070005AB03C3D9F800101A8005F0070888
:10F48800002979D0DFF854B2C5F342525A44C5F383
:10F49800034392F83820944503F1010301D19E45B6
:10F4A8000DD0501E5FFA80FCBCF1040F8DF81420BB
:10F4B8008DF8153040F2D3800023ADF818300A6873
:10F4C80053687BB19847032800F0C180042800F0F6
:10F4D800BA80012800F0B3800023D9F80010002971
:10F4E8004AD00A689A4501D08DF81630536A00222E
:10F4F800C5F300158DF80720002B00F0C4800DF12E
:10F50800070098479DF80730AB4238D0D9F800106B
:10F51800A9B30B685B6993B3284698472FE06FF04F
:10F52800300701236D48591E00EB410100EB4300F1
:10F5380091F81DC0437F91F91C00A3EB0C01131A2D
:10F5480003FB01F3381A93FBF0F363445BB2642BBB
:10F55800D4F8880C6249A8BF642323EAE37300FB4C
:10F5680003F381FB0301DB17C3EB611304EB850194
:10F578009BB2C1F86C312CE600238DF80730029A53
:10F58800059B9A4250D09DF814309DF815109DF8AF
:10F5980016203B70BDF818307970BA70BB80FFF741
:10F5A8009BFDF4F7BBFDFFF73DFDF4F7CBFB012016
:10F5B80018F00AF8C2E6F2F759FDD4F8803C00F5D5
:10F5C8007A703061002B58D05A68121A002A04DB6E
:10F5D80053E05A68121A002A04DA03F108019B68FA
:10F5E800002BF6D13F4A736101200A60B2E66FF042
:10F5F8003707022396E792B2D5E6002D3FF4DFAE37
:10F60800B4F8900CD4F8881C374F101A143801FB42
:10F6180000F187FB0170C917A1EBE00104EB85003D
:10F6280089B2C0F86C11CAE6039A069B9A42AAD11D
:10F63800BDF81020BDF81C309A42A4D17EE6D8440B
:10F6480098F8403049E7D84498F8503045E7D8440E
:10F6580098F8483041E76FF03C07032362E7082B2E
:10F668003FF62AAF013B03EBC000204B33F81030C4
:10F6780023E76FF04107042354E71D49B2E76FF011
:10F68800440705234EE7002D3FF479AF41E76FF0BB
:10F698004607062346E76FF04807072342E712F1BB
:10F6A8004B0F12D012F14C0F0CD012F14D0F02D1AA
:10F6B80017460B2336E712F15C0F0ADB6FF05B0786
:10F6C8000C232FE717460A232CE76FF04A07092374
:10F6D80028E765233BE700BF4C460020B821030814
:10F6E8001F85EB512C000020676666661E2A0308FA
:10F6F80058310020484600202DE9F047B44DB54C5C
:10F70800B54B288BB54AB64FB64EC4F8A032DFF8D1
:10F7180034E3C4F8C472002384B00FFA80F984F883
:10F72800993CC4F8C86204F6984102F1240CDEF84A
:10F73800003022F8029F03F59673944541F8043F80
:10F74800F5D1DFF80483DFF804E3D8F800C0A64B4E
:10F758001CF4805F08BFB5F92490AEF8069003F159
:10F7680064010AE01FFA89F293F8019009F104098B
:10F778002EF81920053399421AD01A78002AF9D19F
:10F7880093F802A0DA789245F4D20AF1FF3909EB2E
:10F79800890909EB890909F561790132BAF1000F84
:10F7A800E0D102EB820202EB820202F56172DBE732
:10F7B8001CF0080F36D11CF4804F7AD11CF0007F62
:10F7C80042D11CF0010F0CF4005315D10BBB1CF4F3
:10F7D800004F23D16B7D13B1022384F8583495F878
:10F7E800282094F8C012131D8B42A8BF0B4684F83A
:10F7F800BD3D04B0BDE8F08744F62062A4F8C222FB
:10F80800002B67D00822794B84F8C022C4F8C43290
:10F81800DDE744F62063A4F8C232F3E7012384F855
:10F828005834DCE72B7A0C2B5BD8DFE813F0110196
:10F8380011018C019C00D9023002300206039D029E
:10F84800640011015A00DB0194F8BC3DBBB9684E55
:10F858001F22022306F1E00086F8E6200D2186F833
:10F86800E730F2F7BBFDD6F8E030B6F8E4209A614D
:10F8780004216048F8F788FE012384F8BC3D5E4AFD
:10F888005E4B5F495248C4F86822C4F89432F8F7CE
:10F89800A1FA5C4A5C4BC4F8C422002144F62062F9
:10F8A800D8F800C084F86C12A4F8C222C4F8C83290
:10F8B80087E7122344F6206284F8C032534BA4F839
:10F8C800C222C4F8C432524A524BC4F8C822C4F8FF
:10F8D800A03273E70C22504B84F8C022C4F8C4321B
:10F8E80075E70820F4F726FAD8F800C0C4F8C472FF
:10F8F800C4F8C8625FE749490A23020192FBF3F2A0
:10F908000023A2F5B06241F823200133102BFAD16D
:10F9180041F60B21424A84F8C0324020414BA4F8FA
:10F92800C212C4F8C422C4F8C83217F0C7FC0028B1
:10F93800D7D06B7A3C4A90F902000092003318BF86
:10F9480001230322CDE9012340210023374A17F080
:10F9580063FB374A031C18BF01231060002BC0D07B
:10F96800D8F800C027E7102342F6F821314A84F876
:10F97800C0324020304BA4F8C212C4F8C422C4F8E4
:10F98800C83217F09BFC81460028AAD01DF074FBF2
:10F99800697A99F902C0AB7A003118BF01214AB2DD
:10F9A800002800F0BF82002B40F053834FF4E1326F
:10F9B8004FF0030E0291CDE9002E60461F4A402108
:10F9C80017F02AFB1E4B1860031C18BF0123C5E75C
:10F9D80048390020D8240020A08601004663002072
:10F9E800A9A40008ADA40008BC31002045A6000861
:10F9F8001838002000380040797F00081D080008EA
:10FA08009827002059A3000839A30008B1A40008CA
:10FA1800C1A40008400D030035A600089426002064
:10FA2800B99E0008ED9E0008A0680600B9A000086D
:10FA3800A4680020C5960008D9960008A99800086F
:10FA480040680020F0350020183D00204863002061
:10FA5800B04BC4F8943C402017F030FC8146002895
:10FA68003FF43FAF4FF0000A84F884AC1DF004FB6C
:10FA78002A7A012A03460FD0C0F098820A2A1FD199
:10FA8800D8F8002012F480621CBF80F00102D2B2C4
:10FA980002F0010284F8842C0321072284F8921CC6
:10FAA80084F8982C01214FF4006284F89C11C4F862
:10FAB800882C0C2142F6F82284F8C012A4F8C2223D
:10FAC800697A9548954AC4F8C8220031C4F8C40236
:10FAD80018BF01214AB299F9020094F884CC002B8E
:10FAE80040F0FA81BCF1000F40F03A8295F80AC064
:10FAF800BCF1000F00F09182012342F008024FF49C
:10FB0800E131CDE9013200910023854A402117F007
:10FB180083FA844B18606B7D94F8C022013BDBB2FA
:10FB28009A4284F8853C9CBF002384F8853C0028D1
:10FB38003FF44AAF94F8843C002B3FF445AF0123CF
:10FB480084F8483D40E77849784BC4F8C43202014C
:10FB58000A2092FBF0F201F12400A2F5B062C4F889
:10FB6800CC1292B2C4F8D002002321F8132001333A
:10FB7800122BFAD142F6F8216D4A84F8C03240209F
:10FB8800A4F8C212C4F8C82217F098FB81460028CE
:10FB98003FF4A7AE1DF070FA6B7A95F80AC0654974
:10FBA80099F90220009100280CBF01210321002BA4
:10FBB80014BF06230723BCF1000F0CBF4FF0000C45
:10FBC8004FF0080C43EA0C0381460191029310465A
:10FBD800594B5A4A402117F01FFAB9F1000F3FF468
:10FBE800F3AEEFE60A220301554993FBF2F34F4ABD
:10FBF800C4F8C422A3F5B063C4F8CC129BB20022A7
:10FC080021F812300132122AFAD142F6F8214D4B6E
:10FC180084F8C0224020A4F8C212C4F8C83217F0F1
:10FC28004DFB00283FF45DAEAB7A697A90F902008B
:10FC3800454A002B0CBF00230823002908BF43F0C6
:10FC480001034FF0030C4FF4E131CDE901C30091FA
:10FC58000023402117F0E0F9C4F8940400283FF489
:10FC6800B3AE3A4B1A78002A40F08C81384A3949A9
:10FC7800116002221A70012394F8582484F8803401
:10FC8800002A7FF4A1AE032384F858349CE6062B9F
:10FC98004FF00C0240F00C8184F8BA3084F8C0228E
:10FCA800002384F8B020DFF8BC9084F88830212243
:10FCB80084F8B93084F8B83084F8AF2042F6F821D7
:10FCC800254A264BA4F8C2124020C4F8C422C4F81E
:10FCD800C83217F0F3FA824600283FF402AE1DF04E
:10FCE800CBF9697A9AF902C0AB7A003118BF0121C1
:10FCF8004AB2002800F03681002B40F0B981032277
:10FD080002910192CDF800906046154A402117F003
:10FD180083F957E698270020AD9A00089DF100085E
:10FD2800DD9A0008B468002024320020C19B000836
:10FD3800D59B0008A086010048320020B59D000828
:10FD480070320020ADAA0008F98E0008476800202C
:10FD5800F036002099AE0008AD900008C590000864
:10FD6800ED93000890D00300102041F27C53C7495E
:10FD7800C74A84F8C0024FF00009A4F8C2324020F4
:10FD88002823C4F8C412C4F8C82284F8909384F8CD
:10FD9800913317F093FA00283FF4A3ADAA7A6B7A4F
:10FDA800BC4990F9020000914A450CBF4A46082216
:10FDB8004B4518BF42F0010203214B46CDE9011221
:10FDC800B54A402117F028F90121C4F8940DF2F73B
:10FDD800D9FAD4F8943DB3EB090318BF0123BDE564
:10FDE800082342F6F821AD4A84F8C0324020AC4BD3
:10FDF800A4F8C212C4F8C422C4F8C83217F05EFAD4
:10FE0800814600283FF46DAD1DF036F96A7A99F9FC
:10FE180002100032034618BF0122002875D04FF0A7
:10FE2800030C4FF4E1330292CDE9003C084600236D
:10FE38009C4A402117F0F0F8C4E50E234FF0000962
:10FE480044F62061984A84F8C0324020974B84F8E1
:10FE5800A493A4F8C212C4F8C422C4F8C83217F094
:10FE68002DFA00283FF43DADB0F800C0697A90F94A
:10FE78000200AB7AB1EB09010CF4825C18BF0121D6
:10FE8800BCF5825F4AB200F0A58084F8A193002BEC
:10FE98005AD042F008024FF0010C4FF4E1310292BF
:10FEA800CDE9001C4B46824A402117F0B5F88BE596
:10FEB800002384F8C02284F8B02084F888301B22FC
:10FEC80084F8B93084F8B830052384F8AF2084F872
:10FED800BA304FF4E139F1E6BCF1000F5CD1AB7AEE
:10FEE800002B51D04FF0030E4FF4E131CDE9001E45
:10FEF80042F00802029263466E4A402117F08CF8DD
:10FF08006D4B18606D4B186005E64FF0010E4FF40D
:10FF1800E13C02920846CDE900CE624A402117F042
:10FF28007BF851E5002B6BD042F008024FF0010E30
:10FF38004FF4E13102920346CDE9001E6046604A63
:10FF4800402117F069F83FE54FF0010C4FF4E1321A
:10FF5800CDE901C100924021554A17F05DF833E51B
:10FF68000323CAE5002B69D042F00802012102925E
:10FF780003460191CDF800906046524A402117F09F
:10FF88004BF821E5002377E64FF0030C4FF4E132FC
:10FF9800CDE901C10092AFE74FF4E13342F0080226
:10FFA80003210093CDE901120023A5E702220321D2
:10FFB80084F8922C4FF4806284F8981CC4F8882C3A
:10FFC800072145F2F05284F89CA184F8C012A4F8E5
:10FFD800C22275E584F8A1933BBB42F008024FF0BA
:10FFE800030C4FF4E1310292CDE9001C304A402164
:08FFF80017F012F8344A354BF2
:020000040801F1
:10000000106000221A70E3E44FF0010E4FF4E13269
:100010000291CDE9002E60462B4A402117F000F8EE
:10002000D6E44FF0010C4FF4E132CDE901C100926A
:100030006FE542F008024FF0030C4FF4E1310292F9
:100040004B46D5E7012202910192CDF8009060461F
:100050001E4A402116F0E4FFBAE442F008020321F0
:100060004FF4E133CDE90031029260460023164A95
:10007000402116F0D5FFA9E442F0080203230292C2
:100080000193CDF8009060460023104A402116F0FD
:10009000C7FF9BE4E9A4000855A6000848E8010052
:1000A00001A50008ED95000805960008799600085E
:1000B000D9A4000811B00008F9A60008DD9A0008CC
:1000C000B468002040680020A9980008ED9300085B
:1000D000D436002024470020C1B1013910B450FAB1
:1000E00081F1441E002014F8013F434083EA0313CA
:1000F000DBB2000ADA0040EA0320A14282EA1313CD
:1001000080EA0300EFD15DF8044B70470846704762
:10011000F7B50023494C4A4E8DF803306023C4F8EC
:10012000A4343378152B07460ED0122B0CD0012B9C
:100130000CBF02258C25FBF737F9002807DA013DB3
:10014000F9D1002003B0F0BD44F62065F3E70A259D
:10015000FBF72AF90130F4D0013D15F0FF05F7D186
:10016000D4F8A024930803EB5203C4F8A434FBF79B
:100170001BF9431CE5D00028F9DC00230DF1030036
:1001800084F8A834FBF764F90028DAD09DF803302E
:100190001B2BD6D10DF10300FBF75AF90028D0D064
:1001A0009DF8032094F8BE3D9A42CAD10DF1050096
:1001B000FBF74EF99DF80530012BC2D801A8FBF7DB
:1001C00047F99DF80430002BBBD00DF10300FBF77D
:1001D0003FF90028B5D09DF803300E2BB1D10DF1B9
:1001E0000300FBF735F90028ABD09DF803203378E6
:1001F0009A42A6D10DF10300FBF72AF90028A0D0FE
:100200009DF80330002B9CD13D46BDF80430EA1B1D
:1002100092B2023B9A4209DB0DF10300FBF718F999
:1002200094F8A804B0FA80F040098BE72846FBF761
:100230000FF9002885D00135E7E700BFD82400205A
:100240006D40002070B5274C94F8BF3D43400646F2
:1002500084F8BF3D082594F8F03304EB8303D3F80A
:10026000D003F30716D5F2F793FC4020F1F74EFFC9
:1002700094F8F03304EB8303D3F8D003F2F782FC55
:100280004020F1F743FF013D15F0FF054FEA560608
:10029000E1D170BDF2F77CFC2020F1F737FF94F834
:1002A000F03304EB8303D3F8D003F2F76BFC202088
:1002B000F1F72CFF94F8F03304EB8303D3F8D00369
:1002C000F2F766FC2020F1F721FF94F8F03304EBFD
:1002D0008303D3F8D003F2F755FC2020F1F716FF83
:1002E000D1E700BFD824002010B50D4C94F8BF0D05
:1002F000FFF7A8FF94F8F03304EB8303D3F8D0039F
:10030000F2F746FC2020F1F701FF94F8F03304EBFC
:100310008304D4F8D003BDE8104002F0C5BE00BF8E
:10032000D824002010B5104C94F8F03304EB83036C
:10033000D3F8D00302F018FEFF20FFF783FFFF2061
:10034000FFF780FF7F20FFF77DFF00231B2084F84D
:10035000BF3DFFF777FF94F8BE0D0130C0B284F8BF
:10036000BE0DBDE810406DE7D82400200B4B10B542
:1003700001241C70FFF7D6FF0020FFF763FF204623
:10038000FFF760FF0E20FFF75DFF2046FFF75AFFE3
:10039000FFF7AAFF0248BDE81040B9E66D40002013
:1003A0006E400020F8B504780546002C3DD004F1DD
:1003B0000A060027FFF7B6FF300AFFF743FFF0B247
:1003C000FFF740FF0E20FFF73DFF1A4B1878FFF7AD
:1003D00039FF3846FFF736FF2046FFF733FF00208E
:1003E000FFF730FF0020FFF72DFF0020FFF72AFF67
:1003F0000020FFF727FF0020FFF724FF0020FFF772
:1004000021FF0020FFF71EFF6B681878FFF71AFF27
:100410006B68013C013314F0FF046B60F4D1FFF70B
:1004200063FF0548BDE8F84072E64FF48576012782
:10043000C0E700BF6D4000206E40002038B5054683
:100440000478FFF76FFF0020FFF7FCFE0420FFF7A2
:10045000F9FE0E20FFF7F6FE0A4BB4FA84F4187882
:100460006409FFF7EFFE2046FFF7ECFE2878FFF760
:10047000E9FEA020FFF7E6FEFFF736FF6868BDE85B
:10048000384045E66D40002038B5154B026893436F
:10049000044622D0134B06251D70FFF743FF0020B2
:1004A000FFF7D0FE0520FFF7CDFE0E20FFF7CAFEB6
:1004B0002846FFF7C7FE0020FFF7C4FE0020FFF725
:1004C000C1FE6078FFF7BEFEA078FFF7BBFEFFF726
:1004D0000BFF0548BDE838401AE6012038BD00BFD3
:1004E00000FFFF006D4000206E4000202DE9F04F1E
:1004F000AE4CDFF8C482C4F89804D1B016F06EFF99
:1005000008F11409002584F8AF5484F8B054FBF7BF
:100510001DF92F28F7D101210020F2F747FBADF894
:100520000850FBF713F90190FBF710F98DF815004F
:10053000FBF70CF98DF81600FBF708F900270646C3
:1005400010ADFBF703F9E8550137FBB29E42F8D135
:10055000FBF7ECF88DF80D00FBF7E8F88DF80C00D0
:10056000BDF80C70B4F8AF3401219F4214BF0327CB
:1005700000270020F2F71AFB002F40F08880019B33
:100580000695303B102B00F23682DFE813F068004E
:100590009300D70297001100AC003402D500A701E8
:1005A000DD0105024D0234022B027802A000AD02EB
:1005B000012602ADB2460021084684F89C1484F856
:1005C0009D14F2F7F3FAD4F89804F1F7B9FE2E204F
:1005D000FAF794FC0198FAF791FC9DF81500FAF7E8
:1005E0008DFC9DF81600FAF789FC50460AF1FF3A97
:1005F0005FFA8AFAFAF782FC0AF1010AAA44D4F8EF
:100600009804F1F7CFFE0028F9D015F8010BFAF79E
:1006100075FC5545F3D13846FAF770FC94F89D14F3
:10062000D4F89804F1F7C6FE94F89C14D4F8980412
:10063000F1F7C0FED4F89804F1F77CFE00210846DB
:10064000F2F7B4FA002E3FF45DAF94F8C13D002BF1
:1006500040F07F820CF09AFD51B0BDE8F08F94F825
:10066000AB34A3B194F8C03D013B032B18D8DFE8AD
:1006700003F002021302FD2302210AA8ADF828307C
:10068000FAF7A6FF0120FAF749FFC12808D1002692
:1006900002AD4FF0010A8EE7FFF768FE0028F6D1A1
:1006A000002684F8AB6484F8AC6402AD4FF0010A14
:1006B0000F2780E76B238DF80830E8E74FF432739B
:1006C000ADF80830002602AD4FF0020A73E72B7830
:1006D0005A1E032A00F2378284F8C03D002602AD7C
:1006E0004FF0010A67E72B7894F8C12D9A4205D89C
:1006F000002602AD4FF0010A08275CE784F8F033CA
:1007000094F8C03D042B0ED8012202FA03F313F033
:10071000160F08D0002302210AA8ADF8283084F86B
:10072000AB24FAF755FF002684F8AB6484F8AC6478
:1007300002AD4FF0010A3EE72B7894F8C12D84F802
:10074000AB749A4284F8AC74D2D984F8F03303269F
:1007500094F8C03D042B31D0FFF708FE70B301219F
:10076000134805F0A1FA48B30221124805F09CFA9B
:1007700020B3B4F8AB3449F2073223F008019142B8
:1007800007D049F20A32934203D049F20B42934216
:1007900014D1032384F8C03D94F8C03D84F8AE34EE
:1007A0000026044D4FF0040A05E700BFD8240020BE
:1007B000842900208329002010220308B8F8002093
:1007C00098F80230ADF81020BB4A8DF812300AAB11
:1007D000106851681D4603C508324A452B46F7D1BB
:1007E000D9F8000099F80420286015210AA82A7178
:1007F000FAF7EEFE082107A8FAF7A1FE00285FD05D
:100800009DF810209DF81C309A4259D19DF8112076
:100810009DF81D309A4253D19DF81E209DF812304C
:100820009A424DD19DF81F3084F8AD349DF82030A8
:1008300084F8AC349DF8213084F8AB34B4F8AB3490
:100840004FF2103223F02001914211D04FF21042AA
:1008500093420DD04FF29032934209D04FF650029E
:10086000934205D003F5BA520F3292B2012A03D84F
:10087000012384F8C03D8FE723F0080249F20731D5
:100880008A4207D049F20A32934203D049F20B421E
:10089000934203D1022384F8C03D7DE741F60672FE
:1008A000934209D043F20632934205D023F4807379
:1008B00043F20642934203D1042384F8C03D6BE720
:1008C000013E16F0FF067FF443AF84F8AB6484F872
:1008D000AC647A4D4FF0040A0F276CE694F8C03DE3
:1008E000032B40F08880764B12251D70FFF71AFD10
:1008F0000020FFF7A7FC0720FFF7A4FC0E20FFF75E
:10090000A1FC2846FFF79EFC1420FFF79BFC00206B
:10091000FFF798FCAC20FFF795FC8820FFF792FCCE
:100920001320FFF78FFC7620FFF78CFCFFF7DCFC31
:100930006448FFF7EDFB00287FF4A9AE002602AD66
:100940004FF0010A0F2736E694F8C02D012A01D096
:10095000042A50D12B788DF80830042A0CBF9B0054
:100960005B00DBB28DF8153005A800238DF816303A
:10097000FAF7A5FE0028E1D04FF4817302210AA8FE
:10098000ADF82830FAF724FE4FF42F70FAF7C6FDC1
:1009900030283FF47CAED1E72B788DF8143094F8F2
:1009A000C03D5A1E032A26D8DFE802F002020F02D9
:1009B000022B05A90CBF07200320FAF7A1FE00288F
:1009C000BCD09DF814A00026F5E505A8FFF75CFD56
:1009D0000028B3D014223A4B0DEB02001A70FFF737
:1009E0002DFDECE72B788DF8143094F8C03D022BE8
:1009F00007D0032B0AD0002602AD4FF0010A0227D0
:100A0000D9E505A90420FAF77BFED8E705A8FFF78A
:100A10003BFD002892D02A4B162205A81A70FFF73A
:100A20000DFD0028CDD189E794F8C03D8DF8146004
:100A3000013B032B3FF62BAEDFE803F0020211026D
:100A400005A8FAF73CFE00283FF478AFFA2205A982
:100A50000120FAF71BFE00287FF419AE6EE705A807
:100A6000FFF712FD00283FF469AF154B132205A8CC
:100A70001A70FFF797FC00287FF409AE5EE794F840
:100A8000C03D8DF81460022B05D0032B1CD0012B28
:100A90007FF454AFAFE705A8FAF711FE00283FF442
:100AA0004DAF40F2DC5205A90520FAF7EFFD002812
:100AB0007FF4EDAD42E700BF142203088329002034
:100AC0006D4000206E40002005A8FFF7DDFC0028E7
:100AD0003FF434AF294B152205A81A70FFF762FCCA
:100AE00000287FF4D4AD29E794F8C0BDBBF1040F12
:100AF00081D105A88DF81460FAF7E1FD00283FF4D4
:100B00001DAF05A8FAF79AFD00283FF417AF4FF480
:100B1000827302210AA8ADF82830FAF759FD142093
:100B2000FAF7FCFC30283FF4B2ADC0287FF406AFE2
:100B3000002602AD4FF0010A5F463CE50026104D4D
:100B40004FF0090A37E5002602AD4FF0010A0927E8
:100B500031E5013BDBB284F8C13D04EB8303D3F8FC
:100B6000D00310B10221F1F73DFC94F8C13D04EB34
:100B70008303D3F8D003F2F705F866E56D40002053
:100B8000D53D0308F8B5044609F0DEFE054630B150
:100B900000222C490120BDE8F840FAF7C3BF2A49DA
:100BA0002046F3F7EDFFA8B9284B4FF47A714FF4C4
:100BB000FA62A3F8C21DA3F8C42DA3F8C61DA3F8BA
:100BC000C82DA3F8CA1DA3F8CC2DA3F8CE1DA3F8F9
:100BD000D02DF8BD20461FF087FB0328064629D8F4
:100BE000204609F0B9FE054658B11FF07DFB0127EC
:100BF0000446284609F0B0FE30B9BDE8F8400AF0D6
:100C000015BA04460746F4E71FF06EFB002FF4D038
:100C1000A4F2EE2240F2DC539A42EED8A0F2EE2289
:100C20009A42EAD8094B03EB8603A3F8C24DA3F816
:100C3000C40DCEE7294603220548BDE8F8400AF076
:100C40001CB800BF9A320020DF3D0308D8240020E2
:100C5000E53D03082DE9F04F89B007461EF04AFB39
:100C6000044628B94120FBF73DF809B0BDE8F08FF4
:100C700002469949994E3846F3F75EFF054600282B
:100C800050D19748974CDFF89482DFF894920AF09D
:100C9000C7F904F59877A3792168A28806EB830346
:100CA00001F13841B2FA82F2890A4131D3F8303188
:100CB000C2F11F02404609F0B0FEE17911B1484689
:100CC00009F0ABFE083409F046FFA742E3D109F072
:100CD00042FF8548854C864FDFF84882DFF848920E
:100CE0000AF09EF9237E072195FBF1F1C1EBC102C9
:100CF00006EB8303AA1A013201313846D3F830A13A
:100D000009F08BFE627E514642B1484609F0A8FFC9
:100D100001350C2D04F11C04E4D1A6E7404609F08E
:100D20009FFFF5E7384607AA72491FF016FB06F544
:100D3000FC7782460025B94617F8353006EB830369
:100D40002246D3F8301150464FEAC508F3F7F4FEB7
:100D500030B10135132DEFD167480AF061F984E70E
:100D600007AA64491FF0F9FA464407461FF0BCFA87
:100D700096F8FE210446002A40F09980002800F3EE
:100D80009F80C844B8F80200F2F7C6FF97F800A0A9
:100D9000BAF1000F00F08880E3B20193019AB8F82D
:100DA0000430564913440293436803933846F3F7DB
:100DB000E7FE40B9DDE90223985451480AF030F9C2
:100DC00053E7012277E0AAF14106F6B2072E04D9D3
:100DD000AAF16106F6B2072E66D8781C1FF084FAD5
:100DE000C3B20F2B82465FD8741C40EA0414E4B2ED
:100DF0002046F0F7A9FF002856D0002C49D023093F
:100E000040330493DFF8249104F00F034FF00008FF
:100E1000059300272FE0B9F80200F2F77DFFB9F83B
:100E2000043042683B44D15CA14223D1454504D102
:100E300001998F421ED00021D154DDE904123148BE
:100E400009F0EBFD5FFA87FB5FFA88F35946184615
:100E50000093FAF729FF454509D12B4809F0DDFD3C
:100E600000985946FAF720FF284809F0D6FD28488F
:100E70000AF0D6F8013799F80630002B08BF012395
:100E80009F42C8DB08F10108B8F1130F09F1080906
:100E9000BFD15FFA8AF206F141011E4809F0E0FE77
:100EA000DDE902239C54E0E60AF0C0F8DDE6002804
:100EB00001DD944207DD0121174809F0DEFED4E68A
:100EC00001287FF47EAF07AA0A4900201FF045FAE7
:100ED000013C074655E700BFED3D0308C01003087D
:100EE000F23D030818380020003E0308CC00002023
:100EF000053E03080B3F03081E3E03080F3A030894
:100F0000263E03082C3E0308503E0308533E0308C8
:100F1000636303085D3E0308B13D0308F53D030824
:100F2000975E0308BC3E0308173E0308B812030887
:100F30002DE9F74F06461EF0DDF9074620B10128DE
:100F400023D133782A2B20D17B487C4EDFF80492C2
:100F50000AF066F8002406F535780D256543731907
:100F60004846D3F8D41209F058FD391C18BF0121A6
:100F700008EB0500013409F0E3FD09F0ECFDB4F5E0
:100F8000807FEAD103B0BDE8F08F3D2130461FF0ED
:100F9000E0FA002800F0C980034613F8012C202A4B
:100FA00003F1FF314FD09B1B013004460130227802
:100FB000202AFAD0DBB2DFF88491009300250D23BC
:100FC00003FB05FB09EB0B07D7F8D4A250461EF034
:100FD00091F95146024601903046F3F7ADFD824645
:100FE000002840F09780009B1A46019B934240F0F6
:100FF0009180534B9B4497F8D83203F03003102B69
:1010000023D0202B50D083BB20461FF06DF9B7F9B9
:10101000D93201B28B4228DCB7F9DB328B4224DBB8
:10102000584609F0EBFC454A46480D2303FB0525CD
:10103000D5F8D41209F0F1FC0021584603B0BDE800
:10104000F04F09F07DBD0B46A7E797F8D9123E4F48
:1010500007EBC107814697F878800646C24502D261
:10106000B9F1000F0AD0002EDDD1384809F0D8FFC1
:10107000584603B0BDE8F04F09F006BE7A6F21462E
:1010800052F82A00F3F77CFD00280CBF4FF001094D
:101090004FF0000905D10FFA8AF1584609F0AEFC6D
:1010A00001260AF1010AD9E7244B97F8D9820D27C6
:1010B000064607FB0537D045D5DD21460C460131F4
:1010C00020782028FAD02C2120461FF042FA8146B1
:1010D00018B908F1FF31514513D1584609F081FC88
:1010E00097F8D83203F00303022B06460CD0032BEB
:1010F0000AD020461FF0F8F806F80A0009F10104AA
:1011000001260AF1010AD6E720461FF0EDF826F87D
:101110001A00F3E70135B5F5807F7FF450AF0C4836
:1011200003B0BDE8F04F09F07BBF304603B0BDE827
:10113000F04FFBF71DB800BF693E0308C01003085D
:10114000941303087C3E0308B8210308873E030874
:10115000F53B0308655E030810B5044609F0F4FB8F
:1011600040B1F0F7C1F8F3F7B9FA0020BDE810403C
:10117000FBF73CBB062205492046F3F7DDFC18B916
:10118000BDE81040F0F7B0B810BD00BF473F0308FE
:101190002DE9F047214FDFF8A480DFF88490DFF8D5
:1011A000A0A0054628461EF0A5F8064660B91C4BCF
:1011B0001C4893F8C8281C4B03EB8203BDE8F0479A
:1011C000D3F8381109F04CBD024639462846F3F7EA
:1011D000B3FC78B91548164C164D09F03DFC54F88F
:1011E000041F19B1284609F018FCF8E7BDE8F047DC
:1011F00009F0B1BC002458F8241021B90E48BDE80C
:10120000F04709F00DBF32462846F3F795FC01344C
:101210000028F0D189F8C8485546C3E7ED3D0308DA
:10122000D8240020953E0308B82103089F3E0308F8
:10123000F0220308BC3E0308F53B0308F422030830
:101240002B5E03082DE9F74F80461EF053F84A4EF7
:101250000446D6F8D47DE8B94848494DDFF84481C2
:1012600009F0DBFB0C26204616F0A6F8384205D024
:1012700006FB04534046996809F0CFFB0134162C55
:10128000F1D117B93F4809F0E7FB03B0BDE8F04FD3
:1012900009F061BC02463C49DFF8E4904046F3F7B0
:1012A0004BFC054678B9394809F0D6FB2C46384D39
:1012B00009EB0403284699680C3409F0AEFBB4F539
:1012C000907FF5D1E1E798F800302D2B03BF08F1AE
:1012D000010804F1FF344FF0010A4FF0000A002525
:1012E0000C2303FB05924046D2F808B00193224636
:1012F0005946F3F721FC019BA0BBBAF1000F1CD0AB
:10130000162D0CD1234BC6F8D43D234809F0A4FB7D
:101310001F48594603B0BDE8F04F09F0A1BC172D96
:1013200004D1D6F8D83DC6F8D43DEEE7284616F0ED
:1013300043F83843C6F8D40DE7E7162D05D1C6F8B3
:10134000D4AD164809F088FBE2E7172D02D1C6F8A4
:10135000D87DF6E7284616F02FF827EA0000C6F8F1
:10136000D40DEEE70135182DBBD10D4803B0BDE813
:10137000F04F09F055BE00BFD8240020AA3E030854
:1013800060230308B43E0308ED3D03089F3E0308B5
:10139000BC3E0308FFFF3F00C03E0308C93E0308F0
:1013A000F53B0308BB3E03082DE9F84F05461DF049
:1013B000A1FF384F0446D7F80090B0B93648374DF2
:1013C000374F09F049FB012655F8241049B106FAB8
:1013D00004F313EA090F02D0384609F01EFB01346A
:1013E000F2E7BDE8F84F09F0B6BB02462D492846A2
:1013F000F3F7A2FB78B92C482C4C2D4D09F02CFBAF
:1014000054F8041F0029ECD00B78002BF8D02846A4
:1014100009F003FBF4E72B78DFF880B02D2B03BF36
:10142000013504F1FF344FF0010A4FF0000A0026A5
:101430005BF82680B8F1000F04D11E48BDE8F84FD4
:1014400009F0EEBD224641462846F3F775FBF8B990
:101450000120B040020604D51748BDE8F84F09F056
:10146000DFBD8305F8D4BAF1000F0AD0F2F766FCAD
:10147000124809F0F1FA41460D48BDE8F84F09F06D
:10148000EFBB40EA090038600D4809F0E5FAF2E7E1
:101490000136CDE7BC670020D13E03088024030855
:1014A000DB3E0308ED3D03089F3E03087C24030850
:1014B000BC3E0308F53B0308DF3E0308C03E0308BB
:1014C000C93E03082DE9F0478AB005461DF012FF1A
:1014D000024630B992490120FAF762F90AB0BDE834
:1014E000F08705228F492846F3F726FB0446B8B952
:1014F0008D4D0146702205F55E601FF013F8C5F8AA
:10150000C444C5F8D044C5F8DC44C5F8E844C5F87F
:10151000F444C5F80045C5F80C45C5F81845DDE7A5
:10152000042282492846F3F707FB044620BB2846DD
:1015300009F012FA07460028D0D01DF0DBFEDFF8D4
:101540001482064658F824501DB9794809F068FD00
:10155000C4E7324629463846F3F7EEFA50B920463A
:1015600009F01CFF2946734809F07AFB7248FFF71F
:10157000A9FFB3E70134E5E7072270492846F3F7EE
:10158000DBFA044600287BD1202128461EF0E1FF2B
:1015900006461DF0AFFE054680BB694809F03DFADE
:1015A0002C46684D21462846013409F036FA0E2CA7
:1015B000F8D109F0D0FA644EDFF89C91634FDFF860
:1015C0009C8100242146484609F027FADFF890A1C3
:1015D000002532680123AB40134214BF394641460F
:1015E0005046013509F019FA0E2DF2D1013409F0F7
:1015F000B2FA082C06F10C06E4D16FE7304601AAD6
:101600005349534E1EF0A9FE02AD002843D0022CD0
:1016100018D1029B072B30D803990D292DD80278B9
:10162000722A1AD06E2A28D13F4A0C2000FB0323CD
:10163000012202FA01F1D3F8C42422EA0102C3F81C
:10164000C42416E01EF050FE01AA45F824003146DD
:1016500000201EF082FE0134D7E7334A0C2000FB45
:101660000323012000FA01F1D3F8C4040843C3F8AE
:10167000C4043248FFF726FF30E709F0D7FCF8E74B
:10168000284601AA3249324E1EF067FE002402AD00
:1016900078B1082C02D109F0C9FC1FE71EF024FE26
:1016A00001AA45F82400314600201EF056FE013400
:1016B000EEE7082CEFD1029B0F2BECD8DDF80CC025
:1016C000BCF1070FE7D8049F0D2FE4D8059E06F163
:1016D0006402C82ADFD8069DFF2DDCD8079864284D
:1016E000D9D808996429D6D88842D4DA099C032C21
:1016F000D1D8C3EBC3020C4B134483F8E40D83F839
:10170000E0CD83F8E17D83F8E26D83F8E35D83F853
:10171000E51D83F8E64D0848FFF7D4FEDEE600BF7E
:10172000B8320020DF3D0308D8240020EB3E030838
:10173000F53B0308F03E03082B5E0308FA3E03085E
:10174000BE3E0308023F03089C2900203E390308DF
:101750000B3F0308F4220308985E03083E3C03088D
:10176000073F03082DE9F0474B4FDFF84481DFF8CE
:1017700044910446204609F0E7F8064630B10022BD
:1017800046490120BDE8F047FBF786BA05223946F5
:101790002046F3F7D1F958B9404B00221A601A617C
:1017A0001A621A631A641A651A661A67BDE8F08726
:1017B000042241462046F3F7BFF90546204615BBF3
:1017C00009F0CAF806460028F0D01DF093FD2C461B
:1017D0005FFA80FA59F8245025B93148BDE8F0473E
:1017E00009F01EBC524629463046F3F7A5F940B928
:1017F000204604F0BBF929462A482B4C09F030FA60
:10180000B8E70134E6E71EF06FFD072805463BD830
:10181000204609F0A1F8064648B3F2F769FF1F4BCE
:1018200003EB051383ED000A0124304609F094F818
:10183000064638B1F2F75CFF184B03EB051383ED56
:10184000010A0134304609F087F8064638B1F2F74C
:101850004FFF124B03EB051383ED020A01343046B0
:1018600009F07AF828B9BDE8F04709F0DFBB044673
:10187000DBE7F2F73DFF094B032C03EB051585ED84
:10188000030A3FF47CAFEEE7314607220748BDE884
:10189000F04709F0F2B900BFDF3D0308EC3F00203C
:1018A000F53B0308F03E03082B5E0308B13D030837
:1018B000EB3E0308F422030870B5054608460E46C1
:1018C0001DF018FD3146044602462846F3F734F968
:1018D00040B92E5D3046F3F763F900B90EB9601CCC
:1018E000284470BD0020FCE72DE9F04F0F4691B071
:1018F000B4490646FFF7E0FF0546002840F0738232
:10190000B1493046FFF7D8FF0546002840F06D8208
:10191000AE493046FFF7D0FF0546002840F0678209
:10192000AB493046FFF7C8FF002805460ABF01242F
:10193000082435460FB144F01004A64EA64FBE420F
:10194000C0F05782A54E012386F8B134EFF7CCFCE6
:10195000A3492846FFF7B0FF08B144F0200414F073
:10196000090F00F027820020FAF778F904F0180335
:10197000182B04D19B4809F06FF809F0ECF89A4B4A
:10198000DFF8CCB21A78002A984A06BF0121134624
:101990000021974A204609F0CBF92046FAF7A2F930
:1019A00096F8C83896F8505E924AA5EB0309D9F12B
:1019B00000050BEB830345EB09052946D3F83831C5
:1019C000204609F09FF996F8503E8A4A0BEB8303B4
:1019D0002946894DD3F83831204609F0A9F9D5EDCB
:1019E000007A864AF5EE407AF1EE10FA0CBF01213A
:1019F0000021204609F09CF92A4681492046FBF740
:101A00004BF9804A204602F51961F9F73BFF96F938
:101A1000E21D7D4AB1FA81F14909204609F088F9B1
:101A20007A4A204602F1D401F9F7BAFE784B1F68D2
:101A3000784BD3F800804FF000090BF5327B5BF850
:101A40002950002D40F0DC8168EA0703DFF804B27A
:101A50000693714B53F82590B9F1000F40F0F181D6
:101A6000D6F8D43DD6F8247FDFF8ECB1DFF8EC816E
:101A700006934D46DFF8E89115F80B301BB1013B9A
:101A8000012202FA03F3069A7A4033EA020214BFF3
:101A9000012600263B4007930BEB050308BF424697
:101AA000D3F808A018BF4A4653463146204609F0ED
:101AB00029F9079A5346002A0CBF4A464246314646
:101AC00020460C3509F034F9B5F5847FD4D1DFF820
:101AD00094C1524F524E0125002313F80C20D95DBA
:101AE00010A810440DF1400E00F8201C985D8644AB
:101AF0000EF8101C2DB1A2EB0008D8F1000545EB43
:101B000008050133082BE8D129460CAB454ADFF81C
:101B100058B1002720468DF8287009F0F3F808AB7B
:101B20002946404A404D204609F002F93F4A4049C3
:101B3000204609F00FF93F4A3F492046FBF748F895
:101B40003E4A3F492046F9F7B1FF3A4A3A49204612
:101B5000F9F730FF3B4A204602F5137109F072F99C
:101B6000394A204602F60D11FAF716F8374A204690
:101B700002F50B71F9F7D6FFA5F6AA184FF0190A6E
:101B800098F800102E7898F8010098F802C098F89C
:101B9000033098F804208E4240F079816E788642B6
:101BA00040F07581AE78664540F07181EE789E42D6
:101BB00040F06D812E79A6EB020EDEF1000646EBB9
:101BC0000E0653E0223F0308293F0308784103082B
:101BD000313F030880730308E0770308D82400200E
:101BE000353F03083E3F0308BC6B0020E96403084F
:101BF000933D03084E3F0308EC3F0020573F030886
